:100000000C9407090C9456090C9456090C94560943
:100010000C9456090C9456090C9456090C945609E4
:100020000C9456090C94171E0C9456090C945609FE
:100030000C9489380C9456090C9456090C94560962
:100040000C9456090C9456090C9483180C94560978
:100050000C94B10E0C9456090C947B0E0C9456091A
:100060000C9466210C9456090C940F340C94560988
:100070000C94818E0C9456090C9473870C94560939
:100080000C9456090C9456090C9456098D21922112
:100090009721A021B721CE21DE21EE212922122491
:1000A000CE21D422E522142332234F23A923042472
:1000B0001F26EC267B27FB273328D628DD2A472B53
:1000C000C12B0A2C542C822CAF2C122D5C2DA62D6A
:1000D0009F2E2E346234A53415352D356E352536D8
:1000E000EC36EC36EC36EC36EC36EC36EC36EC3600
:1000F000EC36EC36EC36A136A336A836C036C2361E
:100100008079197A9E7A007B547BBD7B12833E7C7A
:10011000627C667C667C667C667C667C667C667CD3
:10012000667C947C0F7DA47DC97D0C7E687EF37E09
:10013000DC7F358039803980398039803980398059
:100140003980398071808F80B48010814C81BB816F
:10015000E8818882E882ED82ED82ED82ED82ED8297
:10016000ED82ED82ED82D48CD78CD78CD78CE08C4D
:10017000E38CE68CF88CF58C0A0D3D3D3D3D3D3D14
:100180003D3D3D3D3D3D3D3D3D3D3D3D3D3D3D3D9F
:100190003D3D3D3D3D3D3D3D3D3D3D3D3D000A0D2F
:1001A000426174743A002025642043656C6C7320AE
:1001B00000204C6F77207761726E696E673A202558
:1001C000642E2564000A0D466F756E6420424C2D26
:1001D0004374726C3A20002564000A0D0A0D212137
:1001E000204D495353494E4720424C2D4354524CC5
:1001F0003A202564202121000A0D43616C69627256
:100200006174696E672070726573737572652073AF
:10021000656E736F722E2E004F4B0A0D000A0D464D
:100220006C696768742D74696D65202575206D692A
:100230006E20546F74616C3A2575206D696E0041B3
:100240006E676C654E69636B202020202020204162
:100250006E676C65526F6C6C20202020202020413E
:1002600063634E69636B20202020202020202041E2
:100270006363526F6C6C20202020202020202059A6
:1002800061774779726F202020202020202020488D
:1002900065696768742056616C756520202020416F
:1002A00063635A2020202020202020202020204767
:1002B0006173202020202020202020202020204387
:1002C0006F6D706173732056616C756520202056C8
:1002D0006F6C74616765205B302E31565D20205253
:1002E00065636569766572204C6576656C2020478C
:1002F00079726F20436F6D70617373202020204DE1
:100300006F746F7220312020202020202020204D6B
:100310006F746F7220322020202020202020204D5A
:100320006F746F7220332020202020202020204D49
:100330006F746F7220342020202020202020203154
:100340003620202020202020202020202020203186
:100350003720202020202020202020202020203175
:100360003820202020202020202020202020203164
:100370003920202020202020202020202020205331
:100380006572766F20202020202020202020204809
:100390006F76657267617320202020202020204323
:1003A000757272656E74205B302E31415D20204382
:1003B00061706163697479205B6D41685D202048DC
:1003C000656967687420536574706F696E74203254
:1003D00035202020202020202020202020202032F6
:1003E00036202020202020202020202020202043D4
:1003F0006F6D7061737320536574706F696E7449AB
:1004000032432D4572726F7220202020202020421E
:100410004C204C696D69742020202020202020472A
:1004200050535F4E69636B202020202020202047FE
:1004300050535F526F6C6C20202020202020202100
:10044000212120494E434F4D50415449424C4520B3
:10045000212121002A002E000A0D20444143206F53
:100460007220493243204552524F52212043686541
:10047000636B204932432C2033567265662C20442E
:10048000414320616E6420424C2D4374726C005BCA
:1004900025695D005B25695D002B204D696B726FDE
:1004A0004B6F70746572202B0048573A5625642EA6
:1004B00025642053573A25642E256425630053652F
:1004C0007474696E673A2564202573004D697865F8
:1004D00072204572726F7221004552522532643A81
:1004E000004861726477617265204572726F722094
:1004F000313A2564202121004D697373696E6720AC
:10050000424C2D4374726C3A2564212100493243D8
:10051000204552524F522121210048656967687475
:100520003A202025356900536574706F696E743AFE
:100530002535690050726573737572653A253569A2
:10054000004F66667365743A20202535690048655A
:100550006967687420636F6E74726F6C00444953EE
:1005600041424C4544006163742E206265617269AA
:100570006E67004E69636B3A2020202020202535CD
:100580006900526F6C6C3A202020202020253569AC
:1005900000436F6D706173733A2020202535690028
:1005A0004B25693A25346920204B25693A25346961
:1005B00020004E693A2534692020526F3A2534696B
:1005C000200047733A253469202047693A25346969
:1005D000200050313A253469202050323A253469C0
:1005E000200050333A253469202050343A253469AC
:1005F00020004779726F202D2053656E736F720053
:100600004E69636B25346920282533692E256929B5
:1006100000526F6C6C25346920282533692E2569BA
:100620002900476965722534692028253369290026
:100630004E69636B2025346920282533692E25787F
:100640002900526F6C6C2025346920282533692ECF
:100650002578290059617720202534692028253301
:100660006929004E69636B20253469202825336988
:1006700029282533692900526F6C6C2025346920A4
:1006800028253369292825336929005961772020D5
:100690002534692028253369292825336929004113
:1006A0004343202D2053656E736F72004E69636B58
:1006B0002025346920282533692900526F6C6C206D
:1006C000253469202825336929005A202020202537
:1006D000346920282533692900566F6C7461676579
:1006E0003A2020202533692E253169560043757242
:1006F00072656E743A2020202533692E25316941B8
:1007000000506F7765723A202020202025346957E9
:10071000004469736368617267653A202535696DC5
:1007200041680052656365697665720052432D52D7
:100730005353493A202020202534690052432D513B
:1007400075616C6974793A202534690052432D43F0
:1007500068616E6E656C733A25346900436F6D7025
:10076000617373004D61676E65743A2020202535F2
:1007700069004779726F3A202020202025356900D2
:10078000536574706F696E743A2025356900506F37
:10079000746925693A202025336900506F746925F2
:1007A000693A202025336900536572766F20200056
:1007B000536574706F696E74202025336900506F23
:1007C000736974696F6E3A202533690052616E67F0
:1007D000653A2533692D25336900424C2D437472E7
:1007E0006C204572726F72732000253364202533AC
:1007F0006420253364202533642000424C20546556
:100800006D706572617475726500253364202533DF
:100810006420253364202533642000424C2D43742A
:10082000726C20666F756E64200020256320202086
:1008300025632020202563202020256320002025FB
:10084000632020202563202020256320202025638D
:1008500020002025632020202D2020202D20202056
:100860002D2000313000313100313200466C696793
:1008700068742D54696D65202000546F74616C3A62
:100880002535756D696E004163743A2020253575F4
:100890006D696E0028726573657429000A0D4765DD
:1008A0006E65726174696E672064656661756C74EB
:1008B00020506172616D65746572205365742025E6
:1008C00064000A0D5573696E6720506172616D6531
:1008D00074657220536574202564000A0D47656EA7
:1008E00065726174696E672064656661756C7420F9
:1008F0004D69786572205461626C65000A0D4D691E
:100900007865722D436F6E6669673A2027257327D5
:1009100020282575204D6F746F727329000A0D41D0
:100920004343206E6F742063616C69627261746509
:1009300064210D0A0000008F001E01AD013B02CAB8
:10094000025803E603740402058F051B06A706334D
:1009500007BE074808D2085B09E3096B0AF20A7868
:100960000BFD0B810C040D860D070E870E060F8400
:100970000F00107B10F5106E11E5115B12CF1242C3
:1009800013B31323149214FE146A15D3153B16A146
:100990001605176717C81727188318DE1837198E1A
:1009A00019E319361A871AD61A231B6E1BB61BFDBC
:1009B0001B411C831CC31C001D3C1D751DAB1DE091
:1009C0001D121E421E6F1E9A1EC31EE91E0D1F2EF3
:1009D0001F4D1F691F841F9B1FB01FC31FD31FE123
:1009E0001FEC1FF51FFB1FFF1F0020040100001F4D
:1009F0007200020101487301030202DC7302040366
:100A00000384740300040439742532692E25316986
:100A10005600253364256320253033646D2563003B
:100A2000537461747573004552524F523A20253207
:100A3000642000253469202532693A253032690066
:100A40002534696D25630025336920253369202508
:100A50003369202533690025336920253369202532
:100A60003369202533690054656D70657261747552
:100A70007265732020202000256343202020202041
:100A8000002532692E25316956202533692E2531FE
:100A900069410025346957202536696D4168004D4C
:100AA00061676E65743A25336925252025336925EC
:100AB0006300496E636C692E3A25336925632028EB
:100AC00025692920002532756D2F73205361743AF2
:100AD0002564200020203344004E6F4678004447B0
:100AE000505300486F6D653A2533646D202533649B
:100AF0002563202563004E6F204E61766943747232
:100B00006C21004E6F204572726F722020202020D1
:100B1000202020004E6F7420636F6D7061746962D5
:100B20006C652020004D4B334D6167206E6F742043
:100B3000636F6D7061004E6F20464320636F6D6D73
:100B4000756E69636174004D4B334D616720636F4F
:100B50006D6D756E6963610047505320636F6D6DF5
:100B6000756E69636174696F00636F6D7061737333
:100B70002076616C75652020200052432053696700
:100B80006E616C206C6F737420200046432073707C
:100B900069207278206572726F7220004E6F204E4D
:100BA0004320636F6D6D756E696361740046432009
:100BB0004E69636B204779726F20202020004643E6
:100BC00020526F6C6C204779726F202020200046E5
:100BD0004320596177204779726F20202020200020
:100BE0004643204E69636B20414343202020202050
:100BF00000464320526F6C6C20414343202020204C
:100C000020004643205A2D4143432020202020200D
:100C100020200050726573737572652073656E7362
:100C20006F7220004932432046432D3E424C2D43F3
:100C300074726C2000426C204D697373696E67207A
:100C40002020202020004D69786572204572726F47
:100C50007220202020200043617265667265652045
:100C60004572726F722020004750532046697820E9
:100C70006C6F737420202020004D61676E657420B6
:100C80004572726F7220202020004D6F746F7220A9
:100C90007265737461727420202000424C204C698C
:100CA0006D69746174696F6E202020004750532075
:100CB00052616E676520202020202020004E6F208A
:100CC00053442D436172642020202020200053448F
:100CD0002D4C6F6767696E67206572726F72004690
:100CE0006C79696E672072616E6765212020200033
:100CF0004D617820416C74697475646521202020F1
:100D00000020202020202020202020202020202003
:100D10002020202020200020202532692E25316926
:100D20005620200020202532692E253169562020AA
:100D300000414C543A2534696D20256300414C54E0
:100D40003A2534696D202000414C543A2D2D2D2D2B
:100D5000200020202532693A2530326920200020E9
:100D6000202532693A253032692020004449523A20
:100D700020253364256300430020002020253569A9
:100D80002020002020253569202000493A2532699D
:100D90002E2531694120003A003A003A002D2D2DD0
:100DA0002D2D2D2D2D2D2B2D2D2D2D2D2D2D2D2D75
:100DB0002D2D002D2D2D2D2D2D2D2D2D2D2D2D2D90
:100DC0002D2D2D2D2D2D2D2D003A005341543A253A
:100DD00032642000444953543A2533646D00442062
:100DE000003344002121004D41473A253375252524
:100DF0002000484D3A253364256320256300696E41
:100E0000636C3A2532642563282532692900202045
:100E100020202532756D2F733A2020484D3A253316
:100E2000642563202563004552523A202532642010
:100E300021004552523A2000207777772E4D696B7A
:100E4000726F4B6F707465722E64652020002025D0
:100E500032693A2530326920202532692E253169E0
:100E600056202534696D416800202532693A2530C5
:100E7000326920202532692E2531695620253469B2
:100E80006D4168004449523A253364256300414C62
:100E9000543A2534696D00414C543A2534696D004B
:100EA000414C543A2D2D2D2D2000256300484D3AFC
:100EB00025336425632020444953543A2533646D17
:100EC000202563005057523A2532692E2531694159
:100ED000202825695729200043460020200047503C
:100EE000533A2532756D2F73205341543A256420AF
:100EF000002020334420004E4F46495800444750BC
:100F00005320002020204E6F204E6176694374727A
:100F10006C20202020202020002532692E256920E9
:100F20002532692E2569202532692E256920253232
:100F3000692E256941002533692025336920253331
:100F40006920253369256343002532692E256920F0
:100F50002532692E256941002532692E2569202513
:100F600032692E2569202532692E256920253269AE
:100F70002E256941002533692025336925634320E7
:100F800020202020202020002533692025336920BF
:100F900025336920253369256343004552523A20A1
:100FA0002532642021004552523A2000207777777D
:100FB0002E4D696B726F4B6F707465722E64652075
:100FC000200053657474696E673A25752025732077
:100FD000004D696E3A2532692E25316956202573F8
:100FE0002000414C543A00504F54493A2533752063
:100FF00000284F4E29202000284F46462920004C2B
:10100000494D495400564152494F004449534142C9
:101010004C45440043463A0044495341424C454400
:101020000020284F4E29200020284F464629002026
:101030005445414348004750533A004449534142C4
:101040004C4544002846524545290028484F4D4507
:1010500029002841494429200028484F4C442900B0
:101060002046533A257573656B2000484F4D452047
:10107000414C543A0025756D00484F4C4420004EB9
:10108000693A25346920526F3A25346920433A255C
:1010900033690047733A2534692059613A25346928
:1010A000200050313A2534692050323A25346920E5
:1010B000333A2533690050343A2534692050353AA3
:1010C00025346920363A25336900434F55504C4941
:1010D0004E47204F46462120004C4F4F50494E4727
:1010E0002120004848212000434F4D5041535320B8
:1010F0004F46462120000A0D7777772E4D696B7297
:101100006F4B6F707465722E6465202863292048C8
:101110006953797374656D7320476D6248000A0DD9
:1011200074686520757365206F6620746869732024
:10113000736F667477617265206973206F6E6C7966
:10114000207065726D6974746564200A0D6F6E207D
:101150006F726967696E616C204D696B726F4B6F5E
:10116000707465722D4861726477617265005573A1
:10117000657200486F545420563300414354204454
:10118000534C004A657469005370656B7472756DD9
:101190000050504D000A0D52656365697665723ADC
:1011A0002000532E42757300756E6B6E6F776E2E36
:1011B000205573696E672050504D2E2E2E006E6F95
:1011C0007420737570706F72746564206279206822
:1011D0006172647761726521000A0D466C69676807
:1011E00074436F6E74726F6C0A0D4861726477613C
:1011F00072653A25642E25640A0D536F6674776113
:1012000072653A5625642E2564256320000011245A
:101210001FBECFEFD0E4DEBFCDBF11E0A0E0B1E054
:10122000E0ECF2E201E00BBF02C007900D92AE3A93
:10123000B107D9F71AE0AEEAB1E001C01D92A235BC
:10124000B107E1F77AEAE2E0F0E081E2809357004B
:10125000D4907E010894E11CF11C20EF37EF41E0AF
:1012600050E087016FE0DA01C9012F5F3F4F4F4F18
:101270005F4FABBFFC018791F80181938F016150F3
:1012800067FFF1CFF7016EE081917827709561508B
:1012900067FFFACF8889781729F0F7E9DF1611F48C
:1012A0000000FECF0E94290A0C945F910C9400006C
:1012B00088E791E09F938F9387E695E19F938F93C3
:1012C000E0911304F091140409950F900F900F9082
:1012D0000F90089580916006E82FFF27EE0FFF1F03
:1012E000EE56F84F808191818D5E9F4F14F01092E1
:1012F0000201808191818A5B9F4FCCF48091020131
:101300008823A9F481E080930201809147048F5FD4
:1013100080934704853038F088EE93E09093EE0197
:101320008093ED0104C066E970E00E94233C809147
:10133000470499279093DF058093DE0508951F9356
:10134000CF93DF93182F882389F08EE991E09F9344
:101350008F9387E695E19F938F93E0911304F0912B
:10136000140409950F900F900F900F9080918306B1
:10137000823308F044C084EF91E00E947619EC01BA
:10138000112329F0CE010E947F198823D9F3C2E0EE
:10139000D0E026E530E0809125019091260182176A
:1013A000930730F02196255D3F4FC730D10598F364
:1013B000809183069927C89F9001C99F300DD89FBF
:1013C000300D1124209300011123D9F068EC70E056
:1013D0008C2F0E94233CDF93CF9386EA91E09F936A
:1013E0008F9387E695E19F938F93E0911304F0919B
:1013F000140409958DB79EB706968DBF02C08093E1
:101400000001112311F1809100016AE00E94B29065
:10141000892F99279F938F93809100010E94B2900A
:1014200099279F938F9381EB91E09F938F9387E60A
:1014300095E19F938F93E0911304F0911404099523
:101440002DB73EB7285F3F4F2DBFDF91CF911F9142
:101450000895CFEFD0E4DEBFCDBF8824992414B81F
:1014600015B8B7EEEB2EB3E0FB2E2EEC3FEFE20EFD
:10147000F31EF7FEFACF85E18093010181E887B979
:101480003E9A8FEF88B98BE184B911E015B98EE3EC
:101490008AB987E48BB9469A84B7877F84BF8091E5
:1014A00060008861809360001092600084EC99E095
:1014B0009093EE018093ED011092F9021092F802E0
:1014C00010929707109296071092FB021092FA0260
:1014D0001092FD021092FC0284EC94E0A0E0B0E0D7
:1014E00080934A0190934B01A0934C01B0934D011E
:1014F00028980E94DF190E94B0190E946F150E945F
:1015000060380E94F71F812F0E94C3330E94E56953
:101510000E9473750E944C8D809101018C3010F4F3
:10152000299A01C0299878940E94E23289E1809337
:10153000120410921104809134028260809334026C
:10154000109237020E94554784EF91E00E9476196D
:101550007C018091340280FD05C0C7010E947F1983
:101560008823B9F385EC91E09F938F93A7E6AA2E89
:10157000A5E1BA2EBF92AF92E0911304F09114044A
:10158000099580EA9FE00E9476197C0100E010E056
:101590000F900F900F900F90C4E3D7E0F8EECF2E8E
:1015A000F6E0DF2E0E9455478091340280FD05C091
:1015B000C7010E947F198823B9F3F60180811816AC
:1015C000A4F40BC00E9455478091340280FD05C0F1
:1015D000C7010E947F198823B9F3C7010E947F19B0
:1015E000882319F4888188236CF7888187FF1BC0C2
:1015F0000F5F1F4F1F930F930150104087ED91E035
:101600009F938F93BF92AF92E0911304F0911404D3
:1016100009958091AF018F5F8093AF012DB73EB7E1
:101620002A5F3F4F2DBF0F5F1F4F84E090E0C80E31
:10163000D91E28960C30110508F4B4CF00E010E054
:10164000C1E3D7E0E8EEEE2EE6E0FE2E8B8187FDCB
:1016500022C0F70180811816F4F40F5F1F4F1F930B
:101660000F93015010408AED91E09F938F9387E68E
:1016700095E19F938F93E0911304F09114040995E1
:1016800082E08093EB0181E0809311042DB73EB797
:101690002A5F3F4F2DBF8B8180788B830F5F1F4F59
:1016A00084E090E0E80EF91E28960C30110570F2E7
:1016B0000E94580990915E068091AF01981728F416
:1016C00080912D04806180932D0488EF91E09F9399
:1016D0008F93C7E6D5E1DF93CF93E0911304F091A8
:1016E0001404099588EE93E00E9476197C010E940B
:1016F000FD1F0F900F900F900F90C7010E947F1950
:101700008823D9F388E192E09F938F93DF93CF935F
:10171000E0911304F0911404099580E00E94F23CDA
:10172000809101010F900F900F900F908A3011F06F
:10173000843110F0289801C0289A80ED97E09093AA
:10174000EE018093ED0185E5809349048EE090E001
:101750000E9406319927182F00278FE090E00E9401
:101760000631080F111D1093B5010093B4018AE0F2
:1017700090E00E9406319927182F00278BE090E017
:101780000E940631080F111D1093B3010093B2019E
:101790000F5F1F4F39F08091B4019091B5018F5FB9
:1017A0009F4F41F41092B5011092B4011092B30111
:1017B0001092B2018091B2019091B3019F938F93E7
:1017C0008091B4019091B5019F938F938DE192E048
:1017D0009F938F93DF93CF93E0911304F0911404C0
:1017E00009950E94912588E893E1909345018093A3
:1017F0004401C1E0C09348048C2F0E949F0980914E
:1018000086060E94988C0E94580980ED97E00E94FD
:1018100076197C018AEF90E00E94761983E080932C
:10182000B6051092AE018091CC062DB73EB7285F69
:101830003F4F2DBF84FF02C0C093B6018091B80115
:10184000882311F04798FECF8091F101882309F495
:101850004AC280911701882309F445C21092F10110
:1018600080914704882319F00E946A0902C00E94EF
:10187000854A0E945547209101012A3011F02431F8
:1018800010F0289801C0289A8091EC02882331F04A
:101890008091EC0281508093EC020EC080916F0029
:1018A000806280936F00109293071092920780914C
:1018B0002D04886080932D0480914401909145010E
:1018C0000197909345018093440180914401909148
:1018D0004501892B21F0809135028823C9F180913F
:1018E000440190914501892BD9F40E94ED3385E0A4
:1018F00090E090934501809344018091F005909190
:10190000F10501969093F1058093F00580912D04E7
:10191000816080932D048091B70582608093B70524
:1019200080910701909108018F5F9F4FC1F48091D2
:10193000EB028823A1F088EA91E69093EE01809370
:10194000ED0180E890E0909308018093070107C0C3
:101950002A3011F0243110F0289801C0289A0E94F2
:10196000048E8091F101882309F0BDC18091F803B4
:10197000882319F00E949683B6C1809111018823B3
:1019800011F00E948D1A0E94B3150E9401110E944D
:101990006E1AC7010E947F19882309F4A0C184E14F
:1019A00090E0E80EF91E0E94F61980911204882337
:1019B00061F080911204815080931204809112048E
:1019C000882319F481E08093E801809186068630AF
:1019D00011F40E94447980913502882349F0809166
:1019E0002D04826080932D048091B70582600FC022
:1019F0008091ED019091EE01892B59F48091440181
:101A000090914501079728F08091B7058D7F8093CD
:101A1000B7058091B601882361F08091EC02873987
:101A200040F01092B60188E893E19093EE01809324
:101A3000ED0180910401882321F0815080930401FD
:101A40002EC0809353041092C0021092BF021092D5
:101A5000BE021092BD021092BC021092BB02809195
:101A6000EC028823E1F480910701909108018F5FD7
:101A70009F4FA9F42091B601223089F088E99AE3BA
:101A80009093EE018093ED0180E09CE0909308013B
:101A900080930701222319F082E08093B6018091A0
:101AA000A301893C48F081508093A30180912D04CB
:101AB0008B7F80932D043FC0809173088823F9F0B9
:101AC00080912D04846080932D0489E08093C60367
:101AD00080910701909108018F5F9F4F81F4809161
:101AE000EB02882361F088E99AE39093EE018093FA
:101AF000ED0180E098EA909308018093070110922D
:101B0000B8031092B7031092B6031092B503109267
:101B1000B403109266081092A5081092A4081092BF
:101B2000A7081092A6088FEF9FEF9093A3088093C9
:101B3000A2081092A30180910001282F33278091E1
:101B400025019091260182179307CCF48091B4026D
:101B500080628093B40280910701909108018F5FA9
:101B60009F4FC1F480E797E19093EE018093ED01E0
:101B700080E093E090930801809307010BC080916F
:101B8000ED019091EE01892B29F48091B4028F7DB3
:101B90008093B4020E94A76E84E08093EC01809150
:101BA000B7018F5F8093B701813309F04FC0109266
:101BB000B7018091B40281FF0AC08091B001909179
:101BC000B10101969093B1018093B0013FC05AEAF0
:101BD000852E55E0952E80910306909104069C0178
:101BE000442737FD4095542F80911D0190911E018F
:101BF000A0911F01B0912001281739074A075B0700
:101C000034F4809103069091040601961BC08091E4
:101C10000306909104069C01442737FD4095542FFC
:101C200080911D0190911E01A0911F01B091200192
:101C300082179307A407B5074CF48091030690918F
:101C40000406019790930406809303060894811C70
:101C5000911C32E783163BE0930609F040C08824CC
:101C600099242091B4013091B5012F5F3F4F3093FB
:101C7000B5012093B4018091B2019091B301019616
:101C80009093B3018093B201832F9927682F8EE040
:101C900090E00E940E318091B4019091B501907056
:101CA000682F8FE090E00E940E318091B2019091F8
:101CB000B301892F9927682F8AE090E00E940E31A6
:101CC0008091B2019091B3019070682F8BE090E009
:101CD0000E940E3184E190E00E9476197C010E94FE
:101CE000F76E0E948A758091EC01882309F0A6CDD9
:101CF0000E94066AA3CD1F920F920FB60F92112475
:101D00008F939F93EF93FF93809106018823E1F4D3
:101D10008091D2019091D30101969093D301809349
:101D2000D201FC01E95FFA4FE081ED3019F08F3A02
:101D3000910539F41092D3011092D20181E0809381
:101D40000601E093C60004C01092D3011092D201A4
:101D5000FF91EF919F918F910F900FBE0F901F9069
:101D600018951F920F920FB60F9211242F933F9345
:101D70004F935F936F937F938F939F93AF93BF9393
:101D8000CF93EF93FF9390E08091B801813029F4D5
:101D90008091C6008093CE00CCC08091B801823083
:101DA00029F48091C60080935604C3C08091C60078
:101DB0008093CA015091D8015F3A10F09093D901F5
:101DC0008091CA018D3009F065C08091D9018230BF
:101DD00009F060C09093D901852F99278A5A9B4FAB
:101DE000FC01329740812091D4013091D501241B10
:101DF0003109DC0111978C91281B3109C9019F70B1
:101E00009093D5018093D40146E0969587954A95A5
:101E1000E1F7982F935C9093D6012F733070235C79
:101E20002093D7018081981729F48C91281711F4F9
:101E300091E006C090E08091C7018F5F8093C70159
:101E4000C091C901CC2309F074C0992309F471C071
:101E500081E08093C901580F5093C6015150E52F7E
:101E6000FF27EA5AFB4F8DE080838091580482352A
:101E700009F05FC00E94912588E190E02CE00FB648
:101E8000F894A895809360000FBE20936000C093E3
:101E9000EB014FC02091D901822F99278130910504
:101EA000F9F0823091051CF4892B21F040C0029793
:101EB00011F13DC08091CA01833239F48091C9018A
:101EC000882319F481E08093D9018091CA0180931D
:101ED000560481E08093D8018091CA01992722C0DD
:101EE0002F5F2093D901E52FFF27EA5AFB4F8091FE
:101EF000CA01808309C0E52FFF27EA5AFB4F809172
:101F0000CA0180835F3A20F45F5F5093D80102C01A
:101F10001092D9012091CA018091D4019091D501EC
:101F2000820F911D9093D5018093D40102C010922D
:101F3000D901FF91EF91CF91BF91AF919F918F9177
:101F40007F916F915F914F913F912F910F900FBEB5
:101F50000F901F901895AC01A0E0B0E09D01A8176C
:101F6000B90748F4E7E0F5E08191280F311D11969B
:101F7000A417B507C8F33F70FD01E95FFA4FC90127
:101F800056E0969587955A95E1F7835C8083119684
:101F9000FD01E95FFA4F2F733070822F835C8083DD
:101FA000A85FBA4F8DE08C931092060180910705CF
:101FB0008093C6000895A0E0B0E0E1EEFFE00C944D
:101FC0002B912C859D850E85BB2483E2809307058C
:101FD0009F59909308052093090533E0E32EF12CD7
:101FE000002309F49EC0CF84D888BE016D5E7F4F68
:101FF000A989BA890150109709F493C01097B9F0D4
:10200000F601EB0DF11DB3949081119791F400232B
:1020100049F1FB016E5F7F4FDB01C080D1806E5FB5
:102020007F4F0D90BC91A02DBB24015002C090E0C9
:1020300019C01097B9F0F601EB0DF11DB394408172
:10204000119791F4002341F1FB016E5F7F4FDB019B
:10205000C080D1806E5F7F4F0D90BC91A02DBB24BE
:10206000015002C040E018C01097B1F0F601EB0D2E
:10207000F11DB3941081119781F4002371F0FB01DD
:102080003296DB01CD90DC90BF016E5F7F4FA08167
:10209000B181BB24015001C010E0F701E95FFA4FA4
:1020A000892F86958695835C80830894E11CF11CBA
:1020B000F701E95FFA4F892F99278370907024E028
:1020C000880F991F2A95E1F755279A0194E03695D4
:1020D00027959A95E1F7822B835C80830894E11C15
:1020E000F11CF701E95FFA4F4F705070440F551F14
:1020F000440F551F812F992726E0969587952A959D
:10210000E1F7842B835C80830894E11CF11CF701C8
:10211000E95FFA4F1F73135C10830894E11CF11CF4
:102120006ACFC7010E94AB0FE9E00C944791A3E08E
:102130007A2F4091C6014650442309F458C0E72F36
:10214000FF27EA5AFB4F80818D537F5FE72FFF27E0
:10215000EA5AFB4F20812D537F5FE72FFF27EA5A72
:10216000FB4F30813D537F5FE72FFF27EA5AFB4F3C
:1021700060816D537F5F9927880F991F880F991F82
:10218000522F52955F70582B822F99278F70907025
:10219000F4E0880F991FFA95E1F7232F26952695ED
:1021A000282B832F992783709070E6E0880F991F62
:1021B000EA95E1F7682B41504F3FC9F0EA2FFF271E
:1021C000EA5AFB4F5083AF5F41504F3F81F0EA2FF7
:1021D000FF27EA5AFB4F2083AF5F41504F3F39F052
:1021E000EA2FFF27EA5AFB4F6083AF5FA5CF89E54F
:1021F00094E09093C5018093C401A350A093C301C0
:102200000895A2E0B0E0E7E0F1E10C943191809113
:10221000C901882309F457C40E949710809157047C
:10222000823609F023C3809158049927803791059D
:1022300009F4AFC081379105C4F48A36910509F4D9
:1022400080C28B36910544F48B34910571F186364A
:10225000910509F45FC10AC38D36910509F469C07F
:102260008E36910509F44DC001C38437910541F1C3
:10227000853791054CF48137910509F491C0833776
:10228000910509F4DFC0F2C28737910509F41BC23A
:10229000883791052CF48537910509F4D7C1E6C23A
:1022A0008937910509F46DC1E1C2E091C401F09153
:1022B000C501808191819093970180939601D6C248
:1022C0008091C601A091C401B091C501853140F053
:1022D00080E1E1E3F4E00D9001928A95E1F70DC011
:1022E0008D919D910D90BC91A02D80933104909380
:1022F0003204A0933304B093340480EF8093C1017F
:102300004BC0809106018823E1F38DE490E09F9318
:102310008F938BED96E09F938F9381E08F938F93B4
:102320008EE48F930E94DB0F8DB79EB707968DBF0B
:102330009DC2A091C401B091C5011C91113081F4DE
:102340008DE4EBEDF6E00D9001928A95E1F70E94A5
:102350001F32198380912D048F7E80932D0401C03C
:102360001982809106018823E1F381E090E09F9338
:102370008F93CE0101969F938F9381E08F938F93DC
:102380008DE48F930E94DB0FADB7BEB71796ADBF3C
:102390006DC281E08093CC018FEF8093040166C20F
:1023A000E091C401F091C501E0818E2F8A508A30FE
:1023B00058F48983882311F481E003C0863010F03B
:1023C00085E0898361E00EC08E2F84518A3070F4DD
:1023D0008983882311F481E003C0863010F085E002
:1023E000898360E089810E949F3212C0E983EF3FB8
:1023F00019F40E94823289838981882311F481E053
:1024000003C0863010F085E0898389810E942431E1
:10241000809106018823E1F38BE790E09F938F93EF
:102420008FE596E09F938F9381E090E09F938F9349
:10243000CE0101969F938F9382E08F9381E08F93DB
:1024400081E577C12091C4013091C501D9018C91FA
:102450008150853008F045C0F90181818A3509F045
:1024600040C08091EB028823E1F52F5F3F4F8BE75F
:10247000EFE5F6E0D9010D9001928A95E1F7F901B7
:1024800082910E948F318091A0069927AA27BB27AD
:10249000BC01CD0124EC39E040E050E00E94939073
:1024A000DC01CB0180938E0190938F01A09390016A
:1024B000B09391018091A1069927AA27BB27BC015F
:1024C000CD010E949390DC01CB0180938A0190930F
:1024D0008B01A0938C01B0938D010E94823289837D
:1024E00001C01982809106018823E1F381E090E028
:1024F0009F938F93CE0101969F938F9381E08F934B
:102500008F9383E58F930E94DB0F8DB79EB707965D
:102510008DBF26C0E091C401F091C501E0818E2FEE
:102520008150853018F48E2F0E9424310E9482320F
:102530008983809106018823E1F381E090E09F93F5
:102540008F93CE0101969F938F9381E08F938F930A
:1025500086E48F930E94DB0FADB7BEB71796ADBF71
:102560008091EB02882329F46EE670E089810E9455
:10257000233C80E00E949F09809186060E94988CEF
:1025800075C1E091C401F091C5018081992787FD53
:1025900090959093AD078093AC078181992787FD33
:1025A00090959093AF078093AE078281992787FD1E
:1025B00090959093B1078093B0078381992787FD09
:1025C00090959093B3078093B2078481992787FDF4
:1025D00090959093B5078093B4078581992787FDDF
:1025E00090959093B7078093B6078681992787FDCA
:1025F00090959093B9078093B8078781992787FDB5
:1026000090959093BB078093BA078085992787FDA3
:1026100090959093BD078093BC078185992787FD8E
:1026200090959093BF078093BE078285992787FD79
:1026300090959093C1078093C0078385992787FD64
:1026400090959093C3078093C20710C1E091C40195
:10265000F091C50180810E94B9378A83882319F4DB
:1026600081E0898301C01982809106018823E1F30A
:1026700088E090E09F938F9389E297E09F938F93F8
:1026800021E030E03F932F938091C4019091C501E8
:102690009F938F933F932F93CE0102969F938F9397
:1026A0003F932F93CE01820F931F9F938F9384E0CC
:1026B0008F9381E08F9385E58F930E94DB0FEDB7B9
:1026C000FEB773963CC08091C301893008F4CEC038
:1026D0002091C4013091C5012F5F3F4F88E0A9E2EE
:1026E000B7E0F90101900D928A95E1F7D9018E9139
:1026F0000E940F378A83882319F481E0898301C0FF
:102700001982809106018823E1F321E030E03F93B4
:102710002F93CE0102969F938F933F932F93CE01D9
:10272000820F931F9F938F9382E08F9381E08F930B
:1027300087E58F930E94DB0FEDB7FEB73B96EDBFA9
:1027400095C08091EB02882309F090C00E944B8CC9
:102750008983823019F0843009F088C020E430E0A9
:10276000F8948091C1008F738093C1008091C9005B
:102770008F738093C9008091C100877E8093C100D0
:102780008091C900877E8093C9008091C80087FF2F
:1027900003C08091CE00F9CF8091C00087FF03C0B5
:1027A0008091C600F9CFE091C401F091C501E081AC
:1027B000E13021F482E08093B8012EC0E43611F4B8
:1027C00021E830E081E08093B801832F992780933E
:1027D000CD002093CC008091CD008093C5008091E6
:1027E000CC008093C4008091CA008F7D8093CA0082
:1027F0008091CA008F7E8093CA008091C9008B7F30
:102800008093C9008091CA0084608093CA0080913F
:10281000CA0082608093CA008091CA00877F80933B
:10282000CA008091C200877F8093C2008091C90056
:102830008E7F8093C9008091C10088618093C10020
:102840008091C90088618093C9008091C10080682F
:102850008093C1008091C90080688093C900109264
:102860006E0010926F00109270007894809158045E
:1028700099278436910509F4BBC085369105ACF4DF
:102880008136910509F46FC0823691052CF48B34A2
:10289000910509F45DC00FC18236910509F470C03D
:1028A0008336910509F47FC006C18C36910509F481
:1028B000EDC08D3691054CF48736910509F4F8C0CA
:1028C0008836910509F4B2C0F6C08437910529F025
:1028D0008637910509F4E8C0EEC08091C601A09149
:1028E000C401B091C501803140F080E1E1E3F4E042
:1028F0000D9001928A95E1F70DC08D919D910D90FB
:10290000BC91A02D8093310490933204A0933304A2
:10291000B0933404809106018823E1F31F928091E3
:1029200003018F9384E58F930E94DB0F8AEF8093DE
:10293000C1018FEF8093040180EA9FE00E94761925
:102940009093BA018093B9010F900F900F90B3C08C
:10295000E091C401F091C50180819181909397012C
:1029600080939601A8C0E091C401F091C5018081D7
:1029700080930501803298F08FE1809305010FC0AC
:10298000A091C401B091C5018BE0E9E4F4E00D90A1
:1029900001928A95E1F7809152048093F8058FEFB8
:1029A0008093040188C08091BD019091BE01892B64
:1029B00089F4E091C401F091C501E081EE2351F06A
:1029C0008AE0E89FC00111240E94761990932404A4
:1029D00080932304E091C401F091C50190818AE0C5
:1029E000989FC00111249093BE018093BD0115C032
:1029F0008FEF80930401E091C401F091C5019081B3
:102A00008AE0989FC00111249093C0018093BF0178
:102A1000892B19F081E08093CE0180EA9FE00E942B
:102A200076199093BA018093B90145C08FEF8093D6
:102A30000401E091C401F091C501908197FD08C0A7
:102A400082E08093CB011092BC011092BB011AC0AE
:102A5000909580912D02892B80932D0291818AE09F
:102A6000989FC00111249093BC018093BB0184E026
:102A70008093CB0180EA9FE00E9476199093BA017F
:102A80008093B90181E08093CF0115C08FEF8093CF
:102A90000401E091C401F091C501808180932E0270
:102AA00081E08093D00107C081E08093CD0103C015
:102AB00081E08093D1011092C9011092C50110925A
:102AC000C4011092C301E3E0CE5F0C944D91982FA6
:102AD0008091C00085FFFCCF9093C60008950F93AE
:102AE0001F9388E18093C1008091C0008260809331
:102AF000C0008091C10080688093C1008091C100B6
:102B000080648093C10000E010E00093C5008AE279
:102B100090E08093C4008091BF019091C0010E9419
:102B2000761990932604809325048CED90E00E9402
:102B3000761990935504809354041092270488E5E5
:102B40008093280485E080932B048BE080932904F4
:102B500010922A041093C5010093C4011092C3017E
:102B60001F910F910895A0E1B0E0E9EBF5E10C941D
:102B70002E9180910601882309F4C1C28091B90188
:102B80009091BA010E947F19882361F01092BC01D4
:102B90001092BB011092C0011092BF011092BE01B1
:102BA0001092BD018091BB019091BC01892B41F035
:102BB00080910505909106050E947F19882329F4CC
:102BC0008091CF01882309F460C080910601882399
:102BD00009F45BC08091CB010EE016E08430A8F0D0
:102BE0000E94A72580E590E09F938F931F930F93FA
:102BF00081E08F938F9388E48F930E94DB0F2DB732
:102C00003EB7295F3F4F2DBF34C010922F028FE394
:102C100094E09F938F938AE995E29F938F93E0913D
:102C20001304F0911404099584E190E09F938F932D
:102C30001F930F9381E090E09F938F938BEC91E033
:102C40009F938F9382E08F9381E08F9388E48F939B
:102C50000E94DB0F8091CB01982F8F5F8093CB0177
:102C60002DB73EB7215F3F4F2DBF943010F010922B
:102C7000CB018091BB019091BC010E947619909389
:102C80000605809305051092CF018091D00188231D
:102C900051F180910601882331F10E94A72580E53A
:102CA00090E09F938F938EE096E09F938F9321E027
:102CB00030E03F932F9387E291E09F938F933F9370
:102CC0002F938EE292E09F938F9383E08F9381E026
:102CD0008F938CE48F930E94DB0F1092D0018DB7FD
:102CE0009EB70F968DBF8091CD018823D1F0809142
:102CF00006018823B1F08AE090E09F938F9387E2EA
:102D000094E09F938F9381E08F938F9386E58F93C9
:102D10000E94DB0F1092CD012DB73EB7295F3F4FC8
:102D20002DBF8091D1018823D9F08091060188239D
:102D3000B9F08BE090E09F938F9389E494E09F93A8
:102D40008F9381E08F93809103018F9387E48F931A
:102D50000E94DB0F1092D1018DB79EB707968DBFF1
:102D600080915404909155040E947F19882309F49E
:102D700061C080910601882309F45CC080917B06C4
:102D80009927880F991F880F991F7C010027F7FC4E
:102D90000095102F8091460390914703A09148031E
:102DA000B0914903BC01CD01A80197010E94079190
:102DB000309342042093410480913E0390913F035D
:102DC000A0914003B0914103BC01CD01A80197013E
:102DD0000E94079130934404209343048091C902D8
:102DE000809345048091C8028093460488E090E077
:102DF0009F938F9381E494E09F938F9381E08F93CF
:102E000083E08F938BE68F930E94DB0F80914704C2
:102E10002DB73EB7295F3F4F2DBF853018F086E0B4
:102E20008093470483E690E00E94761990935504BE
:102E3000809354048091BF019091C001892B41F08F
:102E400080912504909126040E947F19882321F403
:102E50008091CE01882339F180910601882319F1F0
:102E60000E940D3B82E490E09F938F9386EB95E068
:102E70009F938F9381E08F938F9384E48F930E942D
:102E8000DB0F1092CE018DB79EB707968DBF809154
:102E9000BF019091C001009731F00E947619909384
:102EA0002604809325048091BD019091BE01892B59
:102EB00009F4B8C080912304909124040E947F19E2
:102EC000882309F4AFC080910601882309F4AAC0C1
:102ED00080917B069927880F991F880F991F7C0185
:102EE0000027F7FC0095102F80914603909147032F
:102EF000A0914803B0914903BC01CD01A8019701FD
:102F00000E940791309316042093150480913E038C
:102F100090913F03A0914003B0914103BC01CD01CA
:102F2000A80197010E940791309318042093170479
:102F300020915B0830915C0840915D0850915E08DB
:102F4000DA01C90163E0880F991FAA1FBB1F6A95A8
:102F5000D1F7820F931FA41FB51F820F931FA41FC9
:102F6000B51F20914A0130914B0140914C01509185
:102F70004D01BC01CD010E94079130931A042093AA
:102F8000190480910E0390910F03A0911003B0914A
:102F9000110349E0B595A795979587954A95D1F77F
:102FA00080931B0480910A0390910B03A0910C0362
:102FB000B0910D0339E0B595A795979587953A950A
:102FC000D1F780931C048091160390911703A09170
:102FD0001803B091190329E0B595A79597958795A2
:102FE0002A95D1F780931D048EE090E09F938F93F4
:102FF00085E194E09F938F9381E08F938F9383E497
:103000008F930E94DB0F8091BD019091BE010E94C1
:10301000761990932404809323042DB73EB7295F3B
:103020003F4F2DBF809105018F3F71F1992704E03B
:10303000880F991F0A95E1F7815C9D4F40E150E0B0
:10304000BC01CE0101960E94E68E80E190E09F9344
:103050008F93CE0101969F938F9381E090E09F9391
:103060008F9385E091E09F938F9382E08F9381E02F
:103070008F9381E48F930E94DB0F8FEF8093050184
:103080008DB79EB70B968DBF8091F8058823D1F040
:10309000809106018823B1F081E090E09F938F93A7
:1030A00088EF95E09F938F9381E08F938F9382E4D5
:1030B0008F930E94DB0F1092F8052DB73EB7295F62
:1030C0003F4F2DBF8091CC018823C9F0809106012C
:1030D0008823A9F084E390E09F938F9382E997E09F
:1030E0009F938F9381E08F938F9380E58F930E94BE
:1030F000DB0F1092CC018DB79EB707968DBFE6E02F
:10310000C05F0C944A911F920F920FB60F92112438
:103110002F933F935F936F937F938F939F93AF937F
:10312000BF93EF93FF9320E08091EC01882329F077
:103130008091EC0181508093EC018091D70388232A
:1031400019F081508093D7038091F40181508093CE
:10315000F4018F3F09F05BC089E08093F401809116
:10316000F2019091F30101969093F3018093F201A3
:10317000809112018F5F817080931201882319F46E
:1031800081E08093F101349903C081E08093F501DF
:103190008091ED019091EE01892B21F18091ED015B
:1031A0009091EE010B9750F08091ED019091EE011E
:1031B0000A979093EE018093ED0104C01092EE0106
:1031C0001092ED018091ED019091EE0120910701A7
:1031D0003091080182239323892B11F021E008C04C
:1031E00020E006C08FEF9FEF9093080180930701C6
:1031F00080910101222331F08A3011F45A9A07C0DC
:10320000479A05C08A3011F45A9801C047988091B6
:10321000F501882309F45AC02091A301222309F063
:1032200055C080914B0883FF51C086B19927FC019E
:10323000E071F07084FF13C08091EF019091F00174
:1032400001969093F0018093EF018091EF019091AE
:10325000F001895E9340D0F12093F50137C0809151
:10326000EF019091F001892B69F18091EF0190912C
:10327000F0018A56914030F58091EF019091F00174
:1032800069E270E00E94BE908091EF019091F001A0
:10329000860F971F9093F0018093EF018091EF01CB
:1032A0009091F0010B9750F08091EF019091F00117
:1032B0000A97909397018093960104C0F093970129
:1032C000E09396011092F0011092EF01FF91EF91BF
:1032D000BF91AF919F918F917F916F915F913F913E
:1032E0002F910F900FBE0F901F9018952091F20113
:1032F0003091F301280F391FC901019608952091DB
:10330000F2013091F301821B930B892F9927869547
:10331000807490700895CF93DF930E947619EC012A
:10332000CE010E947F198823D9F3DF91CF910895B0
:10333000CF93DF930E947619EC0109C080911701A9
:10334000882329F0909317018FEC80937A00CE01A7
:103350000E947F19982F882389F3DF91CF910895D8
:103360009FB7F8945F983E9A469A8091B0008F700C
:103370008093B0008091B00083608093B000809112
:10338000B1008B738093B1008091B1008B6080930A
:10339000B1001092B2008FEF8093B3008091B00023
:1033A00080688093B000809170008A7F8093700065
:1033B000809170008260809370009FBF08958AE0C2
:1033C00090E00E9476199093FB018093FA0182E0CD
:1033D00085BD83EA84BD17BC84EB88BD86E086BDCD
:1033E00080916E00816080936E00089580917501D8
:1033F000282F33272F5730408091A706482F552775
:10340000421753071CF4241B350B0CC0882799273F
:10341000841B950B281739071CF4240F351F02C095
:1034200020E030E0C901AA2797FDA095BA2F20918E
:103430001301309114014091150150911601280F8C
:10344000391F4A1F5B1F20931301309314014093CF
:103450001501509316018091A506992774E0880FF5
:10346000991F7A95E1F7AA2797FDA095BA2F2817FB
:1034700039074A075B078CF08091A606992764E01C
:10348000880F991F6A95E1F7AA2797FDA095BA2F93
:1034900082179307A407B50744F480931301909310
:1034A0001401A0931501B09316018091130190911E
:1034B0001401A0911501B0911601B7FF03C00F963A
:1034C000A11DB11D34E0B595A795979587953A95BF
:1034D000D1F79093FA058093F905089580918806B5
:1034E000882339F082E090E09093FE058093FD05FB
:1034F0000AC084E090E09093FE058093FD058091E2
:103500008B06882319F082E090E002C084E090E00E
:103510009093FC058093FB050895AF92BF92CF92E4
:10352000DF92EF92FF920F931F93CF9380919606B5
:10353000E82FFF27E05BFE4F9681C081809111014B
:10354000E92EFF24E7FCF0940F2D1F2D813009F0A8
:10355000DFC12091460330914703409148035091C9
:103560004903C801B7010E94939097FF04C06158B6
:103570007F4F8F4F9F4F7B018C0187E015950795FB
:10358000F794E7948A95D1F78C2F992787FD90952A
:10359000A92FB92F20913E0330913F034091400362
:1035A00050914103BC01CD010E94939097FF04C04C
:1035B00061587F4F8F4F9F4FC7E0959587957795BF
:1035C0006795CA95D1F757016801A61AB70AC80AC4
:1035D000D90A2091BF033091C003C901B3E0880F1D
:1035E000991FBA95E1F7821B930BAA2797FDA09527
:1035F000BA2FA81AB90ACA0ADB0A80918D06992740
:10360000AA27BB27BC01CD01A60195010E9493907A
:1036100097FF04C061507E4F8F4F9F4F5B016C013D
:10362000A9E0D594C794B794A794AA95D1F78091AF
:103630008B068823D1F02091F9053091FA0580910D
:10364000FB059091FC05289FA001299F500D389FF4
:10365000500D1124CA01F4E0880F991FFA95E1F783
:10366000AA2797FDA095BA2F3EC080917501282FFB
:1036700033278091FB059091FC05289FA001299F8D
:10368000500D389F500D1124CA01E4E0880F991F96
:10369000EA95E1F79C01442737FD4095542F80912E
:1036A0000D0190910E01A0910F01B0911001281B06
:1036B000390B4A0B5B0B80919506E82EFF240027FF
:1036C0001127CA01B901A80197010E9407918091B1
:1036D0000D0190910E01A0910F01B0911001820F88
:1036E000931FA41FB51F80930D0190930E01A0930B
:1036F0000F01B09310018091CB0680FF19C080911B
:103700000D0190910E01A0910F01B0911001B7FF32
:1037100003C00F96A11DB11D74E0B595A7959795AF
:1037200087957A95D1F7A80EB91ECA1EDB1E1AC05E
:1037300080910D0190910E01A0910F01B0911001A7
:10374000B7FF03C00F96A11DB11D64E0B595A79505
:10375000979587956A95D1F78A199B09AC09BD0998
:103760005C016D01C091C8068601750156E0EE0C42
:10377000FF1C001F111F5A95D1F7CC2359F12C2F94
:103780003327442755278091E4019091E501A091CA
:10379000E601B091E701BC01CD010E949390DC01EC
:1037A000CB01E80EF91E0A1F1B1F8C2F99270196CB
:1037B0009C01442737FD4095542FC801B7010E9452
:1037C00007912093E4013093E5014093E601509383
:1037D000E70108C0E092E401F092E5010093E60100
:1037E0001093E7018091E4019091E501A091E60139
:1037F000B091E701B7FF03C0CF96A11DB11D46E010
:10380000B595A795979587954A95D1F79093DF0140
:103810008093DE0180918E06482F55278091FB050D
:103820009091FC05489F9001499F300D589F300DA5
:1038300011248091DE019091DF0182179307B4F08B
:1038400080918F06482F55278091FB059091FC05AC
:10385000489F9001499F300D589F300D1124809151
:10386000DE019091DF01281739077CF48091FB0578
:103870009091FC05489F9001499F300D589F300D55
:1038800011243093DF012093DE0180910101843106
:1038900018F41092110105C0809111018F5F80937F
:1038A000110180912708682F7727AB014F575040AF
:1038B0008091A706282F3327241735071CF4621B95
:1038C000730B0CC088279927821B930B4817590745
:1038D0001CF4620F731F02C06FE770E036E0660FE2
:1038E000771F3A95E1F72091DA013091DB01809161
:1038F0008A06482F5527CB01821B930BBA010E94E1
:10390000D290260F371F3093DB012093DA0185C157
:1039100020913E0330913F03409140035091410379
:10392000C801B7010E94939097FF04C061587F4F70
:103930008F4F9F4F7B018C0127E015950795F794DA
:10394000E7942A95D1F78C2F992787FD9095A92F79
:10395000B92F20914603309147034091480350917D
:103960004903BC01CD010E9493909B01AC0197FFDC
:1039700004C021583F4F4F4F5F4F97E055954795F3
:10398000379527959A95D1F72E0D3F1D401F511F52
:10399000809191069927AA27BB27BC01CD010E94DF
:1039A000939097FF04C061507E4F8F4F9F4F5B01F4
:1039B0006C0189E0D594C794B794A7948A95D1F700
:1039C00080917401682F7727AB014F575040809149
:1039D000A706282F3327241735071CF4621B730B07
:1039E0000CC088279927821B930B481759071CF492
:1039F000620F731F02C06FE770E07B010027F7FCC6
:103A00000095102F8091FD059091FE059C014427A3
:103A100037FD4095542FC801B7010E949390DC01F7
:103A2000CB0104E0880F991FAA1FBB1F0A95D1F78D
:103A30002091090130910A0140910B0150910C0134
:103A4000821B930BA40BB50B2091950633274427BB
:103A50005527BC01CD010E940791809109019091E9
:103A60000A01A0910B01B0910C01820F931FA41FBA
:103A7000B51F8093090190930A01A0930B01B093A5
:103A80000C018091CB0681FF19C0809109019091B2
:103A90000A01A0910B01B0910C01B7FF03C00F9672
:103AA000A11DB11D14E0B595A795979587951A9519
:103AB000D1F7A80EB91ECA1EDB1E1AC080910901DB
:103AC00090910A01A0910B01B0910C01B7FF03C0C6
:103AD0000F96A11DB11DC4E0B595A7959795879543
:103AE000CA95D1F78A199B09AC09BD095C016D0122
:103AF000C091C90686017501F6E0EE0CFF1C001F9F
:103B0000111FFA95D1F7CC2359F12C2F33274427D5
:103B100055278091E0019091E101A091E201B091DF
:103B2000E301BC01CD010E949390DC01CB01E80EC2
:103B3000F91E0A1F1B1F8C2F992701969C014427F1
:103B400037FD4095542FC801B7010E94079120937B
:103B5000E0013093E1014093E2015093E30108C09A
:103B6000E092E001F092E1010093E2011093E301A1
:103B70008091E0019091E101A091E201B091E30117
:103B8000B7FF03C0CF96A11DB11DE6E0B595A7957F
:103B900097958795EA95D1F79093DD018093DC01A5
:103BA00080919206482F55278091FD059091FE0542
:103BB000489F9001499F300D589F300D11248091EE
:103BC000DC019091DD0182179307B4F08091930698
:103BD000482F55278091FD059091FE05489F900143
:103BE000499F300D589F300D11248091DC01909138
:103BF000DD01281739077CF48091FD059091FE05C1
:103C0000489F9001499F300D589F300D11243093EB
:103C1000DD012093DC0110921101CF911F910F91D2
:103C2000FF90EF90DF90CF90BF90AF9008951F92DC
:103C30000F920FB60F9211242F933F934F935F93E0
:103C40006F937F938F939F93EF93FF9340E050E0A8
:103C5000809101019091F601843108F04CC09923C4
:103C600009F082C18091B00086FF24C08091B0002D
:103C70008F7B8093B0008091DE019091DF018755AA
:103C80009E4F9093EA018093E90125E08D3D9207D4
:103C900018F08CED95E005C08757914030F487E728
:103CA00091E09093EA018093E9018091E90190917C
:103CB000EA011CC18091B00080648093B0008091C3
:103CC0009406282F33278DED96E0289FB001299F79
:103CD000700D389F700D1124CB012091F7013091A8
:103CE000F801821B930B9093EA018093E90181E034
:103CF0008093110136C1992309F036C18091B0003B
:103D000086FFF9C08091B0008F7B8093B000E09176
:103D1000F901EE23F1F480919406282F33278DEDDD
:103D200096E0289FB001299F700D389F700D1124D7
:103D3000CB012091F7013091F801821B930B9093F6
:103D4000EA018093E9015093F8014093F701469A04
:103D500008C189EA93E09093EA018093E9018E2FEC
:103D600099278330910589F18430910534F48130AD
:103D7000910559F00297B9F06EC08430910509F4AD
:103D80005DC0059709F45DC066C02091FB053091C8
:103D9000FC053695322F2227379527958091DE0135
:103DA0009091DF010DC02091FD053091FE05369503
:103DB000322F2227379527958091DC019091DD01E4
:103DC000821B930B87559C4F55C04091DA0150914F
:103DD000DB01CA0181549F418F3F910510F440ECF3
:103DE0005FE180918806882379F09A0157FF02C02D
:103DF000215C3F4F66E0359527956A95E1F7809104
:103E00008906281B310913C09A0157FF02C0215FA0
:103E10003F4F54E0359527955A95E1F780918906F3
:103E20009927880F991F880F991F281B390B275531
:103E30003C4F3093EA012093E90120C080910008B3
:103E400002C0809130089927880F991F880F991F09
:103E500087559E4F0FC0FF27EE0FFF1FEE56F84FFE
:103E600020813181220F331F8091E9019091EA0175
:103E7000820F931F9093EA018093E9018091E801FA
:103E8000882331F489EA93E09093EA018093E90171
:103E90008091E9019091EA0175E08D3D970718F056
:103EA0008CED95E005C08757914030F487E791E0AD
:103EB0009093EA018093E9019091F9018091940631
:103EC000981751F08091E9019091EA018C5B904044
:103ED0009093EA018093E9018091F7019091F801B4
:103EE0002091E9013091EA01820F931F9093F8012C
:103EF0008093F70136C08091B00080648093B00059
:103F00008CEB90E09093EA018093E9018091F701B6
:103F10009091F80184549F4F9093F8018093F7019A
:103F20008091EB01882321F08091EC028D3820F400
:103F30008091EB01823031F48091E801882311F007
:103F4000469801C0469A8091F9018F5F8093F901EC
:103F500090919406981728F481E0809311011092B3
:103F6000F90181E08093F6012091E9013091EA01A5
:103F700041E02F37340730F08FEF8093B3002F5F8D
:103F800030400FC02F3F3105C9F0C0F0A9014F5F8D
:103F900050404F37510550F480E88093B3002058CB
:103FA00030403093EA012093E90112C08FEF8093F3
:103FB000B3005093EA014093E9010AC08091E901FE
:103FC0008093B3001092EA011092E9011092F60179
:103FD000FF91EF919F918F917F916F915F914F91A1
:103FE0003F912F910F900FBE0F901F901895109238
:103FF0007C008FEC80937A000895CF93DF9310922A
:10400000000286E987BD83E090E00E940631C82F58
:10401000863E08F4C65FC8BD84E690E00E94981909
:1040200080911B0190911C018152934010F0C0EFD0
:1040300002C0C530F8F0C8BD82E390E00E94981934
:1040400084E594E09F938F9387E695E19F938F9308
:10405000E0911304F0911404099580911B01909153
:104060001C010F900F900F900F908152934010F40D
:10407000C550DFCF6C2F83E090E00E940E31CF302F
:1040800018F0CCE8D0E002C0C0E0D0E0CA3FD105D3
:10409000F8F4C7BD82E390E00E94981986E594E0A9
:1040A0009F938F9387E695E19F938F93E0911304FD
:1040B000F0911404099580911B0190911C010F90BF
:1040C0000F900F900F908052934010F02196DECF0A
:1040D000C0930B0680916C0680FF09C08C2F8A501C
:1040E0008B3E28F080912C04806480932C04C7BD03
:1040F0008CE291E00E949819DF91CF910895EF92A0
:10410000FF921F93CF9310E080ED97E00E94761905
:104110007C01CCE8133019F4CB3008F0C9E010E092
:1041200080910F02909110028C5F934024F4809153
:104130001A0181500AC080910F029091100287509D
:10414000944034F080911A018F5F80931A0101C06E
:1041500011E080910D0290910E028C5F934024F447
:104160008091190181500AC080910D0290910E0238
:104170008750944034F0809119018F5F809319012A
:1041800001C01F5F80910B0290910C028C5F9340E5
:1041900024F48091180181500AC080910B02909103
:1041A0000C0287509440C4F0809118018F5F809377
:1041B000180113C088E594E09F938F9387E695E1FB
:1041C0009F938F93E0911304F091140409950F903D
:1041D0000F900F900F905FC01F5F82E180933A02B3
:1041E000809134028E7F8093340285EA8093BC00F4
:1041F00080911A018A3040F480912C048160809370
:104200002C048AE080931A0180911A01863F40F0C5
:1042100080912C04816080932C0485EF80931A0197
:10422000809119018A3040F480912C04826080933F
:104230002C048AE08093190180911901863F40F097
:1042400080912C04826080932C0485EF8093190167
:10425000809118018A3040F480912C04846080930E
:104260002C048AE08093180180911801863F40F069
:1042700080912C04846080932C0485EF8093180136
:1042800080913A02882339F0C7010E947F19882360
:1042900009F090CFF5CF109217018FEC80937A0040
:1042A000809117018823E1F3CA3020F48AE090E07E
:1042B0000E949819C15009F02DCF86E490E00E9429
:1042C0009819CF911F91FF90EF9008951F920F9230
:1042D0000FB60F921124EF92FF920F931F932F931B
:1042E0003F934F935F936F937F938F939F93AF937E
:1042F000BF93EF93FF9380911802282F3327442711
:1043000055278F5F80931802F9012231310508F09B
:10431000E3C3EA5BFF4F0C94599180917800909130
:10432000790046C0809178009091790047C18091D2
:1043300078009091790090931B0280931A0272C1C9
:1043400080914F0390915003209178003091790033
:10435000821B930B909300068093FF058091FF05CD
:1043600090910006909325028093240279C1809158
:104370007800909179002091510330915203821B73
:10438000930B90930A0680930906809109069091F9
:104390000A069093270280932602A0C380911E02F2
:1043A00090911F022091780030917900820F931F25
:1043B00090931F0280931E0281E091C380911C02A2
:1043C00090911D022091780030917900820F931F07
:1043D00090931D0280931C0284E081C38091CC06DF
:1043E00083FF1AC080912501909126019C01220F24
:1043F000331F280F391F40917800509179008BE0CE
:1044000090E0489FB001499F700D589F700D112496
:10441000CB016EE170E00FC08091250190912601E3
:104420009C01220F331F280F391F80917800909133
:10443000790063E070E00E94BE90260F371F36952A
:10444000279536952795309326012093250185E001
:1044500046C3809178009091790040914B03509130
:104460004C03841B950B9093060280930502809168
:10447000050290910602029704F172E04E3E570742
:1044800084F4209119022B5F20931902255080910A
:10449000B5029091B602845F914018F4215F209399
:1044A000190280911902853684F14F5F5F4F509356
:1044B0004C0340934B03845626C080910502909193
:1044C00006028F5F9F4F0CF572E047325707ECF002
:1044D000209119022550209319022B5F8091B5027B
:1044E0009091B602845F914018F42F5020931902E6
:1044F000809119028C394CF44150504050934C0338
:1045000040934B038C5980931902809178009091CD
:1045100079009093020680930106809105029091A4
:1045200006029C01442737FD4095542F80910603D5
:1045300090910703A0910803B0910903820F931F84
:10454000A41FB51F8093060390930703A09308034D
:10455000B0930903209106033091070340910803AB
:104560005091090357FF04C021503C4F4F4F5F4FFC
:104570006AE055954795379527956A95D1F78091CB
:10458000060390910703A0910803B0910903821BD1
:10459000930BA40BB50B8093060390930703A09392
:1045A0000803B09309032EC180911C0290911D0253
:1045B0002091780030917900820F931F90931D0213
:1045C00080931C02109217028CC2809101018A30E4
:1045D00071F4809178009091790020911A023091C5
:1045E0001B02820F931F01969695879517C04091E5
:1045F0001A0250911B02843158F0209178003091BA
:104600007900240F351F8FEF97E0821B930B06C0B4
:104610008091780090917900840F951F90930C02FF
:1046200080930B0286E05BC280914F039091500310
:104630002091780030917900821B930B90930006B3
:104640008093FF058091FF05909100062091240240
:1046500030912502820F931F90930A0280930902E2
:1046600087E03DC2809178009091790020915103BC
:1046700030915203821B930B90930A068093090694
:104680008091090690910A06209126023091270216
:10469000820F931F90930802809307021FC22091FC
:1046A0001E0230911F028091780090917900280FAE
:1046B000391F30931F0220931E02809101018A301E
:1046C00019F4220F331F04C0220F331F220F331F90
:1046D00030931F0220931E0220911E0230911F0270
:1046E000C90137FD079603E0959587950A95E1F78F
:1046F0009093100280930F028091200290912102EA
:10470000820F931F97FD01969595879590932102AF
:104710008093200220915B0330915C03821B930BFA
:104720009093240180932301209115023091160269
:104730008091230190912401280F391F37FF02C077
:104740002F5F3F4F35952795309316022093150222
:1047500033CE20911C0230911D02809178009091FF
:104760007900280F391F30931D0220931C0280917D
:1047700001018A3019F4220F331F04C0220F331FA6
:10478000220F331F30931D0220931C0220911C0224
:1047900030911D02C90137FD0796F3E09595879585
:1047A000FA95E1F790930E0280930D028091220218
:1047B00090912302820F931F97FD019695958795FF
:1047C00090932302809322022091590330915A033F
:1047D000821B930B9093220180932101209113025D
:1047E000309114028091210190912201280F391FEC
:1047F00037FF02C02F5F3F4F359527953093140246
:104800002093130283E06BC11092180281E0809321
:1048100017018091FC019091FD0101969093FD019B
:104820008093FC01809178009091790090931C0115
:1048300080931B0180911B0190911C01AA27BB272B
:10484000209128023091290240912A0250912B0296
:10485000280F391F4A1F5B1F20932802309329021B
:1048600040932A0250932B0280912C028F5F8093F9
:104870002C02803108F432C180911D0190911E01FB
:10488000A0911F01B09120017C018D0163E0EE0C2D
:10489000FF1C001F111F6A95D1F7E81AF90A0A0BCD
:1048A0001B0BE20EF31E041F151F809100029927B7
:1048B00087FD9095A92FB92FBC01CD0120EB30E2E7
:1048C00040E050E00E949390DC01CB01E81AF90A25
:1048D0000A0B1B0BD801C7010496A11DB11DB7FF20
:1048E00005C0D801C7010B96A11DB11D23E0B595E8
:1048F000A795979587952A95D1F780931D01909359
:104900001E01A0931F01B093200180910306909196
:1049100004067C010027F7FC0095102F80911D01F3
:1049200090911E01A0911F01B0912001E81AF90A8F
:104930000A0B1B0BE092E602F092E7020093E802FA
:104940001093E9022091010230910202409103028A
:104950005091040257FF04C0215F3F4F4F4F5F4FFC
:1049600084E055954795379527958A95D1F780919D
:10497000010290910202A0910302B0910402821BF5
:10498000930BA40BB50B8093010290930202A093AA
:104990000302B09304028091010290910202A0915F
:1049A0000302B09104028E0D9F1DA01FB11F8093C2
:1049B000010290930202A0930302B093040280913B
:1049C000010290910202A0910302B0910402B7FF8C
:1049D00003C00F96A11DB11D14E0B595A79597953D
:1049E00087951A95D1F72091E6023091E702281BAE
:1049F000390B64E0213036071CF020E034E006C0BB
:104A00007CEF2030370714F420E03CEF8091FE016A
:104A10009091FF018091FE019091FF0197FF03C0EB
:104A2000909581959F4FA901F3E0440F551FFA958A
:104A3000E1F78D5B9240C4F08091FE019091FF01FF
:104A40009C01E4E0220F331FEA95E1F7281B390BA4
:104A5000240F351F37FF02C0215F3F4F74E03595AB
:104A600027957A95E1F717C08091FE019091FF019B
:104A70009C0165E0220F331F6A95E1F7281B390B73
:104A8000240F351F37FF02C0215E3F4F45E03595AB
:104A900027954A95E1F73093FF012093FE0180911D
:104AA000280290912902A0912A02B0912B02B7FF0F
:104AB00003C00196A11DB11DB595A7959795879542
:104AC0008093280290932902A0932A02B0932B028C
:104AD00088E080932C0202C01092180282E080933A
:104AE00017028091170280937C008091180288231E
:104AF00019F08FEC80937A00FF91EF91BF91AF9105
:104B00009F918F917F916F915F914F913F912F91E5
:104B10001F910F91FF90EF900F900FBE0F901F907D
:104B2000189590E2EEE0F6E08FE49193815087FFD4
:104B3000FCCF089590912F02903540F4E92FFF2784
:104B4000E25FF94F80839F5F90932F020895AF92A9
:104B5000BF92CF92DF92FF920F931F93CF93DF9379
:104B600020912D0220FF0AC080912E02882311F08F
:104B7000815002C08091270180932E0221FF0CC03A
:104B800090912E0280912701981719F410922E020D
:104B900003C09F5F90932E02822F992780FF04C04D
:104BA00081FF02C010922E020E94912580912E0258
:104BB000282F33279AE9C92E95E2D92EC0911304E4
:104BC000D09114048A3098F481E180932F023F93AE
:104BD0002F938FE894E09F938F93DF92CF92FE0103
:104BE00009952DB73EB72A5F3F4F2DBF11C080E119
:104BF00080932F023F932F9384E994E09F938F93A8
:104C0000DF92CF92FE0109958DB79EB706968DBFB4
:104C100020912E02822F9927AA27BB27FC014197BA
:104C200010F00C94FF2EE85AFF4F0AE9C02E05E25F
:104C3000D02EC0911304D09114040C945991109269
:104C40002F0289E994E09F938F930AE915E2DF929E
:104C5000CF92FE01099584E180932F020F900F906F
:104C60000F900F9086E690E09F938F9388E590E0F9
:104C70009F938F931F921F92809101016AE00E947F
:104C8000B290892F99279F938F93809101010E9461
:104C9000B29099279F938F9389EA94E09F938F9383
:104CA000DF92CF92E0911304F0911404099588E209
:104CB00080932F02EDB7FEB73E96EDBF8CED96E0E8
:104CC0009F938F930E94823299279F938F938EEBAD
:104CD00094E09F938F93DF92CF92E0911304F09131
:104CE0001404099580912D0499272DB73EB7285FAC
:104CF0003F4F2DBFEC01C071D07084FF06C08CE324
:104D000080932F028CEC94E0F1C09091C60399231C
:104D100049F18CE380932F02892F99279F938F93DA
:104D200089ED94E09F938F931F930F93E091130469
:104D3000F09114040995DF93CF939091C60381E11C
:104D4000989FC00111248D5F944F9F938F931F9361
:104D50000F93E0911304F091140409958DB79EB759
:104D60000C9647C190912C049923B1F08CE3809369
:104D70002F02892F99279F938F9381EE94E09F9321
:104D80008F931F930F93E0911304F09114040995EE
:104D9000EDB7FEB7369679C490913502992371F03C
:104DA0008CE380932F02892F99279F938F9388EF0D
:104DB00094E09F938F931F930F93D9C480914401E4
:104DC00090914501069710F00C94082F8CE3809386
:104DD0002F028DE095E0A5C780914B081AE9C12EFE
:104DE00015E2D12EC0911304D091140480FF6BC042
:104DF00010922F028091E6029091E702A091E802C2
:104E0000B091E902BC01CD0125E030E040E050E086
:104E10000E9407913F932F938AE195E09F938F9390
:104E2000DF92CF92FE01099584E180932F028DB726
:104E30009EB706968DBF8091E2029091E302A09109
:104E4000E402B091E502BC01CD0125E030E040E094
:104E500050E00E9407913F932F9387E295E09F9344
:104E60008F93DF92CF92E0911304F091140409958F
:104E700088E280932F02EDB7FEB73696EDBF8091A2
:104E80001B0190911C019F938F9384E395E09F9366
:104E90008F93DF92CF92E0911304F091140409955F
:104EA0008CE380932F022DB73EB72A5F3F4F2DBF73
:104EB00087B599279F938F9381E495E09F938F9374
:104EC000DF92CF928EC010922F028EE495E09F93D6
:104ED0008F93DF92CF92FE01099584E180932F0298
:104EE0000F900F900F900F908DE595E09F938F930B
:104EF000DF92CF921AC710922F0286E695E09F9319
:104F00008F930AE915E2DF92CF92FE01099584E1C1
:104F100080932F020F900F900F900F908091460377
:104F200090914703A0914803B0914903B7FF04C093
:104F300081509C4FAF4FBF4FCAE0B595A79597954D
:104F40008795CA95D1F7BF93AF939F938F9383E7CC
:104F500095E09F938F931F930F93E0911304F0912B
:104F60001404099588E280932F02EDB7FEB73896B6
:104F7000EDBF80913E0390913F03A0914003B0911B
:104F80004103B7FF04C081509C4FAF4FBF4FFAE0C1
:104F9000B595A79597958795FA95D1F7BF93AF9358
:104FA0009F938F9382E895E09F938F931F930F9326
:104FB000E0911304F091140409958CE380932F027F
:104FC0002DB73EB7285F3F4F2DBF809108089091C5
:104FD00009089F938F9381E995E09F938F931F9387
:104FE0000F93E0911304F091140409958DB79EB7C7
:104FF00006968DBF0DC7E1E0FE2EC1E0D0E004E9CA
:1050000017E09F2D969584E1989FC001112480930D
:105010002F02F801828193819F938F932196DF93D2
:10502000CF932197808191819F938F93DF93CF932B
:1050300080EA95E09F938F938AE995E29F938F93FF
:10504000E0911304F091140409952DB73EB7245F45
:105050003F4F2DBF32E0F30E22960C5F1F4F88E0CA
:105060008F1578F6D5C610922F0280916106E82F31
:10507000FF27EE0FFF1FEE56F84F808191819F931F
:105080008F9380916006E82FFF27EE0FFF1FEE56EB
:10509000F84F808191819F938F9382EB95E09F934E
:1050A0008F93DF92CF92FE01099584E180932F02C6
:1050B000EDB7FEB73896EDBF80916306E82FFF2766
:1050C000EE0FFF1FEE56F84F808191819F938F93D3
:1050D00080916206E82FFF27EE0FFF1FEE56F84F74
:1050E0008081918181589F4F9F938F9382EC95E0AF
:1050F0009F938F93DF92CF92E0911304F091140469
:10510000099588E280932F022DB73EB7285F3F4F65
:105110002DBF80916506E82FFF27EE0FFF1FEE568B
:10512000F84F8081918181589F4F9F938F938091F9
:105130006406E82FFF27EE0FFF1FEE56F84F808121
:10514000918181589F4F9F938F9382ED95E09F931C
:105150008F93DF92CF92E0911304F091140409959C
:105160008CE380932F028DB79EB708968DBF8091F8
:105170006706E82FFF27EE0FFF1FEE56F84F8081DE
:10518000918181589F4F9F938F9380916606E82F5E
:10519000FF27EE0FFF1FEE56F84F80819181815857
:1051A0009F4F9F938F9382EE95E063C210922F02E0
:1051B00082EF95E09F938F930AE915E2DF92CF92F9
:1051C000FE010995809101010F900F900F900F90B3
:1051D0008A3009F09DC084E180932F0280915B03A7
:1051E00090915C039C0197FF02C0295F3F4F287F8D
:1051F000821B930B9F938F9380915B0390915C0331
:1052000097FD079673E0959587957A95E1F79F93BB
:105210008F9320915B0330915C0337FF02C0295FBD
:105220003F4F63E0359527956A95E1F780910F022E
:1052300090911002821B930B9F938F9380E096E0D6
:105240009F938F931F930F93E0911304F091140495
:10525000099588E280932F022DB73EB7265F3F4F16
:105260002DBF8091590390915A039C0197FF02C072
:10527000295F3F4F287F821B930B9F938F938091D1
:10528000590390915A0397FD079653E0959587959A
:105290005A95E1F79F938F932091590330915A03C8
:1052A00037FF02C0295F3F4F43E0359527954A9568
:1052B000E1F780910D0290910E02821B930B9F9358
:1052C0008F9381E196E09F938F931F930F93E091CB
:1052D0001304F091140409958CE380932F028DB789
:1052E0009EB70A968DBF80915703909158039F9364
:1052F0008F93809157039091580320910B02309126
:105300000C02821B930B9F938F9382E296E0ADC0B9
:105310008B3019F0843108F4ADC084E180932F0202
:1053200080915B0390915C039C0197FF02C0215F19
:105330003F4F207F821B930B97FD01969595879594
:105340009F938F9380915B0390915C0397FD0F96E1
:1053500024E0959587952A95E1F79F938F93209167
:105360005B0330915C0337FF02C0295F3F4FC3E00E
:1053700035952795CA95E1F780910F02909110021B
:10538000821B930B9F938F9380E396E09F938F9361
:105390001F930F93E0911304F0911404099588E290
:1053A00080932F022DB73EB7265F3F4F2DBF8091D0
:1053B000590390915A039C0197FF02C0215F3F4F10
:1053C000207F821B930B97FD0196959587959F9360
:1053D0008F938091590390915A0397FD0F96A4E003
:1053E00095958795AA95E1F79F938F9320915903FF
:1053F00030915A0337FF02C0295F3F4FF3E03595E4
:105400002795FA95E1F780910D0290910E02821B8B
:10541000930B9F938F9382E496E09F938F931F93B8
:105420000F93E0911304F091140409958CE3809399
:105430002F028DB79EB70A968DBF8091570390912A
:10544000580397FD0196959587959F938F9380912B
:1054500057039091580320910B0230910C02821B4C
:10546000930B9F938F9384E596E09F938F931F9365
:105470000F9303C18D3009F0CBC484E180932F02D8
:1054800080911A0199279F938F9380915B0390914C
:105490005C0397FD0F9674E0959587957A95E1F7F3
:1054A0009F938F9320915B0330915C0337FF02C081
:1054B000295F3F4F63E0359527956A95E1F7809125
:1054C0000F0290911002821B930B9F938F9383E6A0
:1054D00096E09F938F931F930F93E0911304F091A5
:1054E0001404099588E280932F022DB73EB7265FFA
:1054F0003F4F2DBF8091190199279F938F938091E2
:10550000590390915A0397FD0F9654E0959587950E
:105510005A95E1F79F938F932091590330915A0345
:1055200037FF02C0295F3F4F43E0359527954A95E5
:10553000E1F780910D0290910E02821B930B9F93D5
:105540008F9387E796E09F938F931F930F93E0913C
:105550001304F091140409958CE380932F028DB706
:105560009EB70A968DBF8091180199279F938F93BC
:10557000809157039091580397FD019695958795D3
:105580009F938F93809157039091580320910B0222
:1055900030910C02821B930B9F938F938BE896E0C4
:1055A0009F938F931F930F93E0911304F091140432
:1055B0000995EDB7FEB73A9668C010922F028FE9B1
:1055C00096E09F938F93DF92CF92FE01099584E13D
:1055D00080932F020F900F900F900F9080915103A6
:1055E000909152039F938F938091070290910802AC
:1055F0009F938F938CEA96E09F938F93DF92CF9245
:10560000E0911304F0911404099588E280932F022D
:105610002DB73EB7285F3F4F2DBF80914F0390912C
:1056200050039F938F938091090290910A029F9358
:105630008F938BEB96E09F938F93DF92CF92E091C5
:105640001304F091140409958CE380932F028DB715
:105650009EB708968DBF80914B0390914C039F930A
:105660008F9380910502909106029F938F938AEC0D
:1056700096E09F938F93DF92CF92E0911304F09185
:1056800014040995EDB7FEB73896EDBFC1C310926B
:105690002F0280912501909126016AE070E00E941E
:1056A000D2909F938F9380912501909126016AE07B
:1056B00070E00E94D2907F936F9389ED96E09F9364
:1056C0008F93DF92CF92FE01099584E180932F02A0
:1056D0002DB73EB7285F3F4F2DBF8091E0089091D6
:1056E000E1086AE070E00E94BE909F938F938091E2
:1056F000E0089091E1086AE070E00E94BE907F931C
:105700006F938DEE96E09F938F93DF92CF92E0910F
:105710001304F0911404099588E280932F028DB749
:105720009EB708968DBF8091E2089091E3089F9301
:105730008F9381E097E09F938F93DF92CF92E091D8
:105740001304F091140409958CE380932F02EDB7B4
:10575000FEB73696EDBF8091E4089091E5089F93DF
:105760008F9381E197E09F938F93DF92CF92E091A7
:105770001304F091140409952DB73EB72A5F3F4FEB
:105780004FC110922F0283E297E09F938F93DF9295
:10579000CF92FE01099584E180932F020F900F9024
:1057A0000F900F9080919207909193079F938F9302
:1057B0008CE297E09F938F93DF92CF92E091130456
:1057C000F0911404099588E280932F028DB79EB75B
:1057D00006968DBF8091EC0299279F938F938CE35F
:1057E00097E09F938F93DF92CF92E0911304F09113
:1057F000140409958CE380932F02EDB7FEB736961B
:10580000EDBF80919107992701979F938F938CE427
:1058100097E0A9CF10922F028CE597E09F938F938A
:10582000DF92CF92FE01099584E180932F020F90C1
:105830000F900F900F9080919601909197019F93F8
:105840008F9384E697E09F938F93DF92CF92E091BE
:105850001304F0911404099588E280932F028DB708
:105860009EB706968DBF80910808909109089F9376
:105870008F9382E797E09F938F93DF92CF92E0918F
:105880001304F091140409958CE380932F02EDB773
:10589000FEB73696EDBF80910403909105039F9368
:1058A0008F9380E897E05FCFCDEECC2EC2E0DC2E68
:1058B00020E030E0E901B3E0FB2EC0932F02F601B7
:1058C00081916F0199279F938F9389010F5F1F4FDC
:1058D0001F930F938EE897E09F938F938AE995E249
:1058E0009F938F93E0911304F091140409952DB7C1
:1058F0003EB7285F3F4F2DBFFA9464969801F7FE9C
:10590000DCCF86C2A1EFCA2EA2E0DA2EC0E0D0E042
:105910008E01F3E0FF2E00932F02F60181916F01BB
:1059200099279F938F932596DF93CF938BE997E0E9
:105930009F938F938AE995E29F938F93E09113044D
:10594000F091140409952DB73EB7285F3F4F2DBF46
:10595000FA940C5E1F4F2497F7FEDDCF59C21092C8
:105960002F0288EA97E09F938F930AE915E2DF926E
:10597000CF92FE01099584E180932F020F900F9042
:105980000F900F908091750199279F938F9380EBD3
:1059900097E09F938F93DF92CF92E0911304F09161
:1059A0001404099588E280932F028DB79EB706965E
:1059B0008DBF8091DE019091DF0197FD0396959553
:1059C0008795959587959F938F938EEB97E09F93FF
:1059D0008F931F930F93E0911304F0911404099592
:1059E0008CE380932F02EDB7FEB73696EDBF809122
:1059F0008F0699279F938F9380918E0699279F9367
:105A00008F938CEC97E09F938F931F930F93E0916C
:105A10001304F091140409952DB73EB7285F3F4F4A
:105A20002DBFF6C110922F028AED97E09F938F93BE
:105A30007AE9A72E75E2B72EDF92CF92FE01099583
:105A40000F900F900F900F90C1E3D7E000E010E0AF
:105A500062E0F62E802F8C5E80932F028B8D99272B
:105A60008F7790709F938F938B8999278F77907002
:105A70009F938F938B8599278F7790709F938F93A8
:105A80008B8199278F7790709F938F938AEE97E001
:105A90009F938F93BF92AF92E0911304F0911404FF
:105AA00009958DB79EB70C968DBFFA940C5E1F4F6B
:105AB000A096F7FECFCFACC110922F028BEF97E0EC
:105AC0009F938F935AE9A52E55E2B52EDF92CF9280
:105AD000FE0109950F900F900F900F90C1E3D7E052
:105AE00000E010E042E0F42E802F8C5E80932F02C5
:105AF0008F8D992787FD90959F938F938F899927F5
:105B000087FD90959F938F938F85992787FD90951B
:105B10009F938F938F81992787FD90959F938F9364
:105B20008AE098E09F938F93BF92AF92E091130425
:105B3000F09114040995EDB7FEB73C96EDBFFA94C9
:105B40000C5E1F4FA096F7FECFCF62C110922F02BE
:105B50008BE198E09F938F930AE915E2DF92CF9251
:105B6000FE01099584E180932F020F900F900F9012
:105B70000F9080914C07881F8827881F97E0899F86
:105B8000C00111248D969F938F9380914407881FA5
:105B90008827881F96E0899FC00111248D969F93C6
:105BA0008F9380913C07881F8827881F95E0899FE5
:105BB000C00111248D969F938F9380913407881F85
:105BC0008827881F9927880F991F880F991F8D96FE
:105BD0009F938F938AE298E09F938F93DF92CF9267
:105BE000E0911304F0911404099588E280932F0248
:105BF0002DB73EB7245F3F4F2DBF80916C07881FA4
:105C00008827881F9BE0899FC00111248D969F9350
:105C10008F9380916407881F8827881F9AE0899F47
:105C2000C00111248D969F938F9380915C07881FEC
:105C30008827881F99E0899FC00111248D969F9322
:105C40008F9380915407881F8827881F992723E006
:105C5000880F991F2A95E1F78D969F938F938EE376
:105C600098E09F938F93DF92CF92E0911304F0918D
:105C7000140409958CE380932F028DB79EB70C9680
:105C80008DBF80917407881F8827881F9CE0899F9B
:105C9000C00111248D969F938F9382E598E09F9386
:105CA0008F93DF92CF92E0911304F0911404099541
:105CB00080917C07EDB7FEB73696EDBF87FF12C027
:105CC00080E480932F0283E698E09F938F93DF9286
:105CD000CF92E0911304F091140409950F900F9066
:105CE0000F900F908091840787FF12C084E4809307
:105CF0002F0286E698E09F938F931F930F93E09176
:105D00001304F091140409950F900F900F900F90C9
:105D100080918C0787FF7CC088E480932F0289E6FE
:105D200098E09F938F931F930F93E0911304F0914A
:105D3000140409950F900F900F900F9069C0109266
:105D40002F028CE698E09F938F93DF92CF92FE0113
:105D5000099584E180932F020F900F900F900F9080
:105D60008091B2019091B3019F938F938AE798E05D
:105D70009F938F93DF92CF92E0911304F0911404DC
:105D8000099588E280932F022DB73EB72A5F3F4FD7
:105D90002DBF8091B4019091B5019F938F9387E8B7
:105DA00098E09F938F93DF92CF92E0911304F0914C
:105DB0001404099589E480932F028DB79EB7069647
:105DC0008DBF84E998E09F938F93DF92CF92E0910B
:105DD0001304F0911404099580912D020F900F90F7
:105DE0000F900F9083FF14C01092B5011092B40170
:105DF00060E070E08EE090E00E941F3109C0809169
:105E00002701281719F421502093270110922E0200
:105E100010922D02DF91CF911F910F91FF90DF9093
:105E2000CF90BF90AF900895F999FECF92BD81BDFC
:105E3000F89A80B599270895F999FECF1FBA92BDB7
:105E400081BD60BD0FB6F894FA9AF99A0FBE089515
:105E50004AEA20E030E02617370740F4FC01819140
:105E6000480F2F5F3F4F26173707C8F3842F992716
:105E70000895EAEA40E050E04617570778F49C019D
:105E8000F999FECF32BD21BDF89A80B5E80F4F5F7A
:105E90005F4F2F5F3F4F4617570790F38E2F99277D
:105EA000089581E08093620682E08093610683E03A
:105EB0008093600684E08093630685E080936406A7
:105EC00086E08093650687E08093660688E080938D
:105ED000670689E0809368068AE0809369068BE014
:105EE00080936A068CE080936B0608958AE5809320
:105EF0005F0680910101843150F08AE080937F0633
:105F00001092A3068BE180937B068EE40AC083E0A7
:105F100080937F0680E28093A3068EE180937B06C8
:105F200085E58093A0068093A10680E28093A20677
:105F30001092CA068AE680936C0682E28093CC06B1
:105F40001092CD0664E0609386061092C20610920D
:105F5000BF0648E04093790656EE50937A0680E4F7
:105F600080937C069EE190936D068FEF80936F0681
:105F70002FE02093700690936E0610927206409365
:105F8000730684E18093740610927506209371065F
:105F900081E08093880680E78093890689E1809379
:105FA0008A0610928B061092A5061092A6061092F1
:105FB000A7061092A80690E890938C0632E33093DF
:105FC0008D0682E08093CB0620938E0650938F0639
:105FD000609394068DE7809397068093980680934C
:105FE00099069093900625E52093910686E4809388
:105FF00092068CED809393068CE380939506109225
:1060000096068FE58093A90683EF8093AB068AEA14
:106010008093AD068093AE0688E28093AA068093B3
:10602000AC0630939A069AE590939B0630939C06B3
:106030008EEF8093AF0684E68093B0069093B1060E
:106040009093B2069093B3068BE48093B4062093AA
:10605000B5068093B6061092B70686E08093B80620
:106060004093B9069093BA068AE28093BB0685EF07
:106070008093BC068CE88093BD0685E08093BE06C5
:106080001092C0061092C10681E28093830681E4DB
:1060900080938406909385061092C3061092C406DE
:1060A0001092C50686E98093C60690939D0687E305
:1060B00080939E061092C7061092C8061092C906D9
:1060C0000895CF93DF930E94762F8AE0809376061F
:1060D00080E18093770626E0209378069AE59093F6
:1060E0007D0688E780937E069093800680938106E4
:1060F0002093820680E2809387068CE380939F063C
:106100008BE48093A406AEECB6E08CE0E8E2F1E02C
:10611000ED01019009928A95E1F76BE770E0CD01FE
:106120008F5690400E94282F8093DA06DF91CF91FE
:106130000895CF93DF930E94762F88E080937606B0
:1061400030E13093770626E02093780694E690932A
:106150007D0688E780937E06909380068093810673
:10616000209382063093870686E480939F0680936F
:10617000A406AEECB6E08CE0EEE2F1E0ED010190B9
:1061800009928A95E1F76BE770E0CD018F56904058
:106190000E94282F8093DA06DF91CF910895CF9344
:1061A000DF930E94762F26E0209376068AE0809384
:1061B000770684E08093780694E690937D0688E7DE
:1061C00080937E06909380068093810620938206BA
:1061D00080E18093870686E480939F068093A406DF
:1061E000AEECB6E08CE0E6E3F1E0ED01019009925F
:1061F0008A95E1F76BE770E0CD018F5690400E94E1
:10620000282F8093DA06DF91CF910895F999FECF78
:1062100092BD81BDF89A80B599270895F999FECF6E
:106220001FBA92BD81BD60BD0FB6F894FA9AF99A73
:106230000FBE089564E17FE20E94218F08954CE132
:106240005FE20E945B8F0895EF92FF920F931F937E
:10625000CF93C82F8150853008F0C3E08CE7C89FEA
:106260008001112488EEE82E8FEFF82EE00EF11E4B
:106270006BE770E0C7010E94392F682F98012D59F4
:106280003F4F8FB39927AC014270507081FDF9CF19
:1062900032BD21BDF89A80B5861711F0CA0123C01E
:1062A0008FB399279C012270307081FDF9CFF2BC29
:1062B000E1BCF89A80B58A3511F0C90114C08CE7A9
:1062C000C89FC0011124489724E13FE24CE750E009
:1062D000BC018FE596E00E94FC8E0E94E86E0E9451
:1062E000F68A81E090E0CF911F910F91FF90EF909F
:1062F0000895282F863010F025E003C0882309F484
:1063000021E0F999FECF1FBA82E090E092BD81BDF5
:1063100020BD0FB6F894FA9AF99A0FBE0895CF935C
:10632000C82F80915F068A3509F051C0C63010F041
:10633000C5E003C0CC2309F44AC00E94EE8D8091D1
:10634000CD0682FF07C080918406843618F080E570
:10635000809384066BE770E08FE596E00E94282F1B
:106360008093DA068CE7C89FC00111242CE13FE23C
:106370004CE750E06FE576E048970E94398F2CE1BA
:106380003FE24CE050E060E676E080E590E00E947D
:10639000398F6CE070E080E696E00E94282F282F6D
:1063A000F999FECF1FBA8CE590E092BD81BD20BD6A
:1063B0000FB6F894FA9AF99A0FBE8C2F0E94793191
:1063C0000E94E86E0E94F68A81E090E002C080E0C0
:1063D00090E0CF9108956DE470E088EE93E00E9424
:1063E000392F482F8FB399279C012270307081FD7F
:1063F000F9CF85E394E092BD81BDF89A80B584170A
:1064000079F48FB399279C012270307081FDF9CF08
:1064100088EE93E092BD81BDF89A80B5813011F08D
:10642000C901089524E13FE24EE450E068EE73E0D4
:106430008BED96E00E94FC8E81E090E008958091C3
:10644000DB068130A9F46DE470E08BED96E00E94EC
:10645000282F809328072CE13FE24EE450E06BEDBB
:1064600076E088EE93E00E94398F81E090E0089515
:1064700080E090E00895CF93DF9381E08093DB0686
:10648000EBEDF6E08FE0158616861786108A8150B0
:10649000349687FFF8CF80E48093E8068093E9067E
:1064A0001092EA068093EB068093EC0690EC9093B2
:1064B000ED061092EE068093EF068093F0061092A0
:1064C000F1069093F2069093F3068093F4061092EF
:1064D000F5068093F6069093F706ACEDB6E087E0FC
:1064E000ECE3F1E0ED01019009928A95E1F76DE4AA
:1064F00070E0CD0101970E94282F80932807DF913B
:10650000CF910895F999FECF82E090E092BD81BDD0
:10651000F89A80B5282F863078F023E0322FF99949
:10652000FECF1FBA82E090E092BD81BD30BD0FB6B4
:10653000F894FA9AF99A0FBE822F992708951F931B
:10654000CF93C82F162F863010F0C5E003C08823E4
:1065500009F4C1E08C2F99278230910541F08330F6
:10656000910544F4019731F40E94613005C00E9406
:10657000993002C00E94CF301123E1F06CE070E04E
:1065800080E590E00E94392F282FF999FECF8CE505
:1065900090E092BD81BDF89A80B5821759F424E14C
:1065A0003FE24CE050E060E570E080E696E00E945B
:1065B000FC8E02C00E94512F8C2F0E948F31CF91F0
:1065C0001F910895DF92EF92FF920F931F93CF9345
:1065D000FF24DF2CEF2C81E090E00E9406318A3509
:1065E00011F031E0E32E6CE070E080E590E00E9475
:1065F000392FC82FF999FECF8CE590E092BD81BD6F
:10660000F89A80B58C1711F421E0D22EC1E001E098
:1066100010E0EE2029F48C2F0E9424318823C9F544
:1066200091E0F92E1F930F938CE998E09F938F933D
:1066300087E695E19F938F93E0911304F091140402
:1066400009952DB73EB72A5F3F4F2DBF0230110588
:1066500049F0033011054CF40130110531F40E946A
:10666000613005C00E94993002C00E94CF30DD2009
:1066700059F024E13FE24CE050E060E570E080E654
:1066800096E00E94FC8E02C00E94512F8C2F0E9427
:106690008F31CF5F0F5F1F4FC63008F4BACFFF2096
:1066A00019F083E00E9479310E948232C82F0E9443
:1066B00024318C2F99279F938F9382EC98E09F939E
:1066C0008F9307E615E11F930F93E0911304F09168
:1066D0001404099581E090E00E9406312DB73EB781
:1066E0002A5F3F4F2DBF8F3F21F00E94EB3188235F
:1066F00099F48BED98E09F938F931F930F93E09104
:106700001304F091140409950E943B320E941F3239
:106710000F900F900F900F90EE2029F06AE581E026
:1067200090E00E940E3110925E0690E0E8EEF6E0F6
:10673000CFE08081349618160CF49F5FC150C7FFDC
:10674000F8CF90935E06892F99279F938F938CEDB6
:1067500096E09F938F938CEF98E09F938F931F9376
:106760000F93E0911304F091140409950E945809C5
:106770008DB79EB708968DBFCF911F910F91FF9057
:10678000EF90DF900895982F2FB7F8943998389AA2
:1067900088B1836088B98091B9008C7F8093B900FB
:1067A0008AE28093B80010923A0210923802109256
:1067B0003702992379F0E1E3F7E08BE01082118250
:1067C00012821382148215821682178281503896A3
:1067D00087FFF4CF78942FBF089510923A0284E98E
:1067E0008093BC0080E88093BC001092BD001092A2
:1067F000BA001092BB001092B9001092B80010922B
:10680000360280E00E94C3331092BB0085E880937B
:10681000BC008091340282608093340208951F92FC
:106820000F920FB60F9211242F933F934F935F93C4
:106830008F939F93EF93FF9380913A02282F3327F2
:10684000442755278F5F80933A02F901273131059C
:1068500008F0C2C2E759FF4F0C94599181E0809330
:10686000360209C0809138028C3090F48091380251
:106870008F5F8093380280913802E82FFF27EE0F58
:10688000FF1FEE0FFF1FE552F94F8585181654F7CD
:10689000809138028C3070F01092330210923202E4
:1068A0001092380285E080933A0280913702880F77
:1068B0008D5A04C080913802880F8E5A8093BB0095
:1068C00085E87FC280913802E82FFF2783E0EE0F32
:1068D000FF1F8A95E1F7EF5CF84F81818093BB0041
:1068E00085E88093BC0080913802E82FFF27EE0FE7
:1068F000FF1FEE0FFF1FEE0FFF1FEF5CF84F8081B1
:1069000080FF91C080913802E82FFF27EE0FFF1F14
:10691000EE0FFF1FEE0FFF1FEF5CF84F8281882301
:1069200029F080915E06873008F46CC280913202B3
:1069300090913302892B09F065C2809130029091C9
:106940003102892B09F05EC26EC08091380221E0CD
:1069500030E002C0220F331F8A95E2F780913002A7
:106960009091310228233923232B79F0809138022A
:10697000E82FFF27EE0FFF1FEE0FFF1FEE0FFF1F89
:10698000EF5CF84F80E184830DC080913802E82FDE
:10699000FF27EE0FFF1FEE0FFF1FEE0FFF1FEF5C35
:1069A000F84F148280913802E82FFF2753E0EE0F52
:1069B000FF1F5A95E1F7EF5CF84F8481282F3327AA
:1069C00043E0220F331F4A95E1F780913802E82F08
:1069D000FF2793E0EE0FFF1F9A95E1F7EF5CF84F6A
:1069E00082818770822B8093BB0085E88093BC00F6
:1069F0002091380281E090E002C0880F991F2A950B
:106A0000E2F7209132023091330282239323892BC3
:106A100051F089E297E090933E0280933D0288E036
:106A200080933F02EFC184E089C1E0913D02F09183
:106A30003E0281918093BB0085E88093BC00F09377
:106A40003E02E0933D0280913F02815080933F02DD
:106A5000882309F4D7C183E071C18091B9008033E4
:106A600051F580913B02882329F4809138028F5F91
:106A700080933B0280913802E82FFF2783E0EE0FDE
:106A8000FF1F8A95E1F7EF5CF84F838199278F7795
:106A900090708F3791057CF480913802E82FFF27A2
:106AA000EE0FFF1FEE0FFF1FEE0FFF1FEF5CF84F03
:106AB00083818F5F838310923A0284E98093BC00C4
:106AC0008AE090E0909345018093440180913802E0
:106AD0008F5F8093380210923A026DC18091B900A5
:106AE0008034C9F180913702E82FFF27EE0FFF1F96
:106AF000EE0FFF1FEE0FFF1FEF5CF84F83818F77C4
:106B00008383809137028F5F8093370280913702B1
:106B10008C30A0F0109237021092310210923002A5
:106B200080913C028F5F80933C028C3038F0109251
:106B30003C02809134028D7F809334028091340234
:106B400081608093340210923A0284E98093BC0001
:106B50001092360273C080913702E82FFF27EE0FA4
:106B6000FF1FEE0FFF1FEE0FFF1FEF5CF84F83813B
:106B70008068838380913702E82FFF27EE0FFF1F85
:106B8000EE0FFF1FEE0FFF1FEF5CF84F808180FFBD
:106B90002FC080913702E82FFF2753E0EE0FFF1F31
:106BA0005A95E1F7EF5CF84F84819927009751F0EF
:106BB0004097D9F589E297E090933E0280933D0299
:106BC00088E031C080913702992743E0880F991FF0
:106BD0004A95E1F78A5C984F90933E0280933D027C
:106BE0009091370280913C029817E1F483E01BC03A
:106BF00080913702992733E0880F991F3A95E1F782
:106C00008A5C984F90933E0280933D0280913402BB
:106C100081FD06C09091370280913C02981711F4D3
:106C200082E001C081E080933F0280913F02813089
:106C300011F485E801C085EC8093BC0080913B0293
:106C40008093350210923B02DDC0E0913D02F0914D
:106C50003E028091BB00808380913D0290913E0274
:106C6000019690933E0280933D0280913F028150B5
:106C700080933F02823010F085EC5DC0813011F4CA
:106C800085E859C08091340281FF2DC08091B40203
:106C900080FD1DC080913702E82FFF2723E0EE0F13
:106CA000FF1F2A95E1F7EF5CF84F86818A3F79F460
:106CB00080913702E82FFF2793E0EE0FFF1F9A9590
:106CC000E1F7EF5CF84F8081816080830CC0809198
:106CD0003702E82FFF2783E0EE0FFF1F8A95E1F7C9
:106CE000EF5CF84F1082809137028F5F80933702FC
:106CF000809137028C30A0F010923702109231024E
:106D00001092300280913C028F5F80933C028C3065
:106D100038F010923C02809134028D7F80933402CF
:106D200010923A0284E98093BC0080913402816021
:106D30008093340265C08093BC0086E080933A0261
:106D400061C088E9BBCD80913902880F805FB6CDE4
:106D50008091390299278130910561F08230910547
:106D60001CF4892B21F04EC0029739F04BC0809162
:106D70001A01A4CD80911901A1CD809118019ECD59
:106D800080E89CCD10923A0284E98093BC00109276
:106D900036028AE090E0909345018093440180910F
:106DA0003902823088F4809139028F5F80933902F2
:106DB00082E180933A02809134028E7F8093340284
:106DC00085EA8093BC001EC0109239028091340283
:106DD00081608093340216C010923A0284E9809355
:106DE000BC00809134028160809334028AE090E09C
:106DF000909345018093440110923802109237021B
:106E000010923602FF91EF919F918F915F914F9178
:106E10003F912F910F900FBE0F901F9018951F93C9
:106E2000CF93DF93182F8091EB02882321F4809178
:106E3000C101882319F081E090E097C01D3008F06F
:106E400092C01123B1F0E12FFF2723E0EE0FFF1FC7
:106E50002A95E1F7EF5CF84F3597808135968823C6
:106E60000CF081C03897808180FD03C083E090E002
:106E70007CC080912907823019F084E090E075C0D1
:106E800067E070E089E297E00E94282F9091300738
:106E9000891719F085E090E068C080ED97E00E94C6
:106EA0007619EC018091340280FD05C0CE010E946C
:106EB0007F198823B9F3112319F48FEF90E00BC0E9
:106EC000212F33272150304081E090E002C0880F0D
:106ED000991F2A95E2F79093330280933202A1E042
:106EE000B0E0E1E3F7E040E050E06BE0CD01042EDC
:106EF00002C0880F991F0A94E2F720913202309164
:106F0000330282239323892B11F011821282615064
:106F10004F5F5F4F389667FFE9CF109238021092AB
:106F20003A02809134028E7F8093340285EA809306
:106F3000BC008091340280FD05C0CE010E947F1903
:106F40008823B9F38091320290913302892B29F082
:106F5000CE010E947F19882311F380913202909113
:106F60003302009711F082E090E0DF91CF911F9102
:106F700008950F931F93CF93DF93982F8091EB0287
:106F8000882321F48091C101882319F081E090E0E9
:106F900092C09D30A0F4992319F486E090E08BC054
:106FA000C92FDD27FE0133E0EE0FFF1F3A95E1F711
:106FB000EF5CF84F35978081359687FD03C082E0FE
:106FC00090E079C03897808180FD03C083E090E035
:106FD00072C080ED97E00E9476198C018091340296
:106FE00080FD05C0C8010E947F198823B9F321974D
:106FF00021E030E0C90102C0880F991FCA95E2F76D
:107000009093310280933002D901E1E3F7E040E050
:1070100050E06BE0CD01042E02C0880F991F0A9446
:10702000E2F7209130023091310282239323892BA1
:1070300011F01182128261504F5F5F4F389667FFE7
:10704000E9CF109237021092290710923007109260
:107050003A02809134028E7F8093340285EA8093D5
:10706000BC008091340280FD05C0C8010E947F19D8
:107070008823B9F38091300290913102892B29F055
:10708000C8010E947F19882311F38091290782305B
:1070900019F084E090E00FC067E070E089E297E0CB
:1070A0000E94282F90913007891719F085E090E011
:1070B00002C080E090E0DF91CF911F910F91089581
:1070C000CF93DF9380E022E83FEFC6ECD7E0E2E920
:1070D000F7E0DF01853020F411961C921E9202C069
:1070E000318320831982188222968F5F12963296FE
:1070F0008A3180F3109258031092570310925A036A
:107100001092590310925C0310925B03DF91CF91B0
:1071100008951F920F920FB60F9211240F931F9391
:107120002F933F934F935F936F937F938F939F938F
:10713000AF93BF93CF93DF93EF93FF938091CC06F0
:1071400082FDE1C04091860050918700809141020C
:1071500090914202481B590B8091860090918700C4
:107160009093420280934102CA018D549440A091B1
:107170004302B0914402835F9A4178F480914302C4
:1071800080939107149714F01092480181E090E0E9
:1071900090934402809343022BC2AD30B1050CF0B2
:1071A00027C2CA018B5F9040845B914008F086C083
:1071B0008091460190914701481B590BE091C70609
:1071C000EE2351F0FF27EE0FFF1FEE56F84F8081A0
:1071D000918184369105ECF4FD01EA0FFB1FEE5618
:1071E000F84F80819181FA01E81BF90BCF01F7FF7D
:1071F00003C0909581959F4F06975CF48091EC02B7
:10720000883C20F48091EC02865F01C088EC80937A
:10721000EC02FD01EA0FFB1FEE56F84F80819181D1
:107220009C01220F331F280F391F240F351F37FFF2
:1072300002C02D5F3F4FE901D595C795D595C795FC
:10724000CA0101968C179D0714F4219706C041507E
:107250005040C417D5070CF421968091EC02833C72
:10726000E0F08D010A0F1B1FF801EE56F84F8081E8
:1072700091819E01281B390BC90163E070E00E94D7
:10728000D290CB01880F991F860F971F0A53184F72
:10729000D80111969C938E9307C0AA0FBB1FAA53C7
:1072A000B84F11961C921E92E0914302F091440255
:1072B000EE0FFF1FEE56F84FD183C083209143029B
:1072C000309144022F5F3F4F30934402209343029A
:1072D00080910101843108F08BC12530310511F412
:1072E0005D9A01C05D98809143029091440286307E
:1072F000910511F45C9A01C05C98079711F45B9AB0
:1073000077C15B9875C1409186005091870080914C
:10731000450290914602481B590B8091860090913E
:1073200087009093460280934502CA018D54944091
:107330006091AF02835F9A4108F07AC06093400287
:1073400080914002843008F453C09091910780915D
:107350004002981709F04CC05091B0025B3008F41D
:107360003FC0109248011092AF0240E05F31C0F080
:10737000E42FFF27EE0FFF1F9F0125583D4FDF0130
:10738000AE56B84F8D919C91D9018D939C93DF019E
:10739000AA53B84F8D919C91EB56FD4F91838083FA
:1073A000E42FFF27EE0FFF1F9F012E56384FDF01FE
:1073B000A95BBD4F8D919C91D90111969C938E93A1
:1073C000DF01AF59BD4F8D919C91EA53F84F9183E6
:1073D0008083842F8F5F482F8D3040F28093AF02DF
:1073E0008091B0028F3FB9F08F5F8093B00213C0DD
:1073F0008091B002853620F08AE08093B00202C00E
:107400001092B002809101018A3011F0843110F0A5
:10741000289A01C0289881E08093AF028091EB0206
:10742000882309F0E5C08091400280939107E0C075
:107430006D3008F0B5C0CA018B5F9040845B91400D
:1074400008F090C08091460190914701481B590B6C
:10745000E62FFF27EE0FFF1FE95BFD4F8081918133
:10746000FA01E81BF90BCF0105960B9720F5E09187
:10747000C706EE2351F0FF27EE0FFF1FEE56F84F21
:107480008081918184369105B4F48091B0028A3173
:1074900020F08091EC02865F05C08B3028F080914F
:1074A000EC028E5F8093EC028091EC02893C18F034
:1074B00088EC8093EC02E62FFF27EE0FFF1FE95BBD
:1074C000FD4F808191819C01220F331F280F391FAE
:1074D000240F351F37FF02C02D5F3F4FE901D595BF
:1074E000C795D595C795CA0101968C179D0714F4C9
:1074F000219706C041505040C417D5070CF421967F
:107500008091EC028E3BD8F0E62FFF27EE0FFF1F95
:10751000DF01A95BBD4F8D919C919E01281B390B0A
:10752000C90163E070E00E94D290CB01880F991FDF
:10753000860F971FEF59FD4F9183808308C0E62F78
:10754000FF27EE0FFF1FEF59FD4F11821082809130
:10755000AF02E82FFF27EE0FFF1FE95BFD4FD1833E
:10756000C08309C0809101018A3011F0843110F08C
:10757000289A01C0289880910101843188F4809173
:10758000AF02853011F45D9A05C05D98863011F424
:107590005C9A05C05C98873011F45B9A01C05B98D7
:1075A0008091AF02843120F48F5F8093AF0220C0BE
:1075B0008431F1F4809101018A3011F0843110F0AE
:1075C000289A01C028988EE18093AF022CE0C6EC87
:1075D000D7E0ABE7B2E0E2E9F7E08D919D919183CE
:1075E00080833296198218822296215027FFF5CF88
:1075F000FF91EF91DF91CF91BF91AF919F918F91CB
:107600007F916F915F914F913F912F911F910F91BA
:107610000F900FBE0F901F901895EF92FF920F934F
:107620001F9380917B069927880F991F880F991FB8
:107630007C010027F7FC0095102F80914603909164
:107640004703A0914803B0914903BC01CD01A801B3
:1076500097010E9407913093B9052093B805809156
:107660003E0390913F03A0914003B0914103BC01C0
:10767000CD01A80197010E9407913093BB0520938B
:10768000BA0580914F089091500897FD0396959503
:107690008795959587959093BD058093BC058091BE
:1076A0005F089091600897FD03969595879595954D
:1076B00087959093BF058093BE0580915703909165
:1076C000580320910B0230910C02821B930B909374
:1076D000C1058093C0058091E6029091E702A091D8
:1076E000E802B091E902BC01CD0125E030E040E0C4
:1076F00050E00E9407913093C3052093C20580910A
:107700000502909106029093C5058093C40580916F
:107710009601909197019093C9058093C805809137
:107720002501909126019093CB058093CA05809105
:10773000EC0299279093CD058093CC0580910808A1
:10774000909109089093CF058093CE0580913207E0
:1077500099279093D1058093D00580913A07992776
:107760009093D3058093D2058091420799279093F7
:10777000D5058093D40580914A0799279093D70522
:107780008093D6058091DE019091DF019093E10511
:107790008093E0058091E0089091E1089093E505E1
:1077A0008093E4058091E4089091E5089093E705C3
:1077B0008093E6058091E2029091E302A091E402B9
:1077C000B091E502BC01CD0125E030E040E050E0A1
:1077D0000E9407913093E9052093E8058091040306
:1077E000909105039093EF058093EE058091E60854
:1077F00099279093F3058093F2058091B7039091B8
:10780000B8039093F5058093F4058091B5039091AA
:10781000B6039093F7058093F60580912C04882396
:1078200021F480912D04882321F08091B705816097
:1078300003C08091B7058E7F8093B7051F910F918C
:10784000FF90EF9008951F93CF93DF93182FEB01D4
:107850008091EB02882309F5809101018C3010F4AE
:10786000299801C0299A11501F3F81F0D093EE0151
:10787000C093ED018091ED019091EE01892BD1F73C
:10788000CE018C0F9D1F0E948B19EDCF80910101BD
:107890008C3010F4299A01C02998DF91CF911F9163
:1078A0000895CF93DF93809101018D3011F40E94F0
:1078B0007F2010927A0080910F0290911002909395
:1078C00014088093130880910D0290910E029093FA
:1078D00004088093030880910B0290910C0290930E
:1078E0005508809354082091070230910802C9017D
:1078F000880F991F880F991F820F931F820F931F64
:107900009093500880934F082091090230910A0209
:10791000C901880F991F880F991F820F931F820F2B
:10792000931F9093600880935F088FEC80937A0098
:10793000ADEEB2E0C4E6D6E097E08991E82FFF27EC
:10794000EE0FFF1FEE56F84F0190F081E02DE15849
:10795000FF4F1E161F061CF0E0E0F0E005C0EF3FF1
:10796000F10514F0EFEFF0E08C91282F3327E217A8
:10797000F30714F4815004C02E173F0714F48F5FEF
:107980008C939150119697FFD8CF8091A00699279C
:10799000AA27BB27BC01CD0124EC39E040E050E030
:1079A0000E949390DC01CB0180938E0190938F0114
:1079B000A0939001B09391018091A1069927AA27E5
:1079C000BB27BC01CD010E949390DC01CB018093C9
:1079D0008A0190938B01A0938C01B0938D01DF916C
:1079E000CF910895A0E0B0E0E8EFFCE30C9428917B
:1079F000882EC0E0D0E07E016E0110922C04469AE1
:107A0000D0935203C0935103D0935003C0934F03BC
:107A1000D0934C03C0934B03D0935C03C0935B03A0
:107A2000D0935A03C0935903D0935803C09357037C
:107A30001092720110927101109200020E94513C4A
:107A400084E690E00E9498190E94513C80916C0657
:107A500080FF10C080911B0190911C01875B9340B7
:107A600038F480911B0190911C018E5E924010F4BD
:107A70000E94FD1F0FE18AE090E00E94981980911A
:107A80000B0290910C02C80FD91F80910F029091A8
:107A90001002E80EF91E80910D0290910E02C80EA0
:107AA000D91E015007FFE7CF9701205F3F4F369562
:107AB00027953695279530935C0320935B03C60189
:107AC0004096969587959695879590935A038093BF
:107AD00059036096F5E0D695C795FA95E1F7D093EE
:107AE0005803C093570390935603809355033093E4
:107AF000540320935303882009F441C080914F0818
:107B00009091500897FF03C0909581959F4F6CE02E
:107B100070E00E94D2909B017093520360935103D6
:107B200080915F089091600897FF03C090958195C0
:107B30009F4F6CE070E00E94D2907093500360936E
:107B40004F03809101069091020690934C0380931D
:107B50004B03B90184E090E00E941F3160914F0314
:107B60007091500386E090E00E941F3160914B03BA
:107B700070914C0388E090E00E941F3165C084E062
:107B800090E00E941A31909352038093510386E053
:107B900090E00E941A319093500380934F0388E045
:107BA00090E00E941A319C0190934C0380934B0308
:107BB00080915103909152038150984050F48091EC
:107BC0004F03909150038150984018F42150344055
:107BD000D8F18DE199E09F938F9387E695E19F938C
:107BE0008F93E0911304F0911404099580914F084C
:107BF0009091500897FF03C0909581959F4F6CE03E
:107C000070E00E94D2907093520360935103809170
:107C10005F089091600897FF03C0909581959F4FF2
:107C20006CE070E00E94D2907093500360934F0319
:107C3000809101069091020690934C0380934B0330
:107C40000F900F900F900F9010921408109213083D
:107C500010920408109203081092550810925408CC
:107C600084E690E00E9498198091070290910802A2
:107C70009C01220F331F220F331F280F391F280F9B
:107C8000391F3093500820934F088091090290913A
:107C90000A028C01000F111F000F111F080F191F7E
:107CA000080F191F1093600800935F0880917B06EE
:107CB000C82EDD24EE24FF24442737FD4095542FA1
:107CC000C701B6010E9493904B015C01609346038B
:107CD0007093470380934803909349039801442786
:107CE00037FD4095542FC701B6010E949390DC01E7
:107CF000CB0180933E0390933F03A0934003B09346
:107D000041038092260390922703A0922803B09209
:107D1000290380931E0390931F03A0932003B09325
:107D20002103109216031092170310921803109259
:107D3000190380911D0190911E01A0911F01B09126
:107D4000200190930406809303061092FF01109285
:107D5000FE0110920603109207031092080310927E
:107D60000903009196011091970110930503009368
:107D7000040384E690E0909393018093920182E360
:107D800090E09093EE018093ED018091A0069927F9
:107D9000AA27BB27BC01CD0124EC39E040E050E02C
:107DA0000E949390DC01CB018856954CAF4FBF4F9A
:107DB00080938E0190938F01A0939001B0939101D5
:107DC0008091A1069927AA27BB27BC01CD010E945B
:107DD0009390DC01CB018856954CAF4FBF4F8093F9
:107DE0008A0190938B01A0938C01B0938D01109226
:107DF0004F0110924E01C801AA2797FDA095BA2FF6
:107E000020914A0130914B0140914C0150914D011C
:107E1000BC01CD010E949390DC01CB0180935B08F3
:107E200090935C08A0935D08B0935E0810920103E4
:107E3000109200030E94E86E8091B40284608093E7
:107E4000B4028FEF8093DB081092DC0880E280930D
:107E5000DD08CDEED2E0A4E6B6E007E08D91E82F94
:107E6000FF27EE0FFF1FEE56F84F8081918181585A
:107E70008993015007FFF2CF84E68093EC02809152
:107E8000EB01882311F0469A579A80915B039091F9
:107E90005C0380569940815C9B4228F080912C04C1
:107EA000816080932C048091590390915A038056ED
:107EB0009940815C9B4228F080912C0482608093E1
:107EC0002C0480915703909158038C52914089570C
:107ED000954028F080912C04846080932C0480913C
:107EE0005103909152038C529140835C914028F051
:107EF00080912C04886080932C0480914F03909192
:107F000050038C529140835C914028F080912C0466
:107F1000806180932C0480914B0390914C0380509E
:107F200092408355914028F080912C048062809388
:107F30002C0486E4809385010E94F68AECE0CDB79C
:107F4000DEB70C944491A3E1B0E0E9EAFFE30C94BE
:107F50002291809157039091580320910B02309108
:107F60000C02821B930B90935508809354088091C8
:107F700015029091160297FD07969C0113E0359526
:107F800027951A95E1F730931408209313088091F0
:107F900013029091140297FD0796B3E0959587958B
:107FA000BA95E1F7909304088093030830931F0873
:107FB00020931E08909317088093160880914F080D
:107FC00090915008AC01440F551F480F591F209144
:107FD000070230910802C901880F991F880F991F65
:107FE000820F931F820F931F480F591F57FF02C024
:107FF0004D5F5F4F55954795559547955093500860
:1080000040934F0880915F0890916008AC01440F45
:10801000551F480F591F2091090230910A02C901CA
:10802000880F991F880F991F820F931F820F931F2C
:10803000480F591F57FF02C04D5F5F4F5595479539
:10804000559547955093600840935F08209107022B
:1080500030910802C901880F991F880F991F820F5C
:10806000931F820F931F9C01442737FD4095542F87
:108070008091360390913703A0913803B091390372
:10808000820F931FA41FB51F80933603909337036D
:10809000A0933803B09339032091090230910A026A
:1080A000C901880F991F880F991F820F931F820F94
:1080B000931F9C01442737FD4095542F8091320334
:1080C00090913303A0913403B0913503820F931F35
:1080D000A41FB51F8093320390933303A0933403FE
:1080E000B0933503809128089091290820910702C8
:1080F00030910802820F931F9093290880932808DB
:1081000080915708909158082091090230910A02F5
:10811000820F931F909358088093570880914D03C6
:1081200090914E03019690934E0380934D0380915E
:1081300001069091020620914B0330914C03821B63
:10814000930B9C01442737FD4095542F80912E03BB
:1081500090912F03A0913003B0913103820F931FB0
:10816000A41FB51F80932E0390932F03A093300379
:10817000B09331038FEC80937A0010921701209115
:108180001E0330911F034091200350912103298742
:108190003A874B875C8729543B46414050402CF03E
:1081A00028E43BE641E050E00DC089859A85AB8527
:1081B000BC85885B9449AE4FBF4F4CF428EB34E943
:1081C0004EEF5FEF2D833E834F83588708C089852C
:1081D0009A85AB85BC858D839E83AF83B8872091BC
:1081E00026033091270340912803509129032D87BE
:1081F0003E874F87588B29543B46414050402CF0D6
:1082000028E43BE641E050E00DC08D859E85AF85BA
:10821000B889885B9449AE4FBF4F4CF428EB34E9E2
:108220004EEF5FEF29833A834B835C8308C08D85D3
:108230009E85AF85B88989839A83AB83BC83A091DF
:108240005408B0915508BB8BAA8BFD01CF01AA271A
:1082500097FDA095BA2FA0901603B0901703C09079
:108260001803D0901903A80EB91ECA1EDB1EA092D7
:108270001603B0921703C0921803D0921903E0902E
:108280005B08F0905C0800915D0810915E08E80EB4
:10829000F91E0A1F1B1FE0925B08F0925C08009316
:1082A0005D0810935E08F091CF02F98BFF2309F06F
:1082B00098C18091CE02882309F093C180914B0828
:1082C00086FF8FC18091030890910408AA2797FD2B
:1082D000A095BA2FBC01CD0129813A814B815C81E7
:1082E0000E9493909B01AC0197FF04C02150384F2E
:1082F0004F4F5F4FBBE05595479537952795BA95FA
:10830000D1F780917101682E772488249924CA01BD
:10831000B901A40193010E949390DC01CB018093E9
:10832000670390936803A0936903B0936A03B7FF50
:1083300004C08150904FAF4FBF4F1C012D01ACE0E6
:108340005594479437942794AA95D1F720926703C0
:10835000309268034092690350926A038091130837
:1083600090911408AA2797FDA095BA2FBC01CD01C2
:108370002D813E814F8158850E94939097FF04C0C4
:108380006150784F8F4F9F4FFBE09595879577957C
:108390006795FA95D1F7A40193010E949390DC01AF
:1083A000CB0180936B0390936C03A0936D03B09308
:1083B0006E03B7FF04C08150904FAF4FBF4F9C0179
:1083C000AD01ECE05595479537952795EA95D1F79E
:1083D00020936B0330936C0340936D0350936E03B3
:1083E00080916703909168039093FB078093FA074D
:1083F00080916B0390916C039093FF078093FE072D
:10840000221933094409550920936B0330936C03F7
:1084100040936D0350936E03E20EF31E041F151F6D
:10842000E0925B08F0925C0800935D0810935E0890
:10843000809170018823B1F457FF04C02F5F3F4F34
:108440004F4F5F4F5595479537952795A21AB30A19
:10845000C40AD50AA0921603B0921703C09218035B
:10846000D09219032A893B8979010027F7FC0095EE
:10847000102F80916B0390916C03A0916D03B091CC
:108480006E03E80EF91E0A1F1B1FC801B7012981E0
:108490003A814B815C810E9493909B01AC0197FFD4
:1084A00004C02150384F4F4F5F4F6BE055954795B3
:1084B000379527956A95D1F780917201A82EBB2434
:1084C000CC24DD24CA01B901A60195010E94939034
:1084D000DC01CB0180935F0390936003A093610361
:1084E000B0936203B7FF04C08150904FAF4FBF4FAE
:1084F0003C014D013CE095948794779467943A95BC
:10850000D1F760925F037092600380926103909252
:108510006203C801B7012D813E814F8158850E94B9
:10852000939097FF04C06150784F8F4F9F4F2BE07F
:1085300095958795779567952A95D1F7A601950129
:108540000E949390DC01CB018093630390936403BA
:10855000A0936503B0936603B7FF04C08150904FAA
:10856000AF4FBF4FAC01BD018CE075956795579536
:1085700047958A95D1F740936303509364036093C2
:108580006503709366032A893B8937FF03C03095E2
:1085900021953F4F21343105E4F1D401C30197FE09
:1085A00007C0B095A095909581959F4FAF4FBF4F55
:1085B00081389105A105B10584F4DB01CA0177FF7B
:1085C00007C0B095A095909581959F4FAF4FBF4F35
:1085D00081389105A105B105E4F081E080930203A3
:1085E00018C01092FF071092FE071092FB0710921E
:1085F000FA071092630310926403109265031092BD
:10860000660310925F031092600310926103109250
:1086100062038091630390916403A0916503B0911C
:108620006603BC01CD0124E630E040E050E00E944A
:108630000791E0905F03F0906003E21AF30AF09272
:108640001208E092110880915F0390916003A0915D
:108650006103B0916203BC01CD0124E630E040E04B
:1086600050E00E940791DA01C90120916303309123
:1086700064038C01021B130B10930608009305087A
:1086800080914A0190914B01A0914C01B0914D0114
:10869000BC01CD0128E631E040E050E00E9493901B
:1086A00020915B0830915C0840915D0850915E0814
:1086B000261737074807590764F0261B370B480B66
:1086C000590B20935B0830935C0840935D085093EE
:1086D0005E0820915B0830915C0840915D085091E4
:1086E0005E0857FF0CC0260F371F481F591F2093E5
:1086F0005B0830935C0840935D0850935E0860917E
:108700000308709104086E0D7F1D9B01442737FDFF
:108710004095542F80911A0390911B03A0911C0344
:10872000B0911D03820F931FA41FB51F80931A03DE
:1087300090931B03A0931C03B0931D038091D4025C
:108740009091D502681B790BCB01AA2797FDA095C4
:10875000BA2F29853A854B855C85820F931FA41F0C
:10876000B51F80931E0390931F03A0932003B09323
:108770002103C0908A01D0908B01E0908C01F09091
:108780008D01C816D906EA06FB06C4F488EA91E60C
:10879000A0E0B0E08C199D09AE09BF0980931E03CB
:1087A00090931F03A0932003B093210380931A0397
:1087B00090931B03A0931C03B0931D032227332720
:1087C000A9012C193D094E095F0980911E03909162
:1087D0001F03A0912003B091210382179307A407E0
:1087E000B507B4F4D701C601885A9146A040B040FD
:1087F00080931E0390931F03A0932003B093210343
:1088000080931A0390931B03A0931C03B0931D0342
:108810006091130870911408600F711F9B01442729
:1088200037FD4095542F8091220390912303A0910E
:108830002403B0912503820F931FA41FB51F8093BB
:10884000220390932303A0932403B09325038091E4
:10885000D2029091D302681B790BCB01AA2797FD16
:10886000A095BA2F2D853E854F855889820F931F7D
:10887000A41FB51F8093260390932703A09328037A
:10888000B0932903E0908E01F0908F010091900148
:1088900010919101E816F9060A071B07C4F488EA4B
:1088A00091E6A0E0B0E08E199F09A00BB10B809378
:1088B000260390932703A0932803B0932903809362
:1088C000220390932303A0932403B093250322272C
:1088D0003327A9012E193F09400B510B8091260324
:1088E00090912703A0912803B09129038217930741
:1088F000A407B507B4F4D801C701885A9146A0402F
:10890000B0408093260390932703A0932803B0934D
:1089100029038093220390932303A0932403B0930D
:1089200025038091160390911703A0911803B0912D
:10893000190380932A0390932B03A0932C03B093E5
:108940002D038091260390912703A0912803B091D5
:1089500029038093460390934703A0934803B09361
:10896000490380911E0390911F03A0912003B091B1
:10897000210380933E0390933F03A0934003B09361
:1089800041038091220390912303A0912403B0918D
:1089900025038093420390934303A0934403B09331
:1089A000450380911A0390911B03A0911C03B09181
:1089B0001D0380933A0390933B03A0933C03B09331
:1089C0003D03809123019091240197FD079603E0D8
:1089D000959587950A95E1F790931408809313086D
:1089E000809121019091220197FD079613E09595C2
:1089F00087951A95E1F79093040880930308809176
:108A00000F02909110020F9734F488E19CEF90933D
:108A100014088093130880910F0290911002079719
:108A200034F480E398EF9093140880931308209116
:108A300001012A30A9F480910F0290911002835F06
:108A4000934034F088EE93E09093140880931308D9
:108A500080910F02909110028A5F9340DCF014C065
:108A600080910F0290911002815D974034F088EE62
:108A700093E0909314088093130880910F029091D3
:108A80001002805E974034F080ED97E090931408D8
:108A90008093130880910D0290910E020F9734F489
:108AA00088E19CEF909304088093030880910D0265
:108AB00090910E02079734F480E398EF90930408A6
:108AC000809303082A30A9F480910D0290910E0240
:108AD000835F934034F088EE93E090930408809392
:108AE000030880910D0290910E028A5F9340DCF0A2
:108AF00014C080910D0290910E02815D974034F078
:108B000088EE93E0909304088093030880910D020F
:108B100090910E02805E974034F080ED97E0909344
:108B200004088093030860917C01662309F4AFC0B8
:108B3000409123015091240180916F039091700323
:108B4000481B590B509376034093750320912301E2
:108B500030912401280F391F37FF02C02F5F3F4F8C
:108B6000359527953093700320936F034138510555
:108B70001CF080E890E005C040585F4F34F480E876
:108B80009FEF90937603809375034091210150915C
:108B900022018091710390917203481B590B5093ED
:108BA0007403409373032091210130912201280F17
:108BB000391F37FF02C02F5F3F4F35952795309300
:108BC000720320937103413851051CF080E890E056
:108BD00005C040585F4F34F480E89FEF90937403D2
:108BE00080937303462F55278091750390917603E8
:108BF000849FB001859F700D949F700D11249B017F
:108C000077FF02C0215F3F4FF4E035952795FA9535
:108C1000E1F78091130890911408820F931F9093AD
:108C20001408809313088091730390917403849FB8
:108C3000D001859FB00D949FB00D1124AD019D0111
:108C4000B7FF02C0215F3F4FE4E035952795EA95D5
:108C5000E1F78091030890910408820F931F90938D
:108C60000408809303088091230190912401860FCA
:108C7000971F90932401809323018091210190916B
:108C80002201840F951F909322018093210100916E
:108C90001608109117088091FA079091FB0710169B
:108CA00011065CF59C0197FF04C022273327281B7F
:108CB000390BC901AA2797FDA095BA2F2091700101
:108CC000332744275527BC01CD010E9493909B0177
:108CD000AC0197FF04C0215C3F4F4F4F5F4F76E0E0
:108CE00055954795379527957A95D1F78091110835
:108CF00090911208820F931F27C097FF03C0909591
:108D000081959F4FAA2797FDA095BA2F20917001BA
:108D1000332744275527BC01CD010E9493909B0126
:108D2000AC0197FF04C0215C3F4F4F4F5F4F66E09F
:108D300055954795379527956A95D1F780911108F4
:108D400090911208821B930B909312088093110844
:108D5000E0901E08F0901F088091FE079091FF0799
:108D60001E141F045CF59C0197FF04C022273327C3
:108D7000281B390BC901AA2797FDA095BA2F20916E
:108D80007001332744275527BC01CD010E949390E1
:108D90009B01AC0197FF04C0215C3F4F4F4F5F4FD9
:108DA00096E055954795379527959A95D1F78091F7
:108DB000050890910608820F931F27C097FF03C0F4
:108DC000909581959F4FAA2797FDA095BA2F209146
:108DD0007001332744275527BC01CD010E94939091
:108DE0009B01AC0197FF04C0215C3F4F4F4F5F4F89
:108DF00086E055954795379527958A95D1F78091C7
:108E0000050890910608821B930B909306088093A7
:108E1000050880914B0887FF44C0B989BB2309F03E
:108E200040C08091CE028823E1F5E1E0EE16E1E05A
:108E3000FE064CF080911308909114088E0D9F1D32
:108E4000805091400DC0F0E0EF16FFEFFF0664F494
:108E500080911308909114088E0D9F1D80509F4F94
:108E6000909314088093130821E0013012074CF00E
:108E70008091030890910408800F911F80509140C9
:108E80000CC03FEF0030130764F480910308909109
:108E90000408800F911F80509F4F90930408809387
:108EA0000308E2E1CD5E0C943E918091EB028823B1
:108EB00001F58091B4028C7F8093B402A1E3B4E009
:108EC000E1E3F7E09BE08091C101882309F48C93F2
:108ED0008D91818312829150389697FFF4CF8091C3
:108EE000C101882359F08091C10181508093C10153
:108EF00005C08091B40281608093B40280913602F3
:108F0000882319F0109236020895809338028093D6
:108F10003A02809134028E7F8093340285EA8093F6
:108F2000BC000895CF93DF93ADEEB2E0C4E6D6E087
:108F300057E09991E92FFF27EE0FFF1FEE56F84FEC
:108F40000190F081E02DE158FF4FEF3FF10521F056
:108F50001CF0EFEFF0E004C0F7FF02C0E0E0F0E04B
:108F6000993111F4EC931BC04C91242F3327E21755
:108F7000F307A9F0CF01821B930B97FD03969595FC
:108F8000879595958795242F280F2C93822F9927C5
:108F9000E817F90714F4215001C02F5F2C935150AA
:108FA000119657FFC6CF80916E06883F38F0EFEFDD
:108FB000F0E0E81BF109E351FD4F808180938201CD
:108FC00080918201882329F0843618F084E680930A
:108FD000820180917006883F38F0EFEFF0E0E81BE7
:108FE000F109E351FD4F80818093800180918001E0
:108FF000882329F0843618F084E6809380018091DC
:109000007D06883F38F0EFEFF0E0E81BF109E3510F
:10901000FD4F808180937B0180917B018B3010F428
:109020008AE002C08F3F11F480937B018091AA06F1
:10903000883F38F0EFEFF0E0E81BF109E351FD4F16
:10904000808180932A0880912A08863010F485E078
:1090500002C08F3F11F480932A088091AC06883FAC
:1090600038F0EFEFF0E0E81BF109E351FD4F8081AC
:109070008093520880915208863010F485E002C037
:109080008F3F11F48093520880919706873F19F41F
:10909000429905C006C0863F31F4439B02C08CE86C
:1090A0000BC086E409C0883F38F0EFEFF0E0E81B22
:1090B000F109E351FD4F8081809327088091980644
:1090C000873F19F4429905C006C0863F31F4439B9F
:1090D00002C08CE80BC086E409C0883F38F0EFEF8F
:1090E000F0E0E81BF109E351FD4F80818093000817
:1090F00080919906883F38F0EFEFF0E0E81BF10926
:10910000E351FD4F80818093300880916F06883F46
:1091100038F0EFEFF0E0E81BF109E351FD4F8081FB
:109120008093810180917206883F38F0EFEFF0E084
:10913000E81BF109E351FD4F808180937F0180910D
:109140007406883F38F0EFEFF0E0E81BF109E351D7
:10915000FD4F808180937D0180917C06883F38F0AF
:10916000EFEFF0E0E81BF109E351FD4F80818093C0
:109170007E0180917E06883F38F0EFEFF0E0E81B3B
:10918000F109E351FD4F808180937A0180917F0640
:10919000883F38F0EFEFF0E0E81BF109E351FD4FB5
:1091A000808180937C0180918006883F38F0EFEFCA
:1091B000F0E0E81BF109E351FD4F808180937901D4
:1091C00080918106883F38F0EFEFF0E0E81BF1096D
:1091D000E351FD4F80818093780180918706883F1D
:1091E00038F0EFEFF0E0E81BF109E351FD4F80812B
:1091F0008093760180918806883F38F0EFEFF0E0A9
:10920000E81BF109E351FD4F80818093C9028091F1
:109210008906883F38F0EFEFF0E0E81BF109E351F1
:10922000FD4F80818093C80280918A06883F38F084
:10923000EFEFF0E0E81BF109E351FD4F80818093EF
:10924000C70280918B06883F38F0EFEFF0E0E81B13
:10925000F109E351FD4F80818093C6028091A506FC
:10926000883F38F0EFEFF0E0E81BF109E351FD4FE4
:1092700080818093C5028091A606883F38F0EFEF89
:10928000F0E0E81BF109E351FD4F80818093C402B7
:109290008091A706883F38F0EFEFF0E0E81BF10976
:1092A000E351FD4F80818093C3028091A806883FDF
:1092B00038F0EFEFF0E0E81BF109E351FD4F80815A
:1092C0008093C20280918C06883F38F0EFEFF0E087
:1092D000E81BF109E351FD4F808180937501809176
:1092E0009006883F38F0EFEFF0E0E81BF109E3511A
:1092F000FD4F80818093740180919A06883F38F0F9
:10930000EFEFF0E0E81BF109E351FD4F808180931E
:10931000730180919D06883F38F0EFEFF0E0E81B85
:10932000F109E351FD4F80818093720180919E0687
:10933000883F38F0EFEFF0E0E81BF109E351FD4F13
:1093400080818093710180919F06883F38F0EFEF14
:10935000F0E0E81BF109E351FD4F8081809370013B
:109360008091C606883F38F0EFEFF0E0E81BF10986
:10937000E351FD4F808180930F089091C1039923A1
:1093800021F080910F08981720F080910F08882312
:1093900011F490930F0880916C0680934B08809194
:1093A000CC0680932F088091A406883F38F0EFEF19
:1093B000F0E0E81BF109E351FD4F808180936F01DC
:1093C0008091BF06883F38F0EFEFF0E0E81BF1092D
:1093D000E351FD4F80818093620880917601282FB0
:1093E00033272F5F3F4F8CE398E2B9010E94D29060
:1093F000709384016093830180917A06809353086F
:1094000080917906809318089091C1069333E0F11A
:1094100081E08093C102983F58F0EFEFF0E0E91B44
:10942000F109E351FD4F8081823310F41092C102A3
:10943000809185012091C1028217B1F0833088F4B8
:10944000222319F08CED95E002C088EC90E0909317
:10945000EE018093ED0185E08093D6022093850193
:1094600003C08150809385018091A2089091A30848
:1094700097FF0FC08091C102882359F080912C047E
:10948000806880932C0405C01092C1028AE080930A
:1094900085018091A2089091A30897FF1DC080913B
:1094A000EB028823C9F08091C1028823A9F0809142
:1094B0000701909108018F5F9F4F71F488E99AE34B
:1094C0009093EE018093ED0180E094EA909308017F
:1094D000809307011092C1028091C102882369F034
:1094E0008091B30281608093B30280917201823DCA
:1094F00048F4825E8093720105C08091B3028E7F32
:109500008093B302DF91CF910895A7E1B0E0EBE83B
:10951000FAE40C9422910E94A33F8091CD0682FF31
:1095200027C08091D0029091D1020097F1F002E023
:1095300088359007D4F49C0197FF02C02D5F3F4F00
:109540003595279535952795809184069927289FED
:10955000A001299F500D389F500D1124CA0164E6C7
:1095600070E00E94D290CB0106C08DE290E003C073
:109570008091840699279093B2028093B102609102
:10958000F6027091F7027A8369838091180899270F
:109590000A966817790714F49A8389838091EC02FC
:1095A000843608F06AC08091B30282FD66C0809163
:1095B0008B0390918C03009731F0019790938C036B
:1095C00080938B030BC01092EB029093B6028093B2
:1095D000B5028091B4028D7E8093B4028091010126
:1095E0008A3011F0843110F0289A01C028988091B7
:1095F000B5029091B602895E9340E0F18091E60851
:109600008536C0F18091B1029091B2029A8389832C
:109610008091B40280618093B40280916006A82F8B
:10962000BB27AA0FBB1FFD01EA53F84F118210821E
:1096300080916106282F3327220F331FC9018A53D7
:10964000984FFC0111821082AE56B84F11961C92B1
:109650001E922E56384FD90111961C921E9280915F
:109660006306E82FFF27EE0FFF1FEE56F84F11821B
:109670001082B4C21092EB02B1C28091EC028D381C
:1096800008F4ACC28091B4028F7E8093B4029091B2
:10969000850682E3989FC001112490938C038093E8
:1096A0008B03E981FA81B9978CF08091EB028823D2
:1096B00069F08091B5029091B602FFEF8F3F9F074E
:1096C00029F001969093B6028093B5028091B5027D
:1096D0009091B6028F3F910509F008F510920E03A4
:1096E00010920F03109210031092110310920A03AC
:1096F00010920B0310920C0310920D03109277033B
:10970000109278031092790310927A031092160344
:1097100010921703109218031092190305C080913C
:10972000B40282608093B40280916206E82FFF2722
:10973000EE0FFF1FEE56F84F808191818135910524
:109740002CF480911104882309F437C12091EB0295
:10975000222309F032C180916306E82FFF27EE0F24
:10976000FF1FEE56F84F808191818C3491050CF4E7
:1097700001C180918D038F5F80938D03893C08F434
:109780001CC120938D031092B6021092B502309145
:109790006006E32FFF27EE0FFF1FEE56F84F808184
:1097A000918187349105B4F480916106E82FFF27F9
:1097B000EE0FFF1FEE56F84F808191810190F081EE
:1097C000E02DF7FF03C0F095E195FF4FE734F10579
:1097D0000CF478C041E020916106A22FBB27AA0FAC
:1097E000BB1FAE56B84F8D919C9111978734910550
:1097F00044F0E32FFF27EE0FFF1FEE56F84F808156
:1098000091818D919C918734910574F080916006CF
:10981000E82FFF27EE0FFF1FEE56F84F8081918152
:10982000873491050CF042E0E22FFF27EE0FFF1F77
:10983000EE56F84F808191818634910574F48091C1
:109840006006E82FFF27EE0FFF1FEE56F84F8081CE
:109850009181873491050CF043E0E22FFF27EE0F52
:10986000FF1FEE56F84F808191818A5B9F4F74F401
:1098700080916006E82FFF27EE0FFF1FEE56F84F8E
:1098800080819181873491050CF044E0E22FFF271D
:10989000EE0FFF1FEE56F84F808191818A5B9F4F3C
:1098A00074F480916006E82FFF27EE0FFF1FEE563D
:1098B000F84F80819181863491050CF445E0842F26
:1098C0000E94793180916106E82FFF27EE0FFF1F7C
:1098D000EE56F84F808191810190F081E02DF7FFE5
:1098E00003C0F095E195FF4F7E97CCF48091600620
:1098F000E82FFF27EE0FFF1FEE56F84F8081918172
:109900008A5B9F4F64F481E0809347041092D702F2
:1099100088EE93E09093EE018093ED014EC00E949B
:1099200082320E94243180E00E949F098091860645
:109930000E94988C80914B0880FF10C080911B0181
:1099400090911C01875B934038F480911B019091AA
:109950001C018E5E924010F40E94FD1F1092EB01DC
:1099600080E00E94F23C81E08093D7028093EB017B
:10997000579A1AC080819181855B9F4FE4F4809152
:109980008D038F5F80938D03893CB8F02093EB02A9
:1099900020938D031092B6021092B50281E00E94CE
:1099A000F23C81E08093D7020E94823268E770E047
:1099B0000E94233C02C020938D0380916206E82F11
:1099C000FF27EE0FFF1FEE56F84F808191818B5AD3
:1099D0009F4F0CF003C130911104332309F0FEC0F6
:1099E0004091EB02E0916306442309F0CCC0FF27CD
:1099F000EE0FFF1FEE56F84F80819181855B9F4FE0
:109A00000CF0BEC02091C206E22FFF27EE0FFF1F11
:109A1000EE56F84F80819181855B9F4F1CF0222389
:109A200009F0AEC080918E038F5F80938E03893CD6
:109A300008F4D4C040938E0380912C04882309F04D
:109A400098C08091D702882309F493C08091C603FF
:109A5000882309F08EC081E090E09093B602809355
:109A6000B50281E08093EB021092770310927803A5
:109A70001092790310927A03109216031092170332
:109A800010921803109219031092120310921303EC
:109A9000109214031092150380917B06E82EFF2488
:109AA0000027112780914F08909150089C0144276E
:109AB00037FD4095542FC801B7010E949390DC01F7
:109AC000CB018093260390932703A0932803B093A0
:109AD000290380915F08909160089C01442737FD1D
:109AE0004095542FC801B7010E949390DC01CB012F
:109AF00080931E0390931F03A0932003B093210330
:109B00008091460390914703A0914803B091490387
:109B10008093220390932303A0932403B0932503FF
:109B200080913E0390913F03A0914003B091410387
:109B300080931A0390931B03A0931C03B0931D03FF
:109B400010920E0310920F03109210031092110343
:109B500010920A0310920B0310920C0310920D0343
:109B60008091B40288608093B40284E68093D60228
:109B700035C08CED95E09093EE018093ED012EC001
:109B800010928E032BC0FF27EE0FFF1FEE56F84FEB
:109B9000808191818C349105FCF02091C206E22FE6
:109BA000FF27EE0FFF1FEE56F84F80819181855BF6
:109BB0009F4F14F0222381F480918F038F5F809355
:109BC0008F03893C58F03093EB0230938F0310924F
:109BD000B6021092B50202C010928F038091480124
:109BE000815080934801809148018F3F21F08091FE
:109BF000B40284FFA9C30E949247B0907606809178
:109C00009803909199039C01220F331F280F391F4D
:109C1000C0906006AC2DBB27AA0FBB1FFD01EE56FE
:109C2000F84F4B2D552780819181849FF001859FAE
:109C3000F00D949FF00D11242E0F3F1F37FF02C02F
:109C40002D5F3F4FB9017595679575956795AA5337
:109C5000B84F80917706082F11278D919C91809F96
:109C60007001819FF00C909FF00C11246E0D7F1DF0
:109C7000709399036093980380919A0390919B034A
:109C80009C01220F331F280F391FD0906106AD2D84
:109C9000BB27AA0FBB1FFD01EE56F84F80819181B3
:109CA000849FF001859FF00D949FF00D11242E0FDD
:109CB0003F1F37FF02C02D5F3F4FA90155954795C4
:109CC00055954795AA53B84F8D919C91809F7001EF
:109CD000819FF00C909FF00C11244E0D5F1D50934E
:109CE0009B0340939A038091C102882309F448C0E2
:109CF000CB0177FD0396DC01B595A795B595A795A2
:109D0000CA0157FD0396FC01F595E795F595E79592
:109D10008091A401682F772767FD70956A9F900155
:109D20006B9F300D7A9F300D11248091C803482F0E
:109D3000552747FD50954E9FC0014F9F900D5E9F48
:109D4000900D1124280F391F37FF02C0295F3F4FA4
:109D500093E0359527959A95E1F73093FD0220938E
:109D6000FC026E9F90016F9F300D7E9F300D11247D
:109D70004A9FC0014B9F900D5A9F900D11243FC0E8
:109D80008091C006E82FFF27E05BFE4F868180931D
:109D9000A40190819093C803A82FBB27A7FDB0957D
:109DA000A69F9001A79F300DB69F300D1124E92F7B
:109DB000FF27E7FDF095E49FC001E59F900DF49F1C
:109DC000900D1124280F391F37FF02C0295F3F4F24
:109DD00083E0359527958A95E1F73093FD0220932E
:109DE000FC02A49F9001A59F300DB49F300D11245B
:109DF000E69FC001E79F900DF69F900D1124281B50
:109E0000390B37FF02C0295F3F4F03E03595279597
:109E10000A95E1F73093FB022093FA0280916306E2
:109E2000E82FFF27EE0FFF1FEE56F84F808191813C
:109E3000909581959F4F9093F9028093F802853019
:109E4000910514F0049705C00FEF8C3F900734F490
:109E500004969093F9028093F80204C01092F902DC
:109E60001092F8028091B403882309F43EC0282F91
:109E700033278091FC029091FD0297FD079613E035
:109E8000959587951A95E1F7289FA001299F500D78
:109E9000389F500D1124CA0157FD0F96B4E09595D7
:109EA0008795BA95E1F79093FD028093FC0280912B
:109EB000FA029091FB0297FD0796A3E0959587958E
:109EC000AA95E1F7289FB001299F700D389F700D6A
:109ED0001124CB0177FD0F96F4E095958795FA95BF
:109EE000E1F79093FB028093FA028090FC0290903D
:109EF000FD028091B7039091B803881A990A909255
:109F0000FD028092FC020091FA021091FB02809106
:109F1000B5039091B603081B190B1093FB02009335
:109F2000FA0280916206E82FFF27EE0FFF1FEE5620
:109F3000F84FE080F1808FE790E0E80EF91EF09294
:109F4000F702E092F60280917B019927AA2797FDFC
:109F5000A095BA2FBC01CD010E940790DC01CB0176
:109F600020E030E040E251E4BC01CD010E94758F59
:109F7000DC01CB01BC01CD010E94D98FDC01CB01FA
:109F80008093590880917A018093310880917901FA
:109F90009927AA2797FDA095BA2FBC01CD010E9451
:109FA0000790DC01CB0120E030E040E251E4BC014D
:109FB000CD010E94758FDC01CB01BC01CD010E9457
:109FC000D98FDC01CB0180930A08809178018093BE
:109FD00020088091530480FF59C080916208813825
:109FE00008F454C080914C04992787FD90952B2D3F
:109FF0003327829FD001839FB00D929FB00D112413
:10A000008A0E9B1E9092FD028092FC0280914D046C
:10A01000992787FD9095829FF001839FF00D929F75
:10A02000F00D11240E0F1F1F1093FB020093FA0274
:10A0300080914E04282F332727FD30958091F80218
:10A040009091F902820F931F9093F9028093F80286
:10A0500080915004282F332727FD30958091710679
:10A060009927289F8001299F100D389F100D1124DA
:10A0700010934F0100934E0180914F0499278E1544
:10A080009F0524F49093F7028093F6028091F602E4
:10A090009091F70297FF04C01092F7021092F60217
:10A0A00080914B0882FF02C0109231084091FC025F
:10A0B0005091FD02CA0157FD03969C0135952795E5
:10A0C0003595279537FF03C0309521953F4F8091F7
:10A0D000B9029091BA0282179307B4F4CA0157FFEC
:10A0E00003C0909581959F4F97FD03969595879511
:10A0F000959587959093BA028093B902853691051C
:10A1000044F084E690E001C001979093BA028093F6
:10A11000B9024091FA025091FB02CA0157FD039621
:10A120009C01359527953595279537FF03C03095C8
:10A1300021953F4F8091B7029091B8028217930703
:10A14000B4F4CA0157FF03C0909581959F4F97FDC6
:10A15000039695958795959587959093B8028093EA
:10A16000B7028536910544F084E690E001C001977E
:10A170009093B8028093B7028091B40284FF08C024
:10A180001092BA021092B9021092B8021092B7025D
:10A19000ED2DFF27EE0FFF1FEE56F84F40919B0667
:10A1A000242F3327808191812817390744F4809127
:10A1B000CA0682FF04C081E08093CD0213C0ED2D5A
:10A1C000FF27EE0FFF1FEE56F84F842F992720919F
:10A1D0009C06821B9109208131812817390714F4CC
:10A1E0001092CD0240916106E42FFF27EE0FFF1F72
:10A1F000EE56F84F50919B06852F9927222733273B
:10A20000281B390B808191818217930744F4809138
:10A21000CA0683FF04C081E08093CC0216C08091FF
:10A22000CC02882391F0E42FFF27EE0FFF1FEE569C
:10A23000F84F80919C069927851B910920813181D7
:10A240008217930714F41092CC02EC2DFF27EE0F27
:10A25000FF1FEE56F84F40919B06242F3327808135
:10A2600091812817390744F48091CA0680FF04C001
:10A2700081E08093CA0217C08091CA02882399F0B6
:10A28000EC2DFF27EE0FFF1FEE56F84F842F992776
:10A2900020919C06821B9109208131812817390762
:10A2A00014F41092CA0240916006E42FFF27EE0FCB
:10A2B000FF1FEE56F84F50919B06852F99272227B6
:10A2C0003327281B390B808191818217930744F42F
:10A2D0008091CA0681FF04C081E08093CB0216C042
:10A2E0008091CB02882391F0E42FFF27EE0FFF1F10
:10A2F000EE56F84F80919C069927851B9109208185
:10A3000031818217930714F41092CB028091CD0211
:10A31000882319F48091CC02811181E08093CE02D0
:10A320008091CA02882321F48091CB02882351F0C6
:10A3300081E08093CF021092CE021092CD02109253
:10A34000CC0202C08093CF028091CE02882321F4F8
:10A350008091CF02882369F080919A0699272981FC
:10A360003A818217930714F49A83898381E080935A
:10A3700002038091B30299279C012470307082FF00
:10A380002DC08091B7039091B803909581959F4F10
:10A390009093FD028093FC028091B5039091B603E7
:10A3A000909581959F4F9093FB028093FA02809144
:10A3B0008801909189019093F7028093F602809131
:10A3C0004B088B778B6680934B0880912F088C7B92
:10A3D00080932F0888EC809381011EC08091B40285
:10A3E00084FF1AC03093F9022093F8023093FD02E3
:10A3F0002093FC023093FB022093FA029AE590939B
:10A40000590888E78093310890930A0880932008C0
:10A410001092CE021092CF028091230890912408CE
:10A42000A0912508B091260820914603309147035A
:10A430004091480350914903820F931FA41FB51FF9
:10A440008093230890932408A0932508B0932608AE
:10A4500080912B0890912C08A0912D08B0912E0886
:10A46000E0903E03F0903F030091400310914103C0
:10A47000EB82FC820D831E838E0D9F1DA01FB11FDA
:10A4800080932B0890932C08A0932D08B0932E084E
:10A4900080911A0890911B08A0911C08B0911D088A
:10A4A000E0904203F0904303009144031091450370
:10A4B000EF82F88609871A878E0D9F1DA01FB11F96
:10A4C00080931A0890931B08A0931C08B0931D0852
:10A4D00080910B0890910C08A0910D08B0910E0886
:10A4E000E0903A03F0903B0300913C0310913D0350
:10A4F000EB86FC860D871E878E0D9F1DA01FB11F4A
:10A5000080930B0890930C08A0930D08B0930E084D
:10A51000F090CF02FF86FF2029F48091CE0288239D
:10A5200009F460C01092360310923703109238037A
:10A5300010923903109232031092330310923403B5
:10A5400010923503109223081092240810922508C7
:10A550001092260810922B0810922C0810922D08A9
:10A5600010922E0810921A0810921B0810921C08C4
:10A5700010921D0810920B0810920C0810920D08F2
:10A5800010920E088091260390912703A091280332
:10A59000B09129038093220390932303A093240373
:10A5A000B093250380911E0390911F03A091200377
:10A5B000B091210380931A0390931B03A0931C0373
:10A5C000B0931D031092FD011092FC011092D30272
:10A5D0001092D2021092D5021092D4020F8500235D
:10A5E00009F0F8C18091CE02882309F0F3C180916F
:10A5F000010690910206815092402CF48091EB026A
:10A60000882309F4E7C19090DB08A0907B06209096
:10A610004F083090500840905F085090600819141F
:10A620000CF0E3C0BB24CC24DD24CA01B901A6018F
:10A6300095010E94079179018A018091A408909167
:10A64000A508281A390AC101AA2797FDA095BA2F93
:10A65000E81AF90A0A0B1B0B6B817C818D819E81A4
:10A66000A60195010E94079159016A018091A608EF
:10A670009091A708481A590AC201AA2797FDA095E8
:10A68000BA2FA81AB90ACA0ADB0A292C332427FCD4
:10A690003094432C532CC801B701A20191010E94B0
:10A6A000939097FF04C061507E4F8F4F9F4F3B01A7
:10A6B0004C0109E095948794779467940A95D1F7B3
:10A6C000C601B501A20191010E94939097FF04C0B9
:10A6D00061507E4F8F4F9F4F5B016C0119E0D59405
:10A6E000C794B794A7941A95D1F78091B902909125
:10A6F000BA02813491053CF48091B7029091B8027E
:10A7000081349105D4F0D401C30197FE03C00196B2
:10A71000A11DB11D3C014D019594879477946794D8
:10A72000D601C501D7FE03C00196A11DB11D5C0174
:10A730006D01D594C794B794A79480916306E82FD0
:10A74000FF27EE0FFF1FEE56F84F80819181019099
:10A75000F081E02DF7FF03C0F095E195FF4F7A9768
:10A76000A4F0C401B30123E030E040E050E00E94D7
:10A77000079139014A01C601B50123E030E040E00C
:10A7800050E00E94079159016A018091DD08282F4D
:10A79000332727FD3095432F532F261537054805BE
:10A7A000590514F439014A01992787FD9095909530
:10A7B00081959F4FAA2797FDA095BA2F6816790615
:10A7C0008A069B0614F43C014D012A153B054C05F5
:10A7D0005D0514F459016A01A816B906CA06DB061C
:10A7E0000CF0D0C05C016D01CDC0EA2CFF24002725
:10A7F0001127CA01B901A80197010E9407913901E7
:10A800004A01C101AA2797FDA095BA2F681A790AB3
:10A810008A0A9B0A6B817C818D819E81A8019701A8
:10A820000E94079159016A01C201AA2797FDA095CC
:10A83000BA2FA81AB90ACA0ADB0AD401C30197FEC3
:10A8400003C00F96A11DB11D3C014D01F4E095948C
:10A85000879477946794FA95D1F7D601C501D7FE0E
:10A8600003C00F96A11DB11D5C016D01E4E0D594FC
:10A87000C794B794A794EA95D1F78091B9029091C3
:10A88000BA02813491053CF48091B7029091B802EC
:10A8900081349105A4F0C401B30123E030E040E02D
:10A8A00050E00E94079139014A01C601B50123E039
:10A8B00030E040E050E00E94079159016A01809128
:10A8C0006306E82FFF27EE0FFF1FEE56F84F80813B
:10A8D00091810190F081E02DF7FF03C0F095E195A3
:10A8E000FF4F7A97A4F0C401B30123E030E040E0C9
:10A8F00050E00E94079139014A01C601B50123E0E9
:10A9000030E040E050E00E94079159016A0189E17E
:10A910008093940121E262167104810491042CF069
:10A9200070E2672E712C812C912C30EE63163FEF74
:10A9300073063FEF83063FEF930644F460EE662E06
:10A940006FEF762E6FEF862E6FEF962E41E2A416F4
:10A95000B104C104D1042CF050E2A52EB12CC12CBD
:10A96000D12C50EEA5165FEFB5065FEFC5065FEF81
:10A97000D50644F440EEA42E4FEFB42E4FEFC42E74
:10A980004FEFD42E8091260390912703A0912803A6
:10A99000B091290386199709A809B909809326035C
:10A9A00090932703A0932803B093290380911E035B
:10A9B00090911F03A0912003B09121038A199B0954
:10A9C000AC09BD0980931E0390931F03A09320033D
:10A9D000B09321038091FC019091FD018F3F91057F
:10A9E00009F008F4C4C56F85662309F04EC580914F
:10A9F000CE02882309F049C580910203882309F01B
:10AA000044C57091A306788B772309F43EC58091E5
:10AA1000230890912408A0912508B0912608B7FF3B
:10AA200004C081509F4FAF4FBF4FE92EFA2E0B2F1E
:10AA3000112707FD1A95E0922308F092240800934D
:10AA400025081093260880912B0890912C08A0913E
:10AA50002D08B0912E08B7FF04C081509F4FAF4F13
:10AA6000BF4F892F9A2FAB2FBB27A7FDBA95898B94
:10AA70009A8BAB8BBC8B80932B0890932C08A09364
:10AA80002D08B0932E0880917B06A82EBB24CC24E1
:10AA9000DD242091360330913703409138035091E3
:10AAA0003903C601B5010E94939097FF04C061501D
:10AAB0007F4F8F4F9F4F672E782E892E992487FCCA
:10AAC0009A94609236037092370380923803909282
:10AAD0003903209132033091330340913403509174
:10AAE0003503C601B5010E94939097FF04C06150E1
:10AAF0007F4F8F4F9F4F272E382E492E552447FCCE
:10AB00005A9420923203309233034092340350928D
:10AB1000350380912E0390912F03A0913003B091C3
:10AB20003103B7FF04C081509F4FAF4FBF4F892FF4
:10AB30009A2FAB2FBB27A7FDBA9580932E03909336
:10AB40002F03A0933003B0933103D801C7018619B6
:10AB50009709A809B9098093830390938403A0936C
:10AB60008503B09386032091A206E22EFF240027DE
:10AB70001127BC01CD01A80197010E94079159013D
:10AB80006A01209390033093910340939203509372
:10AB9000930389899A89AB89BC8982199309A4098D
:10ABA000B5098093870390938803A0938903B0939A
:10ABB0008A03BC01CD01A80197010E94079120934F
:10ABC0009403309395034093960350939703D601D3
:10ABD000C501D7FE04C081509F4FAF4FBF4F892F93
:10ABE0009A2FAB2FBB27A7FDBA959093D3028093E2
:10ABF000D20257FF04C021503F4F4F4F5F4FBB273A
:10AC000057FDBA95A52F942F832F9093D50280934B
:10AC1000D4028091B9029091BA0281349105DCF49A
:10AC20008091B7029091B80281349105A4F480918B
:10AC30006306E82FFF27EE0FFF1FEE56F84F8081C7
:10AC400091810190F081E02DF7FF03C0F095E1952F
:10AC5000FF4F7A97E4F08091DB088F3FC1F4809139
:10AC6000D2029091D30297FD019695958795909386
:10AC7000D3028093D2028091D4029091D50297FDA5
:10AC80000196959587959093D5028093D4028091F3
:10AC90001A0890911B08A0911C08B0911D08B7FFDD
:10ACA00004C081509F4FAF4FBF4F892F9A2FAB2FBA
:10ACB000BB27A7FDBA9580931A0890931B08A09311
:10ACC0001C08B0931D0880910B0890910C08A0916E
:10ACD0000D08B0910E08B7FF04C081509F4FAF4FD1
:10ACE000BF4F892F9A2FAB2FBB27A7FDBA95809313
:10ACF0000B0890930C08A0930D08B0930E08809158
:10AD0000460390914703A0914803B09149032F81D6
:10AD1000388549855A85281B390B4A0B5B0B2093D4
:10AD20007B0330937C0340937D0350937E0380919B
:10AD30003E0390913F03A0914003B0914103EB8407
:10AD4000FC840D851E85E81AF90A0A0B1B0BE0929C
:10AD50007F03F0928003009381031093820320937A
:10AD60008303309384034093850350938603E092DA
:10AD70008703F09288030093890310938A038091DC
:10AD8000220390912303A0912403B0912503821BF9
:10AD9000930BA40BB50B8093220390932303A093F2
:10ADA0002403B093250380911A0390911B03A09173
:10ADB0001C03B0911D038E199F09A00BB10B80934A
:10ADC0001A0390931B03A0931C03B0931D0388895F
:10ADD0008823E1F0209100033091010321383105EF
:10ADE0004CF080915703909158030196909358032B
:10ADF0008093570320583F4F4CF480915703909114
:10AE000058030197909358038093570310920103BE
:10AE10001092000381E090E090939D0380939C0347
:10AE2000E0908303F09084030091850310918603E2
:10AE3000D801C70117FF07C088279927DC018E19A1
:10AE40009F09A00BB10B81509240A040B04034F05C
:10AE500084E090E090939D0380939C038091A203F3
:10AE60009091A303A091A403B091A503209123087E
:10AE7000309124084091250850912608821B930B9D
:10AE8000A40BB50B815E914BAF4FBF4F8F539C49C5
:10AE9000A040B04028F08091DC0889310CF4FFC05C
:10AEA00021E0E21620E1F20620E0020720E012078E
:10AEB0000CF473C080919E03882309F46AC0D80102
:10AEC000C70117FF07C088279927DC018E199F0942
:10AED000A00BB10B9C01AD01B7FF04C021503E4F48
:10AEE0004F4F5F4FF9E05595479537952795FA9560
:10AEF000D1F780919C0390919D03820F931F9093B3
:10AF00009D0380939C03D801C70117FF03C00796D8
:10AF1000A11DB11DE3E0B595A79597958795EA9595
:10AF2000D1F78093900390939103A0939203B093F1
:10AF3000930389589341A040B04064F088E893E1BE
:10AF4000A0E0B0E08093900390939103A0939203CC
:10AF5000B093930320919003309191034091920319
:10AF60005091930357FF04C021503F4F4F4F5F4F05
:10AF7000232F342F452F552747FD5A958091D20214
:10AF80009091D302820F931F9093D3028093D202A9
:10AF900006C081E080939E0302C010929E0340E0B1
:10AFA000E41640EFF4064FEF04074FEF14070CF0E0
:10AFB00073C080919F03882309F46AC0D801C70138
:10AFC00017FF07C088279927DC018E199F09A00B5E
:10AFD000B10B9C01AD01B7FF04C021503E4F4F4F54
:10AFE0005F4F69E055954795379527956A95D1F755
:10AFF00080919C0390919D03820F931F90939D03DA
:10B0000080939C03D801C70117FF03C00796A11DB9
:10B01000B11D23E0B595A795979587952A95D1F70A
:10B020008093900390939103A0939203B093930322
:10B0300088579C4EAF4FBF4F64F488E79CEEAFEF4C
:10B04000BFEF8093900390939103A0939203B093EA
:10B05000930320919003309191034091920350917A
:10B06000930357FF04C021503F4F4F4F5F4F232F93
:10B07000342F452F552747FD5A958091D202909144
:10B08000D302820F931F9093D3028093D20211C0F8
:10B0900081E080939F030DC010929F030AC010921D
:10B0A0009D0310929C0384E690E09093930180931B
:10B0B00092016889262F332780919C0390919D03EC
:10B0C0002817390724F430939D0320939C03109193
:10B0D000DC08112379F0212F332727FD309580914B
:10B0E0009C0390919D032817390724F430939D0306
:10B0F00020939C03409183035091840360918503C6
:10B1000070918603413851056105710574F0809195
:10B110005B0390915C0320919C0330919D03820F0F
:10B12000931F90935C0380935B0340585F4F6F4F76
:10B130007F4F74F480915B0390915C0320919C039A
:10B1400030919D03821B930B90935C0380935B0370
:10B1500081E090E090939D0380939C03C0908703CF
:10B16000D0908803E0908903F0908A03D701C6014C
:10B17000F7FE07C088279927DC018C199D09AE09C5
:10B18000BF0981509240A040B04034F084E090E08C
:10B1900090939D0380939C038091A6039091A703B5
:10B1A000A091A803B091A90320912B0830912C08FD
:10B1B00040912D0850912E08821B930BA40BB50BC8
:10B1C000815E914BAF4FBF4F8F539C49A040B04021
:10B1D00018F019310CF4FFC001E0C01600E1D006F0
:10B1E00000E0E00600E0F0060CF473C08091A003DC
:10B1F000882309F46AC0D701C601F7FE07C0882773
:10B200009927DC018C199D09AE09BF099C01AD018C
:10B21000B7FF04C021503E4F4F4F5F4F09E0559597
:10B220004795379527950A95D1F780919C03909182
:10B230009D03820F931F90939D0380939C03D701DE
:10B24000C601F7FE03C00796A11DB11D13E0B59519
:10B25000A795979587951A95D1F780939403909326
:10B260009503A0939603B093970389589341A04008
:10B27000B04064F088E893E1A0E0B0E080939403EC
:10B2800090939503A0939603B09397032091940312
:10B2900030919503409196035091970357FF04C056
:10B2A00021503F4F4F4F5F4F232F342F452F5527AE
:10B2B00047FD5A958091D4029091D502820F931F39
:10B2C0009093D5028093D40206C081E08093A003BE
:10B2D00002C01092A00320E0C21620EFD2062FEF8A
:10B2E000E2062FEFF2060CF073C08091A1038823D1
:10B2F00009F46AC0D701C601F7FE07C0882799275D
:10B30000DC018C199D09AE09BF099C01AD01B7FF95
:10B3100004C021503E4F4F4F5F4FE9E05595479590
:10B3200037952795EA95D1F780919C0390919D03DD
:10B33000820F931F90939D0380939C03D701C601B6
:10B34000F7FE03C00796A11DB11D73E0B595A79543
:10B35000979587957A95D1F7809394039093950369
:10B36000A0939603B093970388579C4EAF4FBF4F5F
:10B3700064F488E79CEEAFEFBFEF80939403909363
:10B380009503A0939603B093970320919403309173
:10B390009503409196035091970357FF04C02150A5
:10B3A0003F4F4F4F5F4F232F342F452F552747FDDA
:10B3B0005A958091D4029091D502820F931F909359
:10B3C000D5028093D40211C081E08093A1030DC007
:10B3D0001092A1030AC010929D0310929C0384E670
:10B3E00090E090939301809392014889242F332712
:10B3F00080919C0390919D032817390724F4309382
:10B400009D0320939C038091DC08882379F0282FEA
:10B41000332727FD309580919C0390919D03281739
:10B42000390724F430939D0320939C0340918703B4
:10B43000509188036091890370918A0341385105C6
:10B440006105710574F08091590390915A03209120
:10B450009C0330919D03820F931F90935A03809316
:10B46000590340585F4F6F4F7F4FCCF48091590381
:10B4700090915A0320919C0330919D03821B930B62
:10B4800090935A03809359030AC01092D5021092E8
:10B49000D4021092D3021092D20210920203809131
:10B4A0003108882341F41092D5021092D4021092F0
:10B4B000D3021092D2028091230890912408A09187
:10B4C0002508B09126088093A2039093A303A0932C
:10B4D000A403B093A50380912B0890912C08A09110
:10B4E0002D08B0912E088093A6039093A703A093F4
:10B4F000A803B093A9031092360310923703109259
:10B5000038031092390310923203109233031092D1
:10B5100034031092350310922E0310922F031092D1
:10B5200030031092310310922308109224081092D5
:10B5300025081092260810922B0810922C081092C1
:10B540002D0810922E0810921A0810921B081092C3
:10B550001C0810921D0810920B0810920C081092F3
:10B560000D0810920E081092FD011092FC01E0905F
:10B57000F802F090F902C701F7FE04C08827992766
:10B580008E199F0904973CF080914B0884FD03C0FD
:10B5900082E38093D60210917806A12EBB24CC249E
:10B5A000DD24B701882777FD8095982F9701F7FE56
:10B5B00004C0222733272E193F09442737FD409521
:10B5C000542F0E9493909B01AC01C601B5010E94CB
:10B5D000939097FF04C061507E4F8F4F9F4F59E06B
:10B5E00095958795779567955A95D1F79B01812F0A
:10B5F00099278E9DD0018F9DB00D9E9DB00D112479
:10B60000CD01B7FD03969595879595958795280F5C
:10B61000391F8091D8029091D902280F391F4427F1
:10B6200037FD4095542F2093770330937803409350
:10B63000790350937A038091160390911703A09198
:10B640001803B0911903821B930BA40BB50B8093C5
:10B65000160390931703A0931803B0931903815511
:10B66000934CA040B04064F080E593ECA0E0B0E0E3
:10B670008093160390931703A0931803B0931903B4
:10B680008091160390911703A0911803B0911903AC
:10B69000805B9C43AF4FBF4F64F480EB9CE3AFEF04
:10B6A000BFEF8093160390931703A0931803B093F2
:10B6B0001903009196011091970117FDFCC080912C
:10B6C0004B0883FFF8C080919501815080939501CC
:10B6D000882309F0F4C08DE08093950180914603A2
:10B6E00090914703A0914803B0914903B7FF04C06C
:10B6F00081509E4FAF4FBF4F39E0B595A7959795B5
:10B7000087953A95D1F77C0197FF04C0F094E194B6
:10B71000F108F39480913E0390913F03A091400380
:10B72000B0914103B7FF04C081509E4FAF4FBF4F50
:10B7300029E0B595A795979587952A95D1F79C010E
:10B7400097FF03C0309521953F4FE216F3060CF4A6
:10B750007901B701F7FE02C0695F7F4F2B01A3E0BB
:10B7600055944794AA95E1F722E030E0420E531E2B
:10B7700060905B0870905C0880905D0890905E0817
:10B7800020914A0130914B0140914C0150914D0163
:10B79000C401B3010E94079159016A01309309085D
:10B7A00020930808021B130BC801845E9D4F68E6B6
:10B7B00071E00E94D2909C01245B30408091920104
:10B7C00090919301009731F00197909393018093AA
:10B7D00092011BC049E1E416F104BCF4809100031E
:10B7E00090910103820F931F9093010380930003B4
:10B7F0008091D602882349F081508093D602882315
:10B8000021F4B0920503A0920403809192019091DB
:10B810009301892BF9F4809194019927289FB00115
:10B82000299F700D389F700D1124CB01B2010E9429
:10B83000D290CB01AA2797FDA095BA2F680E791E4A
:10B840008A1E9B1E60925B0870925C0880925D0865
:10B8500090925E088091D602882369F58091040356
:10B86000909105032091080830910908821B930BE1
:10B87000845E9D4F68E671E00E94D2909C01245B3B
:10B88000304080917E0186959927289FD001299F7D
:10B89000B00D389FB00D11249D01B7FF02C0215F8C
:10B8A0003F4FF4E035952795FA95E1F73093D902AB
:10B8B0002093D80204C01092D9021092D80280912D
:10B8C0000203882381F010920A0310920B03109256
:10B8D0000C0310920D0310920E0310920F0310929E
:10B8E000100310921103F090CF02FF20F1F4809129
:10B8F0003108282F332744275527809146039091FC
:10B900004703A0914803B0914903BC01CD010E94B7
:10B910009390DC01CB01BC01CD0128EF3AE240E07D
:10B9200050E00E940791390102C066247724E0901C
:10B93000CE02EE20F1F480913108282F33274427DE
:10B94000552780913E0390913F03A0914003B09111
:10B950004103BC01CD010E949390DC01CB01BC01ED
:10B96000CD0128EF3AE240E050E00E940791290122
:10B9700002C0442455248091050890910608893C12
:10B9800091051CF088EC90E005C088539F4F34F47B
:10B9900088E39FEF90930608809305088091110833
:10B9A00090911208893C91051CF088EC90E005C04C
:10B9B00088539F4F34F488E39FEF9093120880934D
:10B9C00011088091130890911408AA2797FDA0955B
:10B9D000BA2F20915908A22EBB24CC24DD24BC010F
:10B9E000CD01A60195010E9493909B01AC0180912D
:10B9F000050890910608AA2797FDA095BA2FE7E0C1
:10BA0000880F991FAA1FBB1FEA95D1F7280F391F6E
:10BA10004A1F5B1F57FF04C0215C3F4F4F4F5F4FD2
:10BA200076E055954795379527957A95D1F7830117
:10BA3000020F131F1093140800931308809103083A
:10BA400090910408AA2797FDA095BA2FBC01CD01BB
:10BA5000A60195010E9493909B01AC018091110871
:10BA600090911208AA2797FDA095BA2F67E0880F3A
:10BA7000991FAA1FBB1F6A95D1F7280F391F4A1FAC
:10BA80005B1F57FF04C0215C3F4F4F4F5F4FF6E0F5
:10BA90005595479537952795FA95D1F74201820E2E
:10BAA000931E90920408809203088091540890910C
:10BAB0005508880F991FAA2797FDA095BA2F2091A6
:10BAC0000A08332744275527BC01CD010E949390D3
:10BAD0005B016C0197FF08C02FE330E040E050E0CD
:10BAE000A20EB31EC41ED51EE6E0D594C794B7942B
:10BAF000A794EA95D1F780912008282F332744276F
:10BB0000552780912A0390912B03A0912C03B0918B
:10BB10002D03BC01CD010E949390DC01CB01BC013F
:10BB2000CD0120EF35E540E050E00E940791B501DE
:10BB3000620F731F709355086093540801501041B1
:10BB400034F080E090E19093140880931308809182
:10BB50001308909114088050904F34F480E090EFD7
:10BB6000909314088093130851E0851650E19506D0
:10BB700034F080E090E19093040880930308809172
:10BB80000308909104088050904F34F480E090EFC7
:10BB900090930408809303086150704134F080E072
:10BBA00090E19093550880935408809154089091A7
:10BBB00055088050904F34F480E090EF90935508F2
:10BBC0008093540880910001482F552780912501CA
:10BBD000909126014817590794F42091250130913E
:10BBE000260109811A81049FC001059F900D149FB1
:10BBF000900D1124B9010E94BE907A836983298136
:10BC00003A81220F331F220F331F3A832983409139
:10BC10004B0840FD02C00C94FB65EE2009F0EBC719
:10BC2000FF2009F0E8C700E010E048018091D00251
:10BC30009091D1029093E3058093E20520915D03FA
:10BC400030915E032115310509F03FC080911B0141
:10BC500090911C018959934058F087B5803F20F49A
:10BC600080910002815011C081E08093B3034EC0E7
:10BC700080911B0190911C018436910508F587B5D0
:10BC80008031D0F0809100028F5F809300029FE0AE
:10BC900089029001112480910B06821B87BD8CE2E2
:10BCA00091E09093EE018093ED018EE591E0909309
:10BCB0005E0380935D032AC081E08093B20326C0B7
:10BCC000F092B203F092B30321C08091E60290910A
:10BCD000E702A091E802B091E90264E0880F991FA1
:10BCE000AA1FBB1F6A95D1F78093010290930202AD
:10BCF000A0930302B09304021093FF010093FE018E
:10BD00002150304030935E0320935D0320918101E8
:10BD100041FF24C02233D8F4809198018150809350
:10BD200098018F3FD9F5109203038091E60290911C
:10BD3000E702A091E802B091E9028093E2029093B9
:10BD4000E302A093E402B093E50281E004C081E045
:10BD50008093030388EC8093980120C080914E016A
:10BD600090914F01820F911D209171063327829F80
:10BD7000A001839F500D929F500D1124CA01AA2744
:10BD800097FDA095BA2F8093E2029093E302A093CF
:10BD9000E402B093E50281E08093030380914603BF
:10BDA00090914703A0914803B0914903E0904A0164
:10BDB000F0904B0100914C0110914D01BC01CD015F
:10BDC000A80197010E94079159016A0180913E03E1
:10BDD00090913F03A0914003B0914103BC01CD017C
:10BDE000A80197010E940791B901C5010E94BC8476
:10BDF0005C01CC971CF05CE3A52EB12CC5010E9420
:10BE000017725C0180E2809349011092E102109266
:10BE1000E00280910303882309F45FC58091B40296
:10BE200099279C012071307084FD57C58091B30221
:10BE300082608093B30270912F08872F992741E089
:10BE4000C42ED12CC822D92280FD04C080914B0879
:10BE500081FD10C0C980DA803093AB032093AA0320
:10BE60003093E1022093E0028091B402806C8093D1
:10BE7000B402ABC28091B40281FF7AC20091880102
:10BE800010918901C8010F962090F6023090F702B8
:10BE9000821593050CF058C08091B203882309F0F5
:10BEA00053C08091B40287FF15C08091B4028F7790
:10BEB0008093B4028091E6029091E702A091E8029B
:10BEC000B091E9028093E2029093E302A093E4022E
:10BED000B093E5028091B40280648093B402E09054
:10BEE0000F08EE20F1F08091E2029091E302A09120
:10BEF000E402B091E502BC01CD0124E630E040E06F
:10BF000050E00E9407918E2D9927AA27BB27821700
:10BF10009307A407B5072CF4D092E102C092E00287
:10BF200010C0C101801B910B0F9797FF03C0909524
:10BF300081959F4F9093E1028093E0028BE2809382
:10BF400049011092DA0216C1C8010F972816390666
:10BF5000C4F52091B3032223A1F58091B40286FF9A
:10BF600015C08091B4028F7B8093B4028091E60269
:10BF70009091E702A091E802B091E9028093E20279
:10BF80009093E302A093E402B093E5028091B4029F
:10BF900080688093B402C101801B910B0F9697FFBC
:10BFA00003C0909581959F4F909581959F4F909359
:10BFB000E1028093E0028DE2809349012093DA024E
:10BFC000D9C08DE3809349016091DB02662371F152
:10BFD0002091DC023091DD024091DE025091DF02BF
:10BFE0008091E2029091E302A091E402B091E50217
:10BFF00082179307A407B507CCF48091B40280643C
:10C000008093B402862F99279093E1028093E002F7
:10C010008AE08093DA028EE5809349018091B40230
:10C0200087FFA8C08091B4028F7733C0662309F4DC
:10C0300043C02091DC023091DD024091DE0250913C
:10C04000DF028091E2029091E302A091E402B091BC
:10C05000E502281739074A075B0774F58091B40297
:10C0600080688093B402862F9927909581959F4F81
:10C070009093E1028093E00286EF8093DA0286E7F4
:10C08000809349018091B40286FF74C08091B4020C
:10C090008F7B8093B4028091E6029091E702A09199
:10C0A000E802B091E9028093E2029093E302A09348
:10C0B000E402B093E5025EC08091B402807C09F492
:10C0C00059C08091DA02882379F5E090E602F09079
:10C0D000E7020091E8021091E902D801C7018058F7
:10C0E0009040A040B0402091E2023091E3024091A4
:10C0F000E4025091E50282179307A407B5075CF4A8
:10C10000D801C70180589F4FAF4FBF4F281739073D
:10C110004A075B075CF08093E2029093E302A093EE
:10C12000E402B093E50202C01092DA028091B402F8
:10C130008F738093B4021092AB031092AA0371FF25
:10C1400006C084EF91E09093EE018093ED01809121
:10C15000EA02882379F48091E6029091E702A091A7
:10C16000E802B091E902C397A105B1051CF081E096
:10C170008093EA026091AA037091AB038091E00280
:10C180009091E102680F791F7093AB036093AA034B
:10C19000CB0177FF04C088279927861B970B855F03
:10C1A00091400CF4CEC04091DA02442389F1809191
:10C1B000DC029091DD022091E2023091E302821BC9
:10C1C000930B0996439748F48091DC029091DD022D
:10C1D000A091DE02B091DF0212C0242F332727FD89
:10C1E0003095432F532F8091E2029091E302A0916A
:10C1F000E402B091E502820F931FA41FB51F809344
:10C20000E2029093E302A093E402B093E50224C01B
:10C21000809171062091E2023091E3024091E402A4
:10C220005091E5021616170644F463E00E94B2909E
:10C23000280F311D411D511D07C063E00E94B290BF
:10C24000281B3109410951092093E2023093E3028E
:10C250004093E4025093E5021092AB031092AA03BC
:10C26000E090E602F090E7020091E8021091E90206
:10C27000D801C70180509440A040B0402091E20214
:10C280003091E3024091E4025091E5028217930756
:10C29000A407B5075CF4D801C70180509C4FAF4F8D
:10C2A000BF4F281739074A075B0744F08093E20223
:10C2B0009093E302A093E402B093E50280912F08EB
:10C2C00081FF06C084E690E09093EE018093ED013B
:10C2D000809175068823A9F58091DB02882389F572
:10C2E0004091D0025091D10257FF02C04D5F5F4F85
:10C2F0005595479555954795809125019091260133
:10C30000209100013327489FF001499FF00D589F6D
:10C31000F00D1124CF01B9010E94D29070938901D0
:10C3200060938801663471051CF486E490E005C0D2
:10C330006739710534F086E990E090938901809324
:10C34000880180915D0390915E03892BD1F18091EA
:10C35000E6029091E702A091E802B091E902809391
:10C36000E2029093E302A093E402B093E50229C0B5
:10C370008091E6029091E702A091E802B091E90273
:10C3800080599140A040B0408093E2029093E30234
:10C39000A093E402B093E50280917506882311F022
:10C3A000992702C088E790E09093890180938801E3
:10C3B000E980FA80F092D102E092D0028EE280937E
:10C3C0004901C090D002D090D102E090E602F090F6
:10C3D000E7020091E8021091E9022091E202309117
:10C3E000E3024091E4025091E5022E153F0540071B
:10C3F000510724F080912F0880FDBBC280915D031E
:10C4000090915E03892B39F0C090D002D090D10278
:10C4100000E010E0D7C0D801C701821B930BA40B2A
:10C42000B50B80937B0390937C03A0937D03B09323
:10C430007E03823000E890070FEFA0070FEFB007F0
:10C440002CF481E090E8AFEFBFEF09C08F5F9F470A
:10C45000A040B04064F08FEF9FE7A0E0B0E0809391
:10C460007B0390937C03A0937D03B0937E030091A4
:10C470007B0310917C0380918001282F3327442770
:10C48000552780917B0390917C03A0917D03B0910F
:10C490007E03BC01CD010E94939097FF04C0615EB2
:10C4A0007F4F8F4F9F4F25E095958795779567959F
:10C4B0002A95D1F760937B0370937C0380937D036F
:10C4C00090937E0365302EEF72072FEF82072FEFD8
:10C4D00092072CF484E09EEFAFEFBFEF09C06050ED
:10C4E00074408040904064F080E094E0A0E0B0E0D0
:10C4F00080937B0390937C03A0937D03B0937E0392
:10C5000080907B0390907C032091FE013091FF018D
:10C5100037FF02C0295F3F4F83E0359527958A9505
:10C52000E1F74FEF223834071CF421E83FEF05C054
:10C530002038310514F020E830E0C901AA2797FD22
:10C54000A095BA2F20918201332744275527BC019B
:10C55000CD010E94939097FF04C06D5F7F4F8F4F76
:10C560009F4FB2E09595879577956795BA95D1F7E6
:10C570009B015FEF613075071CF420E03FEF06C0C0
:10C580006F3F710519F014F020E031E08091B402A2
:10C59000807C49F0C90137FD03969C0135952795AC
:10C5A000359527950DC080912F0880FF09C0C901DE
:10C5B00037FD07969C01F3E035952795FA95E1F74D
:10C5C000820E931E20917F01222309F454C06091B2
:10C5D000060370910703809108039091090397FF68
:10C5E00004C061587F4F8F4F9F4FE7E09595879527
:10C5F00077956795EA95D1F73327442755270E9409
:10C60000939097FF04C0615E7F4F8F4F9F4F55E01F
:10C6100095958795779567955A95D1F760937B03A4
:10C6200070937C0380937D0390937E036138AFEF1A
:10C630007A07AFEF8A07AFEF9A072CF480E89FEFF5
:10C64000AFEFBFEF0AC06F3F71058105910569F03B
:10C6500064F080E091E0A0E0B0E080937B039093F1
:10C660007C03A0937D03B0937E0380917B03909124
:10C670007C03880E991E80917D01282F332780919D
:10C68000DF08992787FD9095289FF001299FF00DDD
:10C69000389FF00D11249F01F7FF02C021583F4F32
:10C6A000220F232F221F330BFFEF21383F071CF4EB
:10C6B00020E83FEF06C02F3F310519F014F020E0CD
:10C6C00031E0820E931EC401AA2797FDA095BA2FD0
:10C6D000E090D002F090D1029701442737FD4095B9
:10C6E000542FBC01CD010E94939097FF04C061506C
:10C6F0007E4F8F4F9F4F29E095958795779567954A
:10C700002A95D1F7C61AD70A8091E0029091E102EA
:10C71000892B09F060C01E141F040CF05CC0980146
:10C7200017FF03C0309521953F4F2D33310540F45D
:10C730008091FE029091FF028C159D0574F526C034
:10C740002C53304085E0369527958A95E1F72031C6
:10C75000310510F02FE030E04091FE025091FF02D1
:10C7600010161106E4F480E190E0821B930B489FC1
:10C770009001499F300D589F300D1124B4E036953B
:10C780002795BA95E1F72C153D0520F58091860196
:10C7900090918701C816D906F4F06C011CC0205F87
:10C7A0003F4F8091860190918701829F8001839FF6
:10C7B000100D929F100D11249801A4E03695279535
:10C7C000AA95E1F74C155D0514F06A0104C0C21684
:10C7D000D30608F06901C601AA2797FDA095BA2FD4
:10C7E000FDE0880F991FAA1FBB1FFA95D1F795018D
:10C7F000442737FD4095542FBC01CD010E9407917D
:10C8000020937F03309380034093810350938203EE
:10C81000C0907F03D09080038091AC039091AD03D2
:10C820009C01220F331F280F391F2C0D3D1D37FF90
:10C8300002C02D5F3F4FA9015595479555954795E6
:10C840005093AD034093AC0380916D06282F33279E
:10C85000220F331F220F331F241735076CF48091EA
:10C860005308282F3327220F331F220F331F205541
:10C8700030404217530724F03093AD032093AC03AC
:10C8800080912F0880FF14C08091AC039091AD037C
:10C8900029813A818217930724F03093AD032093C6
:10C8A000AC034091AC035091AD035A83498361C0FE
:10C8B00029813A812E193F0937FF02C02D5F3F4F72
:10C8C00035952795359527956091AC037091AD030B
:10C8D000620F731F7A8369834CC080917506882329
:10C8E00001F56091D0027091D10277FF02C06D5FB7
:10C8F0007F4F759567957595679540912501509186
:10C90000260180910001282F3327649FC001659F75
:10C91000900D749F900D1124B9010E94D290CB010B
:10C9200001C09927909389018093880180918801A3
:10C9300090918901873491051CF486E490E005C04C
:10C940008639910534F086E990E0909389018093CF
:10C95000880189819A819093AD038093AC03809183
:10C96000B402806C8093B4028091B3028D7F809377
:10C97000B3028091B40299279C012270307081FF2C
:10C980002BC18091AE039091AF03A091B003B09101
:10C99000B1030097A105B10521F08091EA02813031
:10C9A000B1F4E981FA81CF01AA2797FDA095BA2FAA
:10C9B0001EE0880F991FAA1FBB1F1A95D1F78093FD
:10C9C000AE039093AF03A093B003B093B1038091F3
:10C9D000EA02813019F482E08093EA02E980FA8069
:10C9E000C701AA2797FDA095BA2F9501442737FDC7
:10C9F0004095542FBC01CD010E949390DC01CB01E6
:10CA000080937F0390938003A0938103B09382036C
:10CA1000B7FF04C08150904EAF4FBF4F7C018D01D6
:10CA2000ADE015950795F794E794AA95D1F7E092B4
:10CA30007F03F0928003009381031093820360913F
:10CA4000B5027091B6022FE0603A720750F58091FE
:10CA5000AE039091AF03A091B003B091B1039C01DC
:10CA6000AD01FAE05695479537952795FA95D1F798
:10CA7000821B930BA40BB50BA8019701E4E0220FD6
:10CA8000331F441F551FEA95D1F7820F931FA41F30
:10CA9000B51F8093AE039093AF03A093B003B09300
:10CAA000B10360547F4118F58091AE039091AF03BC
:10CAB000A091B003B091B1039C01AD016CE056951B
:10CAC0004795379527956A95D1F7821B930BA40B51
:10CAD000B50BA8019701F2E0220F331F441F551F29
:10CAE000FA95D1F7820F931FA41FB51F38C080910C
:10CAF000FE019091FF018091FE019091FF0197FF4F
:10CB000003C0909581959F4F8436910584F580915F
:10CB1000E6029091E7022091E2023091E302821B4B
:10CB2000930B81509F4F8F5F914008F58091AE032A
:10CB30009091AF03A091B003B091B1039C01AD01FE
:10CB4000EEE05695479537952795EA95D1F7821BE4
:10CB5000930BA40BB50B8E0D9F1DA01FB11F8093CF
:10CB6000AE039093AF03A093B003B093B103809151
:10CB7000AE039091AF03A091B003B091B1037EE0FA
:10CB8000B695A795979587957A95D1F79093D10209
:10CB90008093D00240917306442399F055279C015D
:10CBA000BA010E94D290C901861B970B9093FF0295
:10CBB0008093FE02260F371F309387012093860152
:10CBC0001FC01092FF021092FE028FEF93E090932D
:10CBD00087018093860114C01092EA021092AE037E
:10CBE0001092AF031092B0031092B1033093D102B0
:10CBF0002093D00205C08091B402806C8093B4026F
:10CC00008091C20381FF37C089819A8197FD039685
:10CC100095958795959587952091B1023091B202AF
:10CC20002817390760F48091D0029091D102892BA6
:10CC300031F0220F331F220F331F3A832983809153
:10CC4000E6029091E702A091E802B091E902809398
:10CC5000E2029093E302A093E402B093E50288E934
:10CC60009AE39093EE018093ED0180E09EE0909333
:10CC700008018093070120911808822F9927880FB7
:10CC8000991F880F991F889669817A81861797075F
:10CC900014F09A838983709153087D8B872F99278D
:10CCA000880F991F880F991F80559040A981BA81DC
:10CCB0008A179B0714F49A8389838091350288230D
:10CCC00041F48091E6088F3F21F48091C6038823C8
:10CCD000E9F08091B5029091B6020297C097B0F446
:10CCE000E981FA811E161F068CF481E090E0909392
:10CCF000B6028093B502E22EFF24EE0CFF1CEE0C70
:10CD0000FF1C8701085D1F4F1A83098329813A811F
:10CD10003093C7052093C6058091770390917803DF
:10CD2000A0917903B0917A0312E0880F991FAA1F8E
:10CD3000BB1F1A95D1F70091540810915508081B94
:10CD4000190B213A31058CF0C90137FD01969595F3
:10CD50008795801791070CF48C01909581959F4FD2
:10CD6000081719076CF48C010BC00135110514F07C
:10CD700000E510E03FEF003B130714F400EB1FEF5A
:10CD80004D89242F3327220F331F220F331FC90150
:10CD900069817A81861B970B801791070CF48C01AF
:10CDA00089819A81821B930B081719070CF48C0157
:10CDB00080911308909114086091FC027091FD021B
:10CDC000861B970B9093220880932108D0903108FE
:10CDD00020910E0330910F034091100350911103E5
:10CDE000DD2041F0661A770AC301AA2797FDA095B6
:10CDF000BA2F04C0AA2797FDA095BA2F280F391F74
:10CE00004A1F5B1F20930E0330930F0340931003C0
:10CE10005093110380910E0390910F03A091100382
:10CE2000B091110381509A4FA040B04064F080E06F
:10CE30009AEFA0E0B0E080930E0390930F03A093CD
:10CE40001003B093110380910E0390910F03A091F2
:10CE50001003B091110380509640AF4FBF4F64F460
:10CE600080E096E0AFEFBFEF80930E0390930F0347
:10CE7000A0931003B0931103C09082062091210863
:10CE80003091220878E0E72EEC1498F08C2D992749
:10CE9000829FA001839F500D929F500D1124CA01C3
:10CEA00057FD07967C0163E0F594E7946A95E1F7F6
:10CEB00012C08C2D86959927829FB001839F700D9B
:10CEC000929F700D1124CB0177FD03967C01F594A0
:10CED000E794F594E794A0908301B09084019501C4
:10CEE000442737FD4095542F80910E0390910F03F6
:10CEF000A0911003B0911103BC01CD010E940791D4
:10CF0000E20EF31E90906F01692D772788279927ED
:10CF1000980117FF04C022273327201B310B37FF4E
:10CF200002C02F5F3F4F35952795A981BA812A0FFF
:10CF30003B1F442737FD4095542F0E94939097FF45
:10CF400004C0615C7F4F8F4F9F4F26E0959587957A
:10CF5000779567952A95D1F79B016E157F050CF49F
:10CF60007B01309521953F4FE216F3060CF47901D1
:10CF700080910308909104086091FA027091FB027D
:10CF8000861B970B909302088093010820910A0357
:10CF900030910B0340910C0350910D03DD2041F0C3
:10CFA000461A570AC201AA2797FDA095BA2F04C0B6
:10CFB000AA2797FDA095BA2F280F391F4A1F5B1F7C
:10CFC00020930A0330930B0340930C0350930D03FB
:10CFD00080910A0390910B03A0910C03B0910D0373
:10CFE00081509A4FA040B04064F080E09AEFA0E0FA
:10CFF000B0E080930A0390930B03A0930C03B093CB
:10D000000D0380910A0390910B03A0910C03B09142
:10D010000D0380509640AF4FBF4F64F480E096E020
:10D02000AFEFBFEF80930A0390930B03A0930C0321
:10D03000B0930D03209101083091020848E04C158F
:10D0400098F08C2D9927829FB001839F700D929F3D
:10D05000700D1124CB0177FD07966C01B3E0D594D8
:10D06000C794BA95E1F712C0C6948C2D9927829F78
:10D07000D001839FB00D929FB00D1124CD01B7FD5B
:10D0800003966C01D594C794D594C7949501442711
:10D0900037FD4095542F80910A0390910B03A09186
:10D0A0000C03B0910D03BC01CD010E940791C20E8B
:10D0B000D31E692D772788279927980117FF04C069
:10D0C00022273327201B310B37FF02C02F5F3F4F32
:10D0D00035952795E981FA812E0F3F1F442737FDAB
:10D0E0004095542F0E94939097FF04C0615C7F4F3E
:10D0F0008F4F9F4FE6E09595879577956795EA95D1
:10D10000D1F79B016C157D050CF46B0130952195D1
:10D110003F4FC216D3060CF4690180911808282EDF
:10D1200033245090C30661E3862E67E0962E58EEB6
:10D13000A52E56E0B52E4BE0442E32E3632E38E0A8
:10D14000732ED5012C9112160CF029C1203429F42C
:10D15000E981FA81FF8BEE8B1FC049815A81CA0198
:10D16000AA2797FDA095BA2F332727FD3095432F87
:10D17000532FBC01CD010E94939097FF04C0615CC6
:10D180007F4F8F4F9F4F26E09595879577956795B1
:10D190002A95D1F77F8B6E8BF5012181203439F4EC
:10D1A0002E893F892E0D3F1D3F8B2E8B2AC0203CA0
:10D1B00039F44E895F894E195F095F8B4E8B21C010
:10D1C000C701AA2797FDA095BA2F332727FD3095D1
:10D1D000432F532FBC01CD010E94939097FF04C0B1
:10D1E000615C7F4F8F4F9F4FB6E095958795779500
:10D1F0006795BA95D1F7AE89BF89A60FB71FBF8BC8
:10D20000AE8BF5012281203439F42E893F892C0D13
:10D210003D1D3F8B2E8B2AC0203C39F44E895F89FF
:10D220004C195D095F8B4E8B21C0C601AA2797FD63
:10D23000A095BA2F332727FD3095432F532FBC01DC
:10D24000CD010E94939097FF04C0615C7F4F8F4F88
:10D250009F4FA6E09595879577956795AA95D1F705
:10D26000AE89BF89A60FB71FBF8BAE8BF501238197
:10D27000203439F42E893F89200F311F3F8B2E8BAC
:10D280002AC0203C39F44E895F89401B510B5F8BCB
:10D290004E8B21C0C801AA2797FDA095BA2F33272E
:10D2A00027FD3095432F532FBC01CD010E94939051
:10D2B00097FF04C0615C7F4F8F4F9F4FF6E09595BD
:10D2C000879577956795FA95D1F7AE89BF89A60FAF
:10D2D000B71FBF8BAE8BF301808191812E893F896F
:10D2E0008217930764F4B901680F791F77FF02C0B2
:10D2F0006F5F7F4F759567957F8B6E8B1DC0552037
:10D3000049F44E895F89440F551F481B590B5F8BA9
:10D310004E8B12C051E0551578F4252D33276E89B8
:10D320007F89861B970BB9010E94D290AE89BF8975
:10D33000A60FB71FBF8BAE8BC101880F991F880F37
:10D34000991FEE89FF898E179F0764F4FD898F2F3F
:10D350009927880F991F880F991F2E893F892817B1
:10D36000390714F09F8B8E8B8E899F8997FD0396CA
:10D370009595879595958795F4018183880F991FD9
:10D38000880F991F2E893F89281B390BC901880FE7
:10D390008283EE89FF89D301ED93FC9303C0F401EE
:10D3A000118212824A9422E030E0620E731E44E041
:10D3B00050E0A40EB51E68E070E0860E971E47FE92
:10D3C000C0CEE2E1C95E0C943E9184B1806A84B91A
:10D3D0003D9A82E58CBD1DBC459A81E0809365082D
:10D3E0008AEA8093760883E8809377088AE08093BE
:10D3F000780810927A081092790810927C0810929E
:10D400007B081092DE0810929A0808953091650802
:10D41000332309F085C00DB407FE82C084E08093F9
:10D42000EC01459A2EB58091C90399278130910569
:10D4300089F0823091051CF4892B21F03EC00297BF
:10D44000B9F03BC0309399082093CA032138A9F55D
:10D4500081E008C0253549F48091CA03820F80938A
:10D46000CA0382E08093C90328C03093C90325C052
:10D4700080919908E82FFF27E554F74F20838F5FAD
:10D48000809399089091CA038032A0F0291769F41B
:10D4900080E2ABEBB8E0EBE9F8E00D9001928A9501
:10D4A000E1F781E080939A0802C030939A081092C5
:10D4B000C90303C0920F9093CA03209175082232CA
:10D4C00008F028C04598000000000000000000009F
:10D4D000000000000000000000000000000000004C
:10D4E000000000000000000000000000000000003C
:10D4F000000000000000E0916E08F0916F08E20F5C
:10D50000F11D80818EBD809197089081890F809355
:10D51000970803C081E0809365082F5F209375080A
:10D520000895EF92FF920F931F9380917B069927A6
:10D53000880F991F880F991F7C010027F7FC009521
:10D54000102F8091460390914703A0914803B0911A
:10D550004903BC01CD01A80197010E9407913093B6
:10D560007A082093790880913E0390913F03A0911F
:10D570004003B0914103BC01CD01A80197010E9475
:10D58000079130937C0820937B0820915B083091B1
:10D590005C0840915D0850915E08DA01C90163E0C2
:10D5A000880F991FAA1FBB1F6A95D1F7820F931F7F
:10D5B000A41FB51F820F931FA41FB51F20914A01FE
:10D5C00030914B0140914C0150914D01BC01CD0176
:10D5D0000E9407913093820820938108809157031D
:10D5E0009091580320910B0230910C02821B930BF7
:10D5F0009093880880938708E0914D03F0914E0343
:10D600008091280890912908BF010E94D2909B0127
:10D61000220F331F220F331F260F371F260F371FEE
:10D6200037FF02C02D5F3F4F3595279535952795DC
:10D6300030937E0820937D08809157089091580878
:10D64000BF010E94D2909B01220F331F220F331F74
:10D65000260F371F260F371F37FF02C02D5F3F4FA2
:10D6600035952795359527953093800820937F0829
:10D6700010924E0310924D03109229081092280820
:10D6800010925808109257088091780899278D3089
:10D69000910509F48CC08E3091055CF48B309105B6
:10D6A00009F4B4C08C3091050CF035C10A9761F0D3
:10D6B000E7C18F30910509F4B3C18F3091050CF4A7
:10D6C00080C14097A9F1DCC18091C90280938B0889
:10D6D0008091C80280938C088091C70280938D0846
:10D6E0008091C60280938E088091C50280938F0836
:10D6F0008091C402809390088091C3028093910826
:10D700008091C202809392088091B4028093930822
:10D710008091B402837F8093B4020E94823280930E
:10D7200094088091C406809395088091B302A6C1A5
:10D730008091E0089091E10890938C0880938B0889
:10D740008091E4089091E50890938E0880938D086D
:10D75000809125019091260180938F08809100018E
:10D760008093900880914901809391089091CB0318
:10D7700090939208E92FFF27A3E0EE0FFF1FAA95D1
:10D78000E1F7EF5CF84F8681809393088381809363
:10D790009408878180939508858180939608892FC6
:10D7A0008F5F6CE00E94B2909093CB0369C180912F
:10D7B000AF0680938B088091B00680938C0880918F
:10D7C000B10680938D088091B20680938E08809177
:10D7D000B30680938F088091B7068093900880915C
:10D7E000B806809391088091B90680939208809141
:10D7F000BC06809393088091BA0680939408809128
:10D80000BB06809395088091BD0638C1F89480913D
:10D810006206E82FFF27EE0FFF1FEE56F84F01902C
:10D82000F081E02DE038F1051CF0EFE7F0E006C0F4
:10D830002FEFE138F20714F4E1E8FFEFE0938B08F3
:10D8400080916306E82FFF27EE0FFF1FEE56F84F7B
:10D850000190F081E02DE038F1051CF0EFE7F0E0F9
:10D8600006C06FEFE138F60714F4E1E8FFEFE0934C
:10D870008C0880916106E82FFF27EE0FFF1FEE5600
:10D88000F84F0190F081E02DE038F1051CF0EFE752
:10D89000F0E006C08FEFE138F80714F4E1E8FFEF9D
:10D8A000E0938D0880916006E82FFF27EE0FFF1FA1
:10D8B000EE56F84F0190F081E02DE038F1051CF0B4
:10D8C000EFE7F0E006C02FEFE138F20714F4E1E8EB
:10D8D000FFEF7894E0938E088091ED0280938F089B
:10D8E0008091EE02809390088091EF0280939108DE
:10D8F0008091F002809392088091F10280939308C6
:10D900008091F202809394088091F30280939508AD
:10D910008091F402B3C080914704863018F01092D1
:10D92000470485E080938B088091BE0680938C0825
:10D930008091E6029091E702A091E802B091E9029D
:10D94000BC01CD0125E030E040E050E00E940791AD
:10D9500030938E0820938D088091E2029091E3022B
:10D96000A091E402B091E502BC01CD0125E030E0D8
:10D9700040E050E00E9407913093900820938F0878
:10D980008091B406809391088091B50680939208A7
:10D990008091B606809393088091EC02809394085E
:10D9A0008091920790919307809395088091C60586
:10D9B0009091C70597FD03969595879595958795C1
:10D9C0005DC010928B0888E580938C0885E0809379
:10D9D0008D088FE180938E088091010180938F08DC
:10D9E00080912C048093900880912D04809391085D
:10D9F00010922C04807180932D0480912E048093CA
:10DA0000920880914B088093930880912F0880930F
:10DA100094088091C006809395088091CD062EC011
:10DA20008091940680938B088091CB0680938C081C
:10DA30008091750180938D0880918D0680938E086A
:10DA400080918E0680938F0880918F068093900836
:10DA5000809174018093910880919106809392083F
:10DA60008091920680939308809193068093940806
:10DA70008091E608809395088091F0058093960840
:10DA800080919A08882309F455C18AEF8093A301F5
:10DA900081E08093950140919C0850919D08CA01B6
:10DAA00081509E4F8F5F9340B0F420919E0830913B
:10DAB0009F08C90181509E4F8F5F934060F4809111
:10DAC0006C0685FF08C05093B8034093B7033093AA
:10DAD000B6032093B5038091A2089091A30821E09A
:10DAE0008936920724F490939701809396012091B0
:10DAF000AC083091AD088091ED019091EE01821754
:10DB0000930740F48091B601882321F43093EE010D
:10DB10002093ED0180919B0899278936910509F49E
:10DB2000A5C08A36910544F48736910571F0883690
:10DB3000910509F462C006C18A36910509F4F3C063
:10DB40008B36910509F4E2C0FDC08091AE08809348
:10DB5000DB088091AF088093DD088091B008809346
:10DB6000DC088091B108809394018091B208809381
:10DB7000DF088091B3088093A4018091B40880935A
:10DB8000C8038091B5088093B4038091C1028823B3
:10DB9000F9F02091B6083091B70837FD19C03093DD
:10DBA00005032093040390919606992389F08FE052
:10DBB000989FC0011124281B390BC90188599E4F19
:10DBC00068E671E00E94D29090930503809304036D
:10DBD0002091BF033091C0038091B8089091B9089B
:10DBE000280F391F37FF02C02F5F3F4F359527950C
:10DBF0003093C0032093BF03A5C08091AE088093EB
:10DC000070088091AF08809371088091B00880936C
:10DC100072088091B108809373088091B208809354
:10DC200074088091B6059091B308892B8093B6054E
:10DC30009091B70593708091B4088C70982B909355
:10DC4000B7058091B5088093C6038091B60880938C
:10DC500099018091B7088093DE088091B80880937D
:10DC6000C2038091B9088093C1036CC08091AE0853
:10DC7000809366088091AF08809367088091B00810
:10DC8000809368088091B108809369088091B208F8
:10DC90009091B30890936B0880936A088091B408C0
:10DCA0009091B50890936D0880936C088091B608A8
:10DCB000992787FD90959093C5078093C40780911D
:10DCC000B7088093DB028091B8089091B9089C0155
:10DCD000442737FD4095542FDA01C90163E0880FCE
:10DCE000991FAA1FBB1F6A95D1F7820F931FA41F0C
:10DCF000B51F820F931FA41FB51F8093DC02909362
:10DD0000DD02A093DE02B093DF021CC08091AE085A
:10DD10008093C5038091AF088093C4038091B008BD
:10DD20008093C3030FC080918606863059F40E9409
:10DD3000BA7608C01092B8031092B7031092B603D7
:10DD40001092B5031F910F91FF90EF90089580916D
:10DD50006508882309F43BC0459886E798E09093CE
:10DD60006F0880936E089091C703E92FFF27E6564E
:10DD7000FE4F9F5F9093C70380818093780899300E
:10DD800010F01092C703109265080E94916A81E01A
:10DD900080937508000000000000000000000000F3
:10DDA0000000000000000000000000000000000073
:10DDB0000000000000000000000000000000000063
:10DDC0000000000080917608809397088EBD08952A
:10DDD00087B18C6087B9429843981092CD0380E850
:10DDE0008093A6011092CC038093A50108958091A1
:10DDF000D20381508093D2038F3F09F019C189E08B
:10DE00008093D2038091B402992780739070892BFC
:10DE100021F480912D0480FF1DC08091AD068823E0
:10DE200051F08091D503882319F484E08093CD03C9
:10DE300081E08093D5038091AE068823B9F080916C
:10DE4000D603882319F484E08093CC0381E0809387
:10DE5000D6030CC01092D5031092D6038091A90668
:10DE60008093D3038091AB068093D4038091D50334
:10DE7000882309F045C08091CA06282F332724FF44
:10DE800007C08091EB02882319F425FD52C053C0CE
:10DE90009091AA06983F48F080912A088D3D28F07D
:10DEA0008091D30388236CF00AC0983F78F080916A
:10DEB0002A08853059F48091D30387FF02C0429825
:10DEC00001C0429A81E08093A60136C08091CD03C3
:10DED00081508093CD038F3F79F580912A088695F4
:10DEE0008093CD038091A601813011F480E801C0B8
:10DEF00086958093A6018091A6019091D30317C0C7
:10DF00008091CD0381508093CD038F3FA9F489E0A8
:10DF10008093CD038091A601813011F480E801C087
:10DF200086958093A6018091A6019091AD068923E4
:10DF300011F0429A01C042988091D603882309F0DB
:10DF400043C09091CA0697FF07C08091EB028823D7
:10DF500019F496FD52C053C09091AC06983F48F01A
:10DF6000809152088D3D28F08091D40388236CF075
:10DF70000AC0983F78F080915208853059F480911A
:10DF8000D40387FF02C0439801C0439A81E0809385
:10DF9000A50136C08091CC0381508093CC038F3F84
:10DFA00079F58091520886958093CC038091A501E4
:10DFB000813011F480E801C086958093A50180919D
:10DFC000A5019091D40317C08091CC038150809318
:10DFD000CC038F3FA9F489E08093CC038091A50105
:10DFE000813011F480E801C086958093A50180916D
:10DFF000A5019091AE06892311F0439A01C0439880
:10E00000429B04C08091B302886003C08091B30238
:10E01000877F8093B302439B06C08091B3028061E7
:10E020008093B30208958091B3028F7E8093B302F0
:10E0300008954FB724E130E0F8948091C9008F77BC
:10E040008093C9008091C9008F7B8093C900809123
:10E05000C9008F7D8093C9005A9A52985B9A539A4F
:10E06000832F99278093CD002093CC008091C80006
:10E0700082608093C80080E18093C9008091CA00CB
:10E080008F778093CA008091CA008F7B8093CA00EB
:10E090008091CA008F7D8093CA008091CA008F7ED4
:10E0A0008093CA008091CA00877F8093CA008091C4
:10E0B000C9008B7F8093C9008091CA0084608093DF
:10E0C000CA008091CA0082608093CA008091C80013
:10E0D00087FF03C08091CE00F9CF8091C90080688E
:10E0E0008093C9004FBF0895EF92FF920F931F9343
:10E0F000CF93DF93482F00E010E08091A70181309B
:10E1000061F41092A70184E48093D7031092D9039D
:10E110001092D8031092DA0339C18091D703882373
:10E1200019F421E030E001C098019091D8039923BF
:10E1300071F4232B11F081E010C084E48093D703A5
:10E140009093D9039093D8039093DA0308C1913048
:10E1500069F4232B09F0F9C082E08093D803809101
:10E16000D9038F5F8093D90383E0F7C09230D1F455
:10E17000232B09F0EAC083E08093D7034093DA03AE
:10E180009091D903923039F41092DB0347FF03C01A
:10E1900081E08093DB0383E08093D8039F5F9093BB
:10E1A000D903DDC0933009F0D0C0232B09F0CDC0D6
:10E1B0009093D70382E08093D8038091D9038F5F37
:10E1C0008093D9032091DA03822F9927782F66272D
:10E1D000842F9927682B792B80918606813049F40A
:10E1E0007370CB018050924063E070E00E94D29047
:10E1F00017C0823061F47770CB018050944066E0A4
:10E2000070E00E94D2902695269526950BC07370DB
:10E2100068567140CB0177FD0196BC0175956795F5
:10E2200026952695022F11270F7010700F5F1F4F34
:10E230000D30110508F082C07801E00EF11EF701E3
:10E24000EE56F84F808191819B01281B390BC90143
:10E2500037FF03C0909581959F4F069704F5E09195
:10E26000C706EE2351F0FF27EE0FFF1FEE56F84FC3
:10E27000808191818436910594F48091EC02883CF0
:10E2800030F48091EC02865F8093EC0208C088EC49
:10E290008093EC0280916F008F7D80936F00F70177
:10E2A000EE56F84F808191819C01220F331F280F79
:10E2B000391F260F371F37FF02C02D5F3F4FE9017F
:10E2C000D595C795D595C795CB0101968C179D0718
:10E2D00014F4219706C061507040C617D7070CF49C
:10E2E00021968091EC02843BD0F0F701EE56F84F76
:10E2F00080819181FE01E81BF90BCF0163E070E0A2
:10E300000E94D290CB01880F991F860F971F26EC91
:10E3100037E0E20EF31EF7019183808307C026ECFD
:10E3200037E0E20EF31EF70111821082000F111F79
:10E330000E56184FF801D183C08311C00231110568
:10E3400070F081E08093A7010AC081E08093A7016B
:10E350001092D9031092DB0384E48093D703809159
:10E36000D903803198F08091DB03882331F48091C8
:10E37000A701882311F4809348011092D9031092C9
:10E38000DB031092D80384E48093D703E6E0CDB793
:10E39000DEB70C944A91CF93FC0197FF05C0CFEFF5
:10E3A000F095E195FF4F01C0C1E028E631E0CF01D3
:10E3B000B9010E94D290FC018B35910554F08B5528
:10E3C00090408A35910538F484EB90E08E1B9F0BCA
:10E3D000FC0141E00DC0CF01855B90408A3591057D
:10E3E00018F4E45BF04003C02E1B3F0BF9014FEF24
:10E3F000EE0FFF1FEB5CF64F259134918C2F992780
:10E4000087FD9095289FB001299F700D389F700D52
:10E410001124842F992787FD9095689FA001699FFB
:10E42000500D789F500D1124CA01CF9108952AE50F
:10E4300030E0281B390BC9010E94CB710895CF939E
:10E44000DF9380E00E94A2868091250190912601B1
:10E450006AE070E00E94D2909F938F938091250193
:10E46000909126016AE070E00E94D2907F936F93B2
:10E4700089E09AE09F938F93C5E9D6E8DF93CF9325
:10E48000E0911304F091140409952DB73EB7285F6D
:10E490003F4F2DBF8091A301882361F186E00E9448
:10E4A000A2868091990199279F938F9380916A0802
:10E4B00090916B086AE070E00E94BE907F936F932A
:10E4C0008FED90E09F938F938091080890910908B9
:10E4D0009F938F9382E19AE09F938F93DF93CF93E3
:10E4E000E0911304F091140409958DB79EB70C9632
:10E4F0008DBF12C086E00E94A28680E29AE09F93C0
:10E500008F93DF93CF93E0911304F0911404099556
:10E510000F900F900F900F908091C603882309F4FD
:10E5200058C08091DC039091DD030E947F198823FD
:10E5300091F08091A801882319F01092A80103C0DE
:10E5400081E08093A8018CED95E00E94761990936C
:10E55000DD038093DC038091A8018823E1F080E053
:10E560000E94A2861F921F929091C60381E1989FFC
:10E57000C00111248D5F944F9F938F93DF93CF93AE
:10E58000E0911304F091140409952DB73EB72A5F6A
:10E590003F4F2DBF1EC086E00E94A2868091C60319
:10E5A00099279F938F9387E29AE09F938F93DF93AE
:10E5B000CF93E0911304F091140409958DB79EB7A1
:10E5C00006968DBF8091EB02882319F08FE480932B
:10E5D000AE0180E10E94A2868091B0019091B101CC
:10E5E0006CE370E00E94BE909F938F938091B00186
:10E5F0009091B1016CE370E00E94BE907F936F93A5
:10E600008091E4089091E5089F938F9383E39AE0CB
:10E610009F938F93C5E9D6E8DF93CF93E0911304DE
:10E62000F0911404099580914B082DB73EB7265FF1
:10E630003F4F2DBF80FF29C08AE10E94A2868091B2
:10E64000490199279F938F938091E6029091E70269
:10E65000A091E802B091E902BC01CD0124E630E0CE
:10E6600040E050E00E9407913F932F9380E49AE0AE
:10E670009F938F93DF93CF93E0911304F091140451
:10E6800009958DB79EB708968DBFDF91CF910895FC
:10E69000CF93DF9380E00E94A28680915007992754
:10E6A00087FD90959F938F9380914807992787FDC9
:10E6B00090959F938F9380914007992787FD909520
:10E6C0009F938F9380913807992787FD90959F930B
:10E6D0008F9387E49AE09F938F93C5E9D6E8DF9301
:10E6E000CF93E0911304F0911404099580E10E9406
:10E6F000A2862DB73EB7245F3F4F2DBF8091700794
:10E70000992787FD90959F938F938091680799270C
:10E7100087FD90959F938F9380916007992787FD40
:10E7200090959F938F9380915807992787FD909597
:10E730009F938F9387E59AE09F938F93DF93CF9377
:10E74000E0911304F0911404099580915E062DB7B1
:10E750003EB7245F3F4F2DBF853098F480E10E9483
:10E76000A28687E69AE09F938F93DF93CF93E09101
:10E770001304F091140409950F900F900F900F90CF
:10E7800018C08730B0F488E10E94A2868FED90E037
:10E790009F938F9388E79AE09F938F93DF93CF9314
:10E7A000E0911304F091140409958DB79EB7069675
:10E7B0008DBFDF91CF9108950F931F9380E00E944A
:10E7C000A2862AE030E08091E0089091E108B9014A
:10E7D0000E94BE909F938F938091E0089091E108F2
:10E7E000B9010E94BE907F936F9380912501909113
:10E7F0002601B9010E94D2909F938F9380912501A9
:10E8000090912601B9010E94D2907F936F9381E885
:10E810009AE09F938F9305E916E81F930F93E09179
:10E820001304F0911404099580E10E94A2868DB72B
:10E830009EB70C968DBF8091E4089091E5089F9358
:10E840008F938091E2089091E3089F938F9383E9DF
:10E850009AE09F938F931F930F93E0911304F0918D
:10E86000140409958DB79EB708968DBF1F910F911F
:10E870000895EF92FF920F931F9380E00E94A2866B
:10E880008FEDE82EF12CFF92EF92809196019091FE
:10E8900097019F938F938091C50399279F938F939F
:10E8A0008FE99AE09F938F9305E916E81F930F93E2
:10E8B000E0911304F0911404099580E10E94A2866E
:10E8C0008DB79EB70A968DBF8091C30399279F93FA
:10E8D0008F93FF92EF928091C40399279F938F9318
:10E8E00082EB9AE09F938F931F930F93E091130411
:10E8F000F091140409958DB79EB70A968DBF1F91AC
:10E900000F91FF90EF9008950F931F93CF93DF9394
:10E910008091A301C5E9D6E8882309F47DC080E091
:10E920000E94A2868091670899279F938F93809178
:10E93000690899279F938F9385EC9AE09F938F9313
:10E940008E01DF93CF93E0911304F09114040995A5
:10E950008DB79EB708968DBF80916808833031F4DB
:10E960008CE00E94A28684ED9AE005C08CE00E94B3
:10E97000A28689ED9AE09F938F93DF93CF93E091E6
:10E980001304F091140409950F900F900F900F90BD
:10E990008091660881FF12C08CE00E94A2868EEDF5
:10E9A0009AE09F938F931F930F93E0911304F0913C
:10E9B000140409950F900F900F900F9080E10E9422
:10E9C000A2868091990199279F938F938FED90E074
:10E9D0009F938F9380916C0890916D089F938F9374
:10E9E00080916A0890916B086AE070E00E94BE9086
:10E9F0007F936F9383EE9AE09F938F9385E996E8D8
:10EA00009F938F93E0911304F091140409958DB7AF
:10EA10009EB70C968DBF12C082E00E94A28686EF40
:10EA20009AE09F938F93DF93CF93E0911304F0913B
:10EA3000140409950F900F900F900F90DF91CF91D4
:10EA40001F910F910895CF93C82F2091DE0320933B
:10EA5000DF0399278F329105E1F0803391051CF493
:10EA60004F9779F027C08F349105D9F08F389105F1
:10EA700009F586E0289FF0011124E551F64F8491B5
:10EA800017C086E0289FF0011124E451F64F8491CD
:10EA90000FC086E0289FF0011124E351F64F8491C6
:10EAA00007C086E0289FF0011124E251F64F8491BF
:10EAB0008093DE039091DE038091DF039813C0E022
:10EAC0000E94A8869091DE0386E0989FF0011124B1
:10EAD000E151F64F259134918C2FF901099580E091
:10EAE00090E0CF9108951092E1081092E008109202
:10EAF000E5081092E4081092E3081092E2081092E0
:10EB0000E6088AE090E00E9476199093E1038093F2
:10EB1000E0030895CF93DF938091E0039091E103A8
:10EB20000E947F19882309F4AFC08091E00390917F
:10EB3000E1030A969093E1038093E003E0E0F0E0C4
:10EB40009F0190E05FEFA1E3B7E04BE0ED018B8127
:10EB500087FF0BC09F5F8D81E80FF11D8981280F12
:10EB6000311D8E81851708F4582F4150189647FFA4
:10EB7000EDCF5093E608232B41F52091E603309129
:10EB8000E7034091E8035091E903BB27A52F942F99
:10EB9000832F9093E5038093E403AA27BB27281BC8
:10EBA000390B4A0B5B0BCF01AA27BB27280F391F54
:10EBB0004A1F5B1F2093E6033093E7034093E8036B
:10EBC0005093E903E5E0F0E013C02091E4033091B5
:10EBD000E5032E173F0718F4E21BF30B02C0E0E039
:10EBE000F0E0892F9927880F991FE80FF91F3596B4
:10EBF000F093E108E093E008EF3FF10578F48091AD
:10EC00002501909126018E9F90018F9F300D9E9F30
:10EC1000300D1124C90164E670E013C0CF01969550
:10EC20008795969587952091250130912601289FFB
:10EC3000A001299F500D389F500D1124CA0169E190
:10EC400070E00E94BE907093E3086093E208209108
:10EC5000E2033091E3032E0F3F1F3093E303209331
:10EC6000E2035EE02131350778F08091E40890916D
:10EC7000E50801969093E5088093E40820513E4012
:10EC80003093E3032093E203DF91CF910895309115
:10EC9000EF03E32FFF2783E0EE0FFF1F8A95E1F7D5
:10ECA000EF5CF84F2781422F552747FD5095809103
:10ECB000F0039927841795072CF42093F0033093E1
:10ECC000F2030AC0222341F08091F10399274817EB
:10ECD000590714F42093F103832F8F5F8093EF0380
:10ECE0008D30D0F01092EF038091F1038F3F19F037
:10ECF0008093EB0302C01092EB038091F0038093AA
:10ED0000EC038091F2038093EA038FEF8093F10389
:10ED10001092F0031092F203089595E1899F802DDF
:10ED200011240E94F18A81E09DE09F938F9383ECF0
:10ED30009AE89F938F93E0911304F091140409953E
:10ED40000F900F900F900F9008958091B40285FF5F
:10ED500003C080E190E008958091EB02882339F0B0
:10ED60008091C603882319F085E090E0089580E043
:10ED700090E0089540E050E030E08091B908992794
:10ED80008A38910591F08B38910524F489389105E2
:10ED900041F016C08D38910581F08E38910549F00B
:10EDA0000FC04FE259E031E10BC04CEE59E03DE1BC
:10EDB00007C047EE58E036E203C04DE059E032E2CA
:10EDC0009091AE0820E08091AF08281770F4931757
:10EDD00060F4DA01A90FB11DE22FFF27E556F74FC6
:10EDE00085898C939F5F2F5FEECF089520E335E7F1
:10EDF000809149018B3211F08D32F9F480917106C6
:10EE0000282F33278091E0029091E102829FA00198
:10EE1000839F500D929F500D1124CA0163E070E052
:10EE20000E94D290CB019B01205D3A48C196C197C8
:10EE300008F03FC02EEF34E73CC0803229F58091C6
:10EE4000B40281FF36C02091ED033091EE03205DC6
:10EE50003A4855E72133350748F085E72439380724
:10EE600018F420E335E702C02456304045E720334C
:10EE70003407F8F454E72D3C350718F020E335E764
:10EE800018C02C593F4F15C08E3549F49091DB02C4
:10EE90008AE0989F90011124205D3A480AC0863785
:10EEA00041F49091DB028AE0989FC0011124281B55
:10EEB000390BC9010895EF92FF920F931F93992781
:10EEC0008A38910509F45DC08B38910524F489389E
:10EED000910551F0D2C18D38910509F416C18E38D3
:10EEE000910509F483C0C9C18091E6029091E702BF
:10EEF000A091E802B091E902BC01CD0124E630E026
:10EF000040E050E00E940791DA01C9018C509E4F09
:10EF100090933309809332090E94F67690933909D1
:10EF20008093380990933B0980933A0990933D0967
:10EF300080933C0920913209309133098091360940
:10EF4000909137092817390724F430933709209313
:10EF5000360980913409909135098217930724F47A
:10EF600030933509209334090E94A57680933109A6
:10EF70008FE299E0909301048093000481E190E096
:10EF80007EC18091E6029091E702A091E802B091E3
:10EF9000E902BC01CD0124E630E040E050E00E94EF
:10EFA0000791DA01C9018C509E4F9093FF0980931D
:10EFB000FE090E94F6769093010A8093000A88E782
:10EFC00090E09093030A8093020A1092050A10922F
:10EFD000040A0E94A5768093EE098CEE99E0909346
:10EFE0000104809300048DE190E049C10E944776BE
:10EFF0008091E6029091E702A091E802B091E902C7
:10F00000BC01CD0124E630E040E050E00E940791D1
:10F01000DA01C9018C509E4F9093FF088093FE083F
:10F0200080912501909126019093F9088093F8082A
:10F0300080912501909126019093FB088093FA0816
:10F04000809108089091090897FD019695958795FC
:10F050008093EA088093F10820916C0830916D0844
:10F0600037FF02C02F5F3F4F359527952093EF085C
:10F0700080916A0890916B0864E170E00E94BE90F4
:10F080006093F0082093F6086093F7080E94F676E4
:10F09000909307098093060988E790E09093090907
:10F0A000809308098091250190912601909303098E
:10F0B000809302098091EB038C5E8093FC08809121
:10F0C000EC038C5E8093FD088091E4089091E50844
:10F0D0006AE070E00E94BE90709305096093040995
:10F0E0000E94A5768093E9088091E0089091E1085C
:10F0F000909301098093000987EE98E090930104B2
:10F100008093000486E290E0BAC00E944776809126
:10F110006A0890916B0864E670E00E94BE9070935C
:10F12000200960931F09809108089091090897FDB4
:10F130000196959587958093100980916C08909120
:10F140006D0897FD01969595879580931509809197
:10F150000001482F55279A012B5F3F4F80912501D1
:10F16000909126012817390784F480912501909108
:10F170002601841B950B9C01220F331F280F391F7A
:10F18000822F825180931C0902C010921C09E090CA
:10F19000E602F090E7020091E8021091E902C8014E
:10F1A000B70124E630E040E050E00E940791309340
:10F1B0001E0920931D0937FF04C010921E091092EA
:10F1C0001D09C801B70124E630E040E050E00E948C
:10F1D0000791DA01C9018C509E4F909322098093C8
:10F1E0002109809125019091260190931709809320
:10F1F0001609809125019091260190931909809319
:10F2000018090E94F676909324098093230988E7D1
:10F2100080932509809125019091260190932909D9
:10F22000809328098091EB038C5E80931A0980916A
:10F23000EC038C5E80931B098091E4089091E508B3
:10F240006AE070E00E94BE9070932B0960932A09D7
:10F250000E94A57680930F098091E0089091E108C3
:10F2600090932709809326098DE099E090930104FB
:10F270008093000482E290E002C080E090E01F9161
:10F280000F91FF90EF900895EF92FF920F931F93CD
:10F29000CF93DF938091ED039091EE039C0103E007
:10F2A000220F331F0A95E1F7281B390B8091FE01CD
:10F2B0009091FF01280F391F37FF02C0295F3F4F90
:10F2C00013E0359527951A95E1F73093EE032093D7
:10F2D000ED039091F403992309F011C38091F30396
:10F2E000282F3327442755278F5F8093F303F90195
:10F2F0002131310508F000C3E058FF4F0C945991BB
:10F300008091B40285FF2AC080E00E94F18A80913A
:10F310002501909126016AE070E00E94D2909F93AF
:10F320008F9380912501909126016AE070E00E9400
:10F33000D2907F936F9387E19DE09F938F9384EEAC
:10F340009AE89F938F93E0911304F0911404099528
:10F350002DB73EB7285F3F4F2DBF28C080E00E94E9
:10F36000F18A80912501909126016AE070E00E9467
:10F37000D2909F938F9380912501909126016AE00E
:10F3800070E00E94D2907F936F9384E29DE09F9300
:10F390008F9383EC9AE89F938F93E0911304F091FD
:10F3A000140409958DB79EB708968DBF80914B08C0
:10F3B00080FF39C0809103038823E9F08AE00E942E
:10F3C000F18A8091490199279F938F938091E6025A
:10F3D0009091E702A091E802B091E902BC01CD0151
:10F3E00024E630E040E050E00E9407913F932F93E5
:10F3F00081E39DE084C68AE00E94F18A8091E60262
:10F400009091E702A091E802B091E902BC01CD0120
:10F4100024E630E040E050E00E9407913F932F93B4
:10F420008DE39DE098C78AE00E94F18A88E49DE020
:10F4300017C68091B40285FF2AC085E10E94F18A37
:10F440008091B0019091B1016CE370E00E94BE9098
:10F450009F938F938091B0019091B1016CE370E024
:10F460000E94BE907F936F9382E59DE09F938F9360
:10F4700084EE9AE89F938F93E0911304F091140423
:10F4800009952DB73EB7285F3F4F2DBF28C085E1B6
:10F490000E94F18A8091B0019091B1016CE370E01B
:10F4A0000E94BE909F938F938091B0019091B10183
:10F4B0006CE370E00E94BE907F936F938FE59DE0B8
:10F4C0009F938F9383EC9AE89F938F93E09113041B
:10F4D000F091140409958DB79EB708968DBF8FE102
:10F4E0000E94F18A80E690E09F938F9380910808B4
:10F4F000909109089F938F938CE69DE09F938F9343
:10F50000C3ECDAE8DF93CF93E0911304F091140495
:10F5100009958091B3022DB73EB7285F3F4F2DBFAD
:10F5200080FF06C089E20E94F18A87E79DE069C3F7
:10F5300089E20E94F18A89E79DE0A9C68091B40220
:10F5400085FF1BC08AE20E94F18A8091E4089091B5
:10F55000E5089F938F938BE79DE09F938F9384EEB5
:10F560009AE89F938F93E0911304F0911404099506
:10F570008DB79EB706968DBF1BC08AE20E94F18AA6
:10F580008091E4089091E5089F938F9383E89DE034
:10F590009F938F9383EC9AE89F938F93E09113044A
:10F5A000F091140409952DB73EB72A5F3F4F2DBF48
:10F5B00086E30E94F18A8091E0089091E1086AE078
:10F5C00070E00E94BE909F938F938091E00890918D
:10F5D000E1086AE070E00E94BE907F936F938BE831
:10F5E0009DE09F938F9383EC9AE89F938F93E09194
:10F5F0001304F091140409958DB79EB70896B9C607
:10F6000089E00E94F18A87E99DE09F938F9303EC44
:10F610001AE81F930F93E0911304F09114040995D5
:10F620008EE10E94F18A0F900F900F900F9089E960
:10F630009DE09F938F931F930F93E0911304F0919C
:10F640001404099583E30E94F18A0F900F900F90A4
:10F650000F908BE99DE09F938F931F930F93E09101
:10F660001304F091140409958FE30E94F18A0F901E
:10F670000F900F900F908DE99DE09F938F931F93B4
:10F680000F93E0911304F091140409958EE70E9402
:10F69000F18A0F900F900F900F9083EB9DE09F9356
:10F6A0008F931F930F938AC78091A301882309F436
:10F6B00062C08DE50E94F18A89EC9DE09F938F9353
:10F6C000C3ECDAE8DF93CF93E0911304F0911404D4
:10F6D000099584E50E94F18A0F900F900F900F908A
:10F6E0008091670899279F938F938BEC9DE09F9360
:10F6F0008F93DF93CF93E0911304F0911404099555
:10F700008EE50E94F18A2DB73EB72A5F3F4F2DBF8D
:10F7100080916A0890916B086AE070E00E94BE9048
:10F720007F936F9384ED9DE09F938F93DF93CF93AF
:10F73000E0911304F091140409958DB79EB70696D5
:10F740008DBF80916808833081F48091660881FFC5
:10F7500006C08BE50E94F18A8EED9DE098C58BE591
:10F760000E94F18A81EE9DE092C58BE50E94F18AAC
:10F7700084EE9DE01DC784E0CDC38091A301882362
:10F7800009F47AC08091F603C3ECEC2ECAE8FC2E93
:10F79000882309F44BC089E60E94F18A8091C50351
:10F7A00099279F938F9387EE9DE09F938F93FF926E
:10F7B000EF92E0911304F0911404099585E70E94FB
:10F7C000F18A2DB73EB72A5F3F4F2DBF8091990137
:10F7D00099279F938F9300E610E01F930F938091DA
:10F7E0006C0890916D089F938F9382EF9DE09F939B
:10F7F0008F93FF92EF92E0911304F0911404099516
:10F8000082E70E94F18A8DB79EB70A968DBF8091DC
:10F81000C30399279F938F931F930F938091C403E2
:10F8200099279F938F938EEF9DE063C689E60E9490
:10F83000F18A8091990199279F938F9380E690E0B8
:10F840009F938F9380916C0890916D089F938F93F5
:10F850008091690899279F938F938EE09EE09F93F4
:10F860008F93FF92EF92E0911304F09114040995A5
:10F870008DB79EB70C967DC585E04CC39091C603AD
:10F880009923D1F08091FD03882381F09E3170F49B
:10F8900087E00E948D7683E90E94F18A8091C603F9
:10F8A00099279F938F9387E29EE09EC383E90E94EE
:10F8B000F18A82E39EE0ADC383E90E94F18A88E386
:10F8C0009EE0CEC30E94A576809342098091220AD1
:10F8D000863059F48091F603882319F01092F603CC
:10F8E00099C681E08093F60395C6883009F092C6E8
:10F8F0000E94F68A81E0D5C39093F30393C69130BA
:10F9000009F0DAC38091F303282F332744275527C2
:10F910008F5F8093F303F9012131310508F07DC633
:10F92000EF56FF4F0C9459918091B40285FF43C06C
:10F9300080E00E94F18A8091E4089091E5089F930D
:10F940008F9380912501909126016AE070E00E94DA
:10F95000D2909F938F9380912501909126016AE028
:10F9600070E00E94D2907F936F938091B00190914C
:10F97000B1016CE370E00E94BE909F938F938091E1
:10F98000B0019091B1016CE370E00E94BE907F9352
:10F990006F938EE49EE09F938F9384EE9AE89F93FB
:10F9A0008F93E0911304F091140409952DB73EB79D
:10F9B000225F3F4FABC580E00E94F18A8091E4084E
:10F9C0009091E5089F938F93809125019091260156
:10F9D0006AE070E00E94D2909F938F9380912501FE
:10F9E000909126016AE070E00E94D2907F936F931D
:10F9F0008091B0019091B1016CE370E00E94BE90E3
:10FA00009F938F938091B0019091B1016CE370E06E
:10FA10000E94BE907F936F9389E69EE0C6C285E107
:10FA20000E94F18A80E690E09F938F9380919601E7
:10FA3000909197019F938F9384E89EE09F938F937B
:10FA4000C3ECDAE8DF93CF93E0911304F091140450
:10FA5000099580914B082DB73EB7285F3F4F2DBFCA
:10FA600080FF51C080910303882339F18FE10E9408
:10FA7000F18A8091E6029091E702A091E802B091AC
:10FA8000E902BC01CD0124E630E040E050E00E94F4
:10FA900007913F932F938EE89EE09F938F9383ED82
:10FAA0009AE89F938F93E0911304F09114040995C1
:10FAB0008DB79EB706968DBF38C08FE10E94F18A40
:10FAC0008091E6029091E702A091E802B091E902EC
:10FAD000BC01CD0124E630E040E050E00E940791F7
:10FAE0003F932F9387E99EE09F938F93DF93CF936C
:10FAF000E0911304F091140409952DB73EB72A5FE5
:10FB00003F4F2DBF12C08FE10E94F18A80EA9EE034
:10FB10009F938F93DF93CF93E0911304F09114049C
:10FB200009950F900F900F900F9089E20E94F18A33
:10FB30008091490199279F938F938AEA9EE09F9332
:10FB40008F93DF93CF930DC48091A3018823F9F0A5
:10FB50008BE20E94F18A8091990199279F938F935C
:10FB600080916A0890916B086AE070E00E94BE90F4
:10FB70007F936F9380E690E09F938F9380916C08C2
:10FB800090916D089F938F938DEA9EE05CC182E017
:10FB9000C1C18FE30E94F18A8091E2089091E3084D
:10FBA0009F938F938091E0089091E1086AE070E064
:10FBB0000E94BE909F938F938091E0089091E108FE
:10FBC0006AE070E00E94BE907F936F9384EC9EE0A9
:10FBD0009F938F93C3ECDAE8DF93CF93E091130404
:10FBE000F091140409958091B3022DB73EB7265FBA
:10FBF0003F4F2DBF80FF0AC082E50E94F18A88ED49
:10FC00009EE09F938F9383ED9AE8D6C482E50E948D
:10FC1000F18A8BED9EE03BC38091A301B3ECEB2E08
:10FC2000BAE8FB2E882309F449C084E50E94F18AD2
:10FC30008091670899279F938F93809169089927EE
:10FC40009F938F938EED9EE09F938F93E701FF929A
:10FC5000EF92E0911304F091140409958DB79EB7CB
:10FC600008968DBF80916808833051F484E60E9425
:10FC7000F18A81EF9EE09F938F93FF92EF920BC0EA
:10FC800084E60E94F18A87EF9EE09F938F9384EE33
:10FC90009AE89F938F93E0911304F09114040995CF
:10FCA0000F900F900F900F908091660881FFBAC45B
:10FCB00084E60E94F18A8DEF9EE0E9C284E50E940D
:10FCC000F18A83E09FE09F938F93FF92EF9276C437
:10FCD0008091F503A3ECEA2EAAE8FA2E882309F412
:10FCE00050C089E60E94F18A80914E076AE00E9426
:10FCF000B290892F99279F938F9380914E070E94EE
:10FD0000B29099279F938F93809146070E94B2905B
:10FD1000892F99279F938F93809146070E94B290D5
:10FD200099279F938F9380913E070E94B290892FCD
:10FD300099279F938F9380913E070E94B2909927B5
:10FD40009F938F93809136070E94B290892F9927B5
:10FD50009F938F93809136070E94B29099279F932B
:10FD60008F9389E19FE09F938F93FF92EF92E091B1
:10FD70001304F091140409952DB73EB72C5E3F4F44
:10FD8000C5C389E60E94F18A80E690E09F938F9335
:10FD900080915007992787FD90959F938F9380912D
:10FDA0004807992787FD90959F938F9380914007EF
:10FDB000992787FD90959F938F9380913807992776
:10FDC00087FD90959F938F9386E39FE09F938F93FA
:10FDD000FF92EF92E0911304F091140409958DB70E
:10FDE0009EB70E96C6C28091F50390915E06882359
:10FDF00009F48DC0943009F48CC09630A1F58EE7DB
:10FE00000E94F18A80915E076AE00E94B290892F79
:10FE100099279F938F9380915E070E94B2909927B4
:10FE20009F938F93809156070E94B290892F9927B4
:10FE30009F938F93809156070E94B29099279F932A
:10FE40008F9389E49FE09F938F9383EC9AE89F932D
:10FE50008F93E0911304F091140409952DB73EB7E8
:10FE6000245F3F4F53C3973008F4DCC38EE70E94F2
:10FE7000F18A80916E076AE00E94B290892F9927DB
:10FE80009F938F9380916E070E94B29099279F93C2
:10FE90008F93809166070E94B290892F99279F9334
:10FEA0008F93809166070E94B29099279F938F93BA
:10FEB00080915E070E94B290892F99279F938F931C
:10FEC00080915E070E94B29099279F938F938091B3
:10FED00056070E94B290892F99279F938F93809104
:10FEE00056070E94B29099279F938F9388E59FE0D1
:10FEF0009F938F9383EC9AE89F938F93E0911304E1
:10FF0000F091140409958DB79EB7449632C294308F
:10FF100021F486E00E948D7685C39630F1F48EE759
:10FF20000E94F18A80E690E09F938F938091600712
:10FF3000992787FD90959F938F93809158079927D4
:10FF400087FD90959F938F9385E79FE09F938F9375
:10FF500083EC9AE89F938F93D0C2973008F462C3E2
:10FF60008EE70E94F18A80E690E09F938F938091C4
:10FF70007007992787FD90959F938F9380916807CD
:10FF8000992787FD90959F938F938091600799277C
:10FF900087FD90959F938F9380915807992787FDB0
:10FFA00090959F938F9388E89FE09F938F9383EC26
:10FFB0009AE89F938F930ECF9091C603992309F4EB
:10FFC0004AC08091FD038823F9F09E31E8F487E070
:10FFD0000E948D7683E90E94F18A8091C603992759
:10FFE0009F938F938BE99FE09F938F9383ED9AE884
:10FFF0009F938F93E0911304F091140409952DB70A
:020000021000EC
:100000003EB72A5F3F4F82C283E90E94F18A86EAA7
:100010009FE09F938F9303EC1AE81F930F93E09157
:100020001304F091140409951F921F929091C60336
:1000300081E1989FC00111248D5F944F9F938F930E
:100040001F930F93E0911304F091140409958DB759
:100050009EB70A968EC183E90E94F18A8CEA9FE0DE
:100060009F938F9383EC9AE8A7C20E94A576809312
:1000700042098091220A863079F48091F503882321
:1000800019F01092F50303C081E08093F50385E039
:100090000E948D7686E0B3C2883031F40E94F68AE1
:1000A00082E08093F403B4C2813009F0B3C20E94AD
:1000B000F68A1092F403ACC2923009F0B1C280917A
:1000C000F303282F3327442755278F5F8093F303AB
:1000D000F9012131310508F0A0C2EE55FF4F0C9413
:1000E000599180E00E94F18A8EEC96E09F938F9365
:1000F0000E94823299279F938F9382EC9FE09F9377
:100100008F9383ED9AE89F938F93E0911304F0917E
:10011000140409952DB73EB7285F3F4FF7C185E11D
:100120000E94F18A8CED96E09F938F93809100015D
:100130006AE00E94B290892F99279F938F938091B4
:1001400000010E94B29099279F938F9381ED9FE0C9
:100150009F938F9383EC9AE89F938F93E09113047E
:10016000F0911404099573CF8AE20E94F18A82EE1D
:100170009FE09F938F93C3ECDAE8DF93CF93E091F6
:100180001304F0911404099580914B080F900F907F
:100190000F900F9080FF41C080916C06909181017B
:1001A00081FD0BC0892F99279F938F9387EE9FE046
:1001B0009F938F93DF93CF931DCFE0911304F09122
:1001C0001404933318F081EF9FE002C088EF9FE0A2
:1001D0009F938F93DF93CF9309950F900F900F907C
:1001E0000F9080912F08E0911304F09114049091E6
:1001F000810180FF0BC0892F99279F938F938FEFE9
:100200009FE09F938F93DF93CF93AFC0892F992760
:100210009F938F9385E090E1CFC08BE090E137C052
:100220008FE30E94F18A84E190E19F938F93C3EC66
:10023000DAE8DF93CF93E0911304F0911404099569
:100240000F900F900F900F908091C106882319F4A2
:1002500088E190E11CC08091C102E0911304F0910B
:100260001404882319F081E290E102C088E290E151
:100270009F938F93DF93CF9309950F900F900F90DB
:100280000F908091CC0686FFCDC18FE290E19F93C5
:100290008F93DF93CF9392C184E50E94F18A86E326
:1002A00090E19F938F93C3ECDAE8DF93CF93E091D3
:1002B0001304F0911404099580914B080F900F904E
:1002C0000F900F9085FD03C08BE390E111C08091EA
:1002D000AF06883F10F4E82F07C0EFEFF0E0E81B0F
:1002E000F109E351FD4FE081E23358F484E490E1F9
:1002F0009F938F93DF93CF93E0911304F0911404B5
:1003000016C0E43B18F08BE490E1F2CF8091CC066C
:10031000E0911304F091140485FF03C082E590E19D
:1003200002C089E590E19F938F93DF93CF93099566
:100330000F900F900F900F908091C506882309F4BD
:1003400071C18EE50E94F18A8091C50699279F931D
:100350008F9380E690E19F938F9383EC9AE89F932D
:100360008F93E0911304F091140409958DB79EB713
:1003700006968DBF57C189E60E94F18A8BE690E10F
:100380009F938F93C3ECDAE8DF93CF93E09113044C
:10039000F091140409950F900F900F900F90809199
:1003A000C406E0911304F0911404882351F09927B6
:1003B0009F938F9385E790E19F938F93DF93CF93E4
:1003C0001DCE89E790E19F938F93DF93CF93FAC07F
:1003D0008091F703F3ECEF2EFAE8FF2E882309F063
:1003E00053C08EE70E94F18A8091750199279F93EF
:1003F0008F9380916106E82FFF27EE0FFF1FEE56C7
:10040000F84F808191819F938F9380916006E82FB0
:10041000FF27EE0FFF1FEE56F84F808191819F93CB
:100420008F938FE790E19F938F93FF92EF92E091EC
:100430001304F0911404099583E90E94F18A8DB7A1
:100440009EB70A968DBF80916306E82FFF27EE0FB7
:10045000FF1FEE56F84F808191819F938F9380917B
:100460006206E82FFF27EE0FFF1FEE56F84F808140
:10047000918181589F4F9F938F9383E990E19F9340
:100480008F93FF92EF9241CE8EE70E94F18A809186
:10049000EF0299279F938F938091EE0299279F9364
:1004A0008F938091ED0299279F938F9382EA90E139
:1004B0009F938F93FF92EF92E0911304F0911404B5
:1004C000099583E90E94F18A8DB79EB70A968DBF80
:1004D0008091F20299279F938F938091F10299273F
:1004E0009F938F938091F00299279F938F9386EB30
:1004F00090E19F938F93FF92EF92E0911304F0911C
:10050000140409952DB73EB7265F3F4F2DBF8AC013
:100510008091FD03882309F485C08EE70E94F18A4B
:1005200080914B0886FD11C08AEC90E19F938F93D8
:1005300084EE9AE89F938F93E0911304F091140452
:1005400009950F900F900F900F908091CA069927F0
:100550008F709070892B89F089ED90E19F938F9334
:1005600084EE9AE89F938F93E0911304F091140422
:1005700009950F900F900F900F9080914B0882FF7C
:1005800011C083EE90E19F938F9384EE9AE89F933E
:100590008F93E0911304F091140409950F900F903C
:1005A0000F900F9080914B0883FD3CC088EE90E146
:1005B0009F938F9384EE9AE89F938F93E091130417
:1005C000F091140409950F900F900F900F902AC08E
:1005D0000E94A5768093420925C00091220A063028
:1005E00089F48091F703882319F01092F70303C070
:1005F00081E08093F70386E00E948D7687E00E9479
:100600008D7608C0013031F40E94F68A0093F4031D
:100610001092F3031092220A05C01092F30302C055
:100620001092F403E6E0CDB7DEB70C944A914FB7D1
:1006300028E130E0F8948091C9008F778093C90059
:100640008091C9008F7B8093C9008091C9008F7D04
:100650008093C9005A9A52985B9A539A832F99278C
:100660008093CD002093CC008091C800826080935D
:10067000C80080E18093C9008091CA008F77809381
:10068000CA008091CA008F7B8093CA008091CA0003
:100690008091CA008F7E8093CA008091CA008860D2
:1006A0008093CA008091C9008B7F8093C90080919C
:1006B000CA0084608093CA008091CA0082608093DF
:1006C000CA008091C80087FF03C08091CE00F9CF97
:1006D0008091C90080688093C9008091200A84605D
:1006E0008093200A4FBF08959091D703992341F436
:1006F0008F3031F49093F90380E58093D703089508
:10070000E091F903EF5FE093F903E83121F481E030
:100710008093F8030895E93120F089E18093F9038B
:100720000895FF27E75FF54F80830895A0E0B0E0CC
:10073000ECE9F3E80C942A9191E0D92E82E0A82EFE
:10074000BD2CE12C01E0F02E8091200A82FDB5C085
:1007500080916F008F7D80936F00E091C706EE233C
:1007600051F0FF27EE0FFF1FEE56F84F8081918169
:10077000843691055CF48091EC02883C20F48091F1
:10078000EC028C5E01C088EC8093EC0280910A0A36
:10079000682F77278091FA0381508093FA038F3F67
:1007A00031F41CE7C12E82E08093FA0302C0C4E258
:1007B000CC2E40E04C1508F07EC0EA2DFF27E75F05
:1007C000F54F80818D2111F06E297F298D2D99277C
:1007D000880F991FD82E882319F4B1E0DB2EAD0CB9
:1007E000EE0CFF1C20E0E21628E0F20609F061C0E2
:1007F000A1E0EA2EF12CCB018050944065E070E03E
:100800000E94D290AB2DBB27FD01EA0FFB1FEE56D5
:10081000F84F808191819C01220F331F280F391FCF
:10082000260F371F37FF02C02D5F3F4FE901D595D7
:10083000C795D595C795CB0101968C179D0714F4E4
:10084000219706C061507040C617D7070CF4219657
:100850008091EC02833CD8F08D010A0F1B1FF80138
:10086000EE56F84F80819181FE01E81BF90BCF0114
:1008700063E070E00E94D290CB01880F991F860F31
:10088000971F0A53184FF8019183808307C0AA0F5E
:10089000BB1FAA53B84F11961C921E92EB2DFF2737
:1008A000EE0FFF1FEE56F84FD183C08360E070E07B
:1008B000B3944F5F7FCF109248011092F803EAE0A3
:1008C000CDB7DEB70C9446910895089500242227F1
:1008D0003327442751E0BB27EE27FF27A0E1660F0F
:1008E000771F881F991F001C221F331F441F660F8C
:1008F000771F881F991F001C221F331F441F2AF4D3
:10090000050E2B1F3E1F4F1F04C0051A2B0B3E0B5D
:100910004F0B550FBB1FEE1F587F556047FD5250C0
:10092000AA95E9F6E695B7955795E695B795579543
:10093000852F9B2F08952227332741E0552768E014
:10094000880F991F221F331F880F991F221F331FE3
:100950001AF4240F351F02C0241B350B440F551FFA
:10096000487F456037FD42506A9551F75695479547
:1009700056954795842F0895AA2797FF04C0809520
:1009800090958A1F9A1F77FF04C0609570956A1F23
:100990007A1F669F9001779FA001679F300D411DD0
:1009A0005A1F300D411D5A1F889FF001999F2E0F2D
:1009B0003F1F401D511D899F300D411D5A1F300D95
:1009C000411D5A1FCA01B901112480CF4FB720E43D
:1009D00030E0F8948091C9008F778093C9008091AE
:1009E000C9008F7B8093C9008091C9008F7D80935F
:1009F000C9005A9A52985B9A539A832F99278093E9
:100A0000CD002093CC008091C80082608093C80004
:100A100088E18093C9008091CA008F778093CA00D3
:100A20008091CA008F7B8093CA008091CA008F7D1D
:100A30008093CA008091CA008F7E8093CA00809103
:100A4000CA00877F8093CA008091C9008B7F809302
:100A5000C9008091CA0084608093CA008091CA0056
:100A600082608093CA008091C80087FF03C0809194
:100A7000CE00F9CF8091C90080688093C9004FBF34
:100A800008950F931F93CF93DF93482F4F5F8931C2
:100A900008F08BC080919107841720F44F5F40933A
:100AA00091074150CB0183539B4268E170E00E9463
:100AB000D290A42FBB27FD01EA0FFB1FEE56F84F83
:100AC000808191819B01281B390BC90137FF03C02D
:100AD000909581959F4F069794F48091EC02883C05
:100AE00030F48091EC02865F8093EC0208C088ECC1
:100AF0008093EC0280916F008F7D80936F00FD01E9
:100B0000EA0FFB1FEE56F84F808191819C01220F66
:100B1000331F280F391F260F371F37FF02C02D5FE5
:100B20003F4FE901D595C795D595C795CB0101965E
:100B30008C179D0714F4219706C061507040C617AA
:100B4000D7070CF421968091EC02843BD8F08D01FC
:100B50000A0F1B1FF801EE56F84F80819181FE01AC
:100B6000E81BF90BCF0163E070E00E94D290CB014B
:100B7000880F991F860F971F0A53184FF80191830A
:100B8000808307C0AA0FBB1FAA53B84F11961C92AF
:100B90001E92E42FFF27EE0FFF1FEE56F84FD18372
:100BA000C083443011F410924801DF91CF911F911E
:100BB0000F910895CF93DF932091230A822F9927D5
:100BC000807F9070409709F06CC02F3109F046C0CB
:100BD0008091240A809304042091260A209306041D
:100BE0008091270A80930504822F99279093930779
:100BF00080939207222309F054C080916006282F29
:100C00003327220F331FF901EA53F84F1182108264
:100C100080916106A82FBB27AA0FBB1FFD01EA53D5
:100C2000F84F1182108280916306E82FFF27EE0FA4
:100C3000FF1FCF018A53984FEC01198218822E565C
:100C4000384FE90119821882AE56B84F11961C929E
:100C50001E92EE56F84F1182108223C0C22FCF7021
:100C6000CA30F8F48091240A80934F0A8091250AB3
:100C700080934E0A8091260A8093510A8091270A18
:100C80008093500A60914E0A70914F0A8C2F0E94F7
:100C900041856091500A7091510A8C2F8F5F0E949C
:100CA0004185DF91CF910895CF93C82F8F3F49F4AD
:100CB000809107048F3F29F41092090410920804D0
:100CC00032C020910904222339F4CF3111F485E098
:100CD00001C084E080930A0480910A049091080482
:100CE0008217A0F4892F8095809308048F3F19F410
:100CF0008EEF8093080480910804C81711F40E94B5
:100D0000DA8510920904109208040BC0E22FFF2725
:100D1000ED5DF54FC0832F5F209309049C0F9093E6
:100D20000804C0930704CF9108959091030493326F
:100D300040F4E92FFF27E55DF54F80839F5F909397
:100D400003040895833218F48D5F8093030408959B
:100D500090E2EEE2FAE08FE19193815087FFFCCFC1
:100D60000895CF93CFB723E031E0F8948091C90084
:100D70008F778093C9008091C9008F7B8093C900D1
:100D80008091C9008F7D8093C9005A9A52985B9ACE
:100D9000539A832F99278093CD002093CC00809184
:100DA000C80082608093C80088E18093C900809168
:100DB000CA008F778093CA008091CA008F7B80938E
:100DC000CA008091CA0080628093CA008091CA00E4
:100DD00080618093CA008091CA0088608093CA00B5
:100DE0008091C90084608093C9008091CA008460AA
:100DF0008093CA008091CA0082608093CA0080916B
:100E0000C80087FF03C08091CE00F9CF8091C90050
:100E100080688093C9008091C90080648093C90074
:100E20000E94A886CFBFCF910895282F99278F7051
:100E30009070892B31F4209580910204822B80934D
:100E4000020408958091AB01882309F44BC080917E
:100E5000B40285FD04C08091AE01882381F082E94F
:100E600080932B0A83E280932C0A8091AE01882321
:100E700009F485E580932D0A1092AE0102C080939B
:100E80002B0A8091AC018F3071F4809102040E9492
:100E90002375882341F081E980932B0A80932C0AE3
:100EA00081E380932D0A1092AB018091C80085FFE9
:100EB000FCCF8091C9008F7E8093C9008091C900CA
:100EC0008E7F8093C90080912B0A882311F48EEFC6
:100ED00001C08EE78093CE00809102048093AC0124
:100EE0001092020408951F920F920FB60F921124D0
:100EF0008F939F93EF93FF939091AB01992309F008
:100F000040C080910B04882361F480912B0A8823D0
:100F100011F483E003C0813999F481E080930B04DC
:100F20000FC0833099F480912B0A882349F0909365
:100F30002B0A8091C9008E7F8093C9008EEF1EC05E
:100F40008091C90081608093C9000EC0833261F432
:100F50008091C9008E7F8093C9008FEF8093CE006F
:100F600081E08093AB0114C080910B04E82FFF2730
:100F7000E55DF54F8F5F80930B0480818093CE00F9
:100F800007C010920B048091C90080618093C90052
:100F9000FF91EF919F918F910F900FBE0F901F9037
:100FA0001895EF92FF920F931F93CF93DF937C01DD
:100FB0008B01EA01452B39F0F80181918F01F7018E
:100FC00009952197C9F7E6E0CDB7DEB70C944A91B1
:100FD000EF92FF920F931F93CF93DF937C018B01CE
:100FE000EA01452B41F0F8010F5F1F4F8491F70193
:100FF00009952197C1F7E6E0CDB7DEB70C944A9189
:101000000F931F93CF938C01C62F161634F480E2F2
:10101000F8010995C1501C16D4F3CF911F910F917F
:1010200008950F931F93CF938C01C62F161634F497
:1010300080E3F8010995C1501C16D4F3CF911F919C
:101040000F910895A5E3B0E0E8E2F8E80C9422914E
:101050002E96EEADFFAD2E978824992454018091F1
:10106000FC03882321F42C961FAE1EAE2C975EE461
:10107000452E512C4C0E5D1E6F01B60105C0153278
:1010800039F00894C11CD11CF60114911123B9F751
:10109000A601461B570B31F02C968EAD9FAD2C97B9
:1010A0000E94E887112309F46AC20894C11CD11C6C
:1010B000FF24FDA6FCA64FEFE42EF9A6F601089446
:1010C000C11CD11C1491153721F0812F8062883703
:1010D000B1F4F0FE0AC0F20124E030E0420E531EEB
:1010E00080809180A280B3800AC0F20142E050E08B
:1010F000440E551E808191814C01AA24BB241032DC
:1011000021F489A58823D1F61DC0133219F458E0C3
:10111000F52AD4CF1A3211F01D3291F41A3259F453
:10112000F20182E090E0480E591EE081ECA7EE2328
:101130002CF6E195ECA790E1F92AAFEDFA22BECFAB
:101140001B3211F419A7BACF1E32C1F5F60108946B
:10115000C11CD11C14911A3279F4F20122E030E062
:10116000420E531E408151813FEF4F3F530714F40D
:101170004FEF5FEFE42EA2CF40E050E0812F80538D
:101180008A30A0F4CA0133E0880F991F3A95E1F73D
:10119000840F951F480F591F410F511D4053504058
:1011A000F6010894C11CD11C1491E8CF8FEF4F3F7A
:1011B000580714F44FEF5FEFE42E85CF103329F476
:1011C000F4FC7CCF90E2F92A79CF812F81538930CA
:1011D000D8F440E050E0CA0123E0880F991F2A9517
:1011E000E1F7840F951F480F591F410F511D4053C0
:1011F0005040F6010894C11CD11C1491812F8053DA
:101200008A3048F34CA75FCF183619F4A4E0FA2AC5
:1012100055CF1C3619F4B1E0FB2A50CF133661F4D8
:101220003E010894611C711CF20122E030E0420E84
:10123000531E808189833CC1143421F0143611F08F
:10124000193651F5143411F431E0F32AF0FE0AC0D6
:10125000F20144E050E0440E551E80809180A2804F
:10126000B3800CC0F20182E090E0480E591E8081EC
:1012700091814C01AA2497FCA094BA2CB7FE0AC015
:10128000B094A09490948094811C911CA11CB11CDA
:101290008DE289A70AE06FC01F3411F01F3631F4C8
:1012A0001F3411F491E0F92A08E064C0103779F492
:1012B000F201A2E0B0E04A0E5B1E808191814C01F8
:1012C000AA24BB2400E1B0E4FB2A18E753C013377B
:1012D000C1F5F20122E030E0420E531E60807180C1
:1012E0006114710489F43E010894611C711C88E248
:1012F00089838EE6F301818385E78B838CE68C837B
:101300008D8389E28E831F82E7FC13C08E2D99277F
:1013100087FD9095AC0160E070E0C3010E94EF8E04
:10132000009729F0382E3618E3140CF0C3C03E2C79
:10133000C1C0F30101900020E9F731973E2E361825
:10134000B9C0153511F0153731F4153511F4F1E048
:10135000FF2A0AE00FC0183519F0183709F0A0C0AD
:1013600000E1F3FE07C081149104A104B10411F05F
:1013700020E4F22A19A6EDA6E7FC02C03FEDF32215
:1013800089E2682E712C6C0E7D1E81149104A104DB
:10139000B10421F44DA5442309F47BC0802F992783
:1013A000AA27BB278EA79FA7A8ABB9AB202E3324B3
:1013B00090E0891690E0990691E0A90690E0B906C0
:1013C00048F0C501B4012EA53FA548A959A90E941E
:1013D000E59017C0AFEF8A169104A104B10449F05B
:1013E00040F0C401B1010E94BE909B0144275527E3
:1013F00008C0882D602F0E94B290282F33274427E1
:1014000055272AAB3BAB4CAB5DAB0A3059F48AA9EC
:10141000880F880F880F9AA9990F890F382D381BCC
:10142000832F10C0003139F48AA98295807F482D1E
:10143000481B842F07C08AA9880F880F880F582D52
:10144000581B852F90E02EA53FA548A959A98216C3
:101450009306A406B50608F091E08AA89BA8ACA85C
:10146000BDA88A3010F4805D04C0895A183509F48B
:101470008F7DD3018E933D01992309F099CF0830D8
:1014800041F4F3FE06C0803321F080E3FD01829336
:101490003F01CE010196382E3618F8E23F0E0BC000
:1014A000112309F46CC03E010894611C711C19835E
:1014B000B1E03B2E19A6032D2DA4231827FC2224CE
:1014C00089A5882311F00F5F02C0F6FC0E5F020DA4
:1014D000EF2CFF24C70180739070892B49F48CA5F1
:1014E000801B682F2C968EAD9FAD2C970E94008894
:1014F00089A5882331F041E050E0BE01675D7F4F50
:101500000AC0E6FE0EC080E38AA71BA742E050E0B7
:10151000BE01665D7F4F2C968EAD9FAD2C970E94CD
:10152000D187C70180739070809749F48CA5801B88
:10153000682F2C968EAD9FAD2C970E941188622D3E
:101540002C968EAD9FAD2C970E941188832D9927E4
:1015500087FD9095AC01B3012C968EAD9FAD2C9775
:101560000E94D187E4FE89CD2CA5201B2CA7622FD9
:101570002C968EAD9FAD2C970E9400887ECDE2E127
:10158000CB5C0C943E91982F80912A0A883A50F4B3
:1015900080912A0AE82FFF27E05CF64F93838F5F44
:1015A00080932A0A0895982F80912A0A883A58F43D
:1015B00080912A0AE82FFF27E05CF64F906893831A
:1015C0008F5F80932A0A0895982F8091FD038823C6
:1015D00021F0892F0E94D38A0895892F0E94C38AFF
:1015E0000895883A10F480932A0A089580E090E2E2
:1015F000E3E4F9E091938F5F883AE0F308954FB701
:1016000021E830E0F8948091C9008F778093C90079
:101610008091C9008F7B8093C9008091C9008F7D24
:101620008093C9005A9A52985B9A539A832F9927AC
:101630008093CD002093CC008091C800826080937D
:10164000C80088E18093C9008091CA008F77809399
:10165000CA008091CA008F7B8093CA008091CA0023
:101660008F7D8093CA008091CA008F7E8093CA00CC
:101670008091CA00877F8093CA008091C9008460EE
:101680008093C9008091CA0084608093CA008091D1
:10169000CA0082608093CA008091C90081608093F3
:1016A000C9008091C80087FF03C08091CE00F9CFA8
:1016B0008091C90080688093C9004FBF3CE7309398
:1016C000E7082DE720930C098EE88093E808109234
:1016D0000109109200091092EA0830932F09209313
:1016E0003F09109239091092380910923B09109263
:1016F0003A0910923D0910923C0984EF91E09093D1
:101700003709809336099093350980933409909373
:101710003309809332091092310989E880933009A6
:1017200010923E093093EC092093080A1092EE09BA
:101730008AE88093ED091092F1091092F009109255
:10174000EF091092F3091092F4091092F509109222
:10175000F6091092F8091092F9091092FA091092FC
:10176000FB091092FF091092FE091092FD091092D8
:10177000FC0930930D0920932E0910920F098DE872
:1017800080930E098BE78093400980E8809341099C
:10179000109242098091EA0890E2E3E4F9E0919323
:1017A0008F5F883AE0F38DE78093EB090895CF933C
:1017B000C82F80910C04803879F48C2F0E945B77BD
:1017C0008093FF038091FF03882311F1C093290ABE
:1017D0008091FF038F5F12C08F37D1F48091220A6E
:1017E000882329F48C2F80958F708093220A80E4BF
:1017F00099E090930104809300048DEA8093FF03A5
:101800008091C9008F7E8093C90082E08093FE039F
:10181000C0930C04CF9108953091FE03332331F02F
:101820008091FE0381508093FE0308958091FF0311
:10183000882381F14091FF0390910D04413091F490
:10184000292F30930D048091C90080618093C900D5
:101850008091FD03882319F03093FD0310C040935D
:10186000FD030DC0E0910004F09101048191F0931B
:101870000104E0930004282F980F90930D048091A9
:10188000C80085FFFCCF2093CE008091FF038150DC
:101890008093FF0308952FB740E0F894E0E0F0E074
:1018A00081E2809357009491E2E0F0E0809357004A
:1018B0003491E4E0F0E08093570084912FBF9E3193
:1018C00099F4363941F4893011F441E00DC08A3081
:1018D00059F442E009C0373939F4863011F443E055
:1018E00003C0853009F444E0842F992708959FB7F9
:1018F000F8948091C900877F8093C9008091C900C6
:101900008F7E8093C9008091C9008F778093C90032
:101910008091C9008F7B8093C9008091C9008F7D21
:101920008093C90052985A9A53985B9A9FBF089522
:101930001F93CF93DF93182F8091FC03882309F422
:10194000A7C08091AA01181709F4A2C08091FB03D7
:10195000882321F40E944B8C8093FB0382ED91E05D
:10196000909347018093460185E991E19F938F937E
:10197000C7E6D5E1DF93CF93E0911304F09114040F
:1019800009950F900F900F900F90812F9927AA27FC
:10199000BB27FC01099778F5ED54FF4F2091130404
:1019A000309114040C94599181E991E102C088E8C6
:1019B00091E19F938F93DF93CF93F901099527C00E
:1019C00083E891E1F6CF8BE791E1F3CF83E791E1F3
:1019D0009F938F93DF93CF93F901099588ED91E061
:1019E000909347018093460112C08EE691E1E1CFCA
:1019F00082EA91E1DECF88EA91E19F938F93DF93B2
:101A0000CF93E0911304F0911404099510E00F9026
:101A10000F900F900F908091FB03843011F0823073
:101A200011F50E94778C812F8150833018F40E9429
:101A300019702CC0143019F40E94B18627C01530DB
:101A400019F40E94E68422C0183019F40E946484BC
:101A50001DC0163019F40E94FF8A18C01730B1F467
:101A60000E94178313C0112389F08EEB91E19F939D
:101A70008F9387E695E19F938F93E0911304F09104
:101A8000140409950F900F900F900F901093AA01D6
:101A9000DF91CF911F9108950F931F9381E0809361
:101AA000FC034091A901EEE1F1E120E030E05FE4C8
:101AB000849199272F5F3F4F829FB001839F700DC4
:101AC000929F700D112446275150319657FFF0CF49
:101AD0004093A901E6EFF0E120E030E057E2849185
:101AE00099272F5F3F4F829FB001839F700D929F78
:101AF000700D112446275150319657FFF0CF409377
:101B0000A9018091FB03882321F40E944B8C8093D0
:101B1000FB038091A901833459F088E190E029E228
:101B20000FB6F894A895809360000FBE20936000D4
:101B300082E298E890931404809313040E94580959
:101B400085E690E09F938F9388E590E09F938F9335
:101B50001F921F92809101016AE00E94B290892F2A
:101B600099279F938F93809101010E94B2909927AA
:101B70009F938F9389ED91E19F938F9307E615E1F2
:101B80001F930F93E0911304F091140409958EE1D3
:101B900091E19F938F931F930F93E0911304F09122
:101BA0001404099586EF90E19F938F931F930F93F1
:101BB000E0911304F091140409950E94580983ECF4
:101BC0008093810080916F00806280936F008DB759
:101BD0009EB746968DBF1F910F9108958091C506BF
:101BE0008D3338F08091660887FD03C08CE38093C5
:101BF000C50680917506882331F08055853618F02A
:101C00008FE78093750608958091FC03882309F47B
